:10000000FCFB0220D1010000B902010071020100D5
:100010007102010071020100710201007102010010
:10002000710201007102010071020100B9020100B8
:10003000B9020100710201002924010079260100A2
:10004000B9020100B9020100B9020100B9020100C0
:10005000B9020100B9020100B9020100B9020100B0
:10006000B9020100B9020100B9020100B9020100A0
:10007000B9020100B9020100B9020100B902010090
:10008000B9020100B9020100B9020100B902010080
:10009000B9020100B9020100B9020100B902010070
:1000A000A5FE0000B9FE0000B9020100B90201007E
:1000B000491CFF1FB9020100B90201001928010003
:1000C000B9020100352A0100B9020100512C0100DA
:1000D000B9020100512D0100B90201007DFE0000AE
:1000E000B9020100B9020100B9020100B902010020
:1000F000B9020100B9020100B9020100B902010010
:10010000B90201003107FF1FB9020100B902010065
:10011000B9020100DD100100B9020100B9020100BD
:10012000B9020100B9020100B9020100B9020100DF
:10013000B9020100B9020100B9020100B9020100CF
:10014000B9020100B9020100512E0100B9020100FB
:10015000B9020100B9020100B9020100B9020100AF
:10016000B902010091FE0000CDFE0000B9020100BD
:10017000B9020100B9020100B9020100B90201008F
:10018000B902010001FF0000B9020100B90201003B
:10019000B9020100B9020100512F0100B9020100AA
:1001A000B9020100B9020100B9020100E1FE00003C
:1001B000B9020100B9020100B9020100B90201004F
:1001C000B9020100B9020100B9020100B90201003F
:1001D000614B4CF220524DF6281010B51A80188051
:1001E00000BF00BF5D4C10F06BF84FF03061216034
:1001F0005B4B5C49A3604FF470005B4A5B4BE26071
:1002000008605B4C5B481C6090F800C05FEA0C71B2
:1002100004D590F800E04EF008020270564C574AA0
:10022000574BAA212170574CA34204D252F8040F15
:1002300043F8040BF8E7544954480024814202D2A1
:1002400041F8044BFAE75249524A002352F823007E
:1002500041F823000133742BF8D14F4C4F498023D0
:1002600004F8013B8C42FBD14D4B4E48484A02609A
:10027000A3F5805C8A242421A0221C708CF8011034
:100280008CF800209CF806008207FBD59CF80640FD
:10029000E406FBD4444991F806E00EF00C03082B69
:1002A000F9D142486022027002300478802CFCD1DF
:1002B0003D4B01215D2219715A7198798006FCD558
:1002C00093F806C0384C5FEA4C61F9D5384B394990
:1002D0001960002220205A602070A17901F00C03DF
:1002E0000C2BFAD1344A354C354814600168354C32
:1002F00011F4807303D14FF4A85223600260324995
:10030000324808600023072231484B6041F8042C32
:10031000C1F80C0D62B610F0EFF82468E20705D5BD
:100320002C4810F0D7F82C4B2C4919602C4A107827
:10033000430609D5284C294B2168994204D1254808
:1003400010F0C8F80022226013F0BEFC0FF0BEFFD0
:100350000FF0EEFEFEE700BF0E20054030800440A7
:10036000823F040088ED00E00100002B002008E03F
:100370000300008502D0074000E00740383A04003F
:100380003007FF1F8833FF1F8833FF1F18E5012048
:100390000002FF1F0000000000E400E064E400E051
:1003A0000050064008ED00E00040064001E0074034
:1003B000448004400000060204800440C01007008E
:1003C00010D0034014D0034014E000E01FBF02002F
:1003D00000002020E70976671CE00340A5C3945A7B
:1003E00000F00740FFFFFFFFFFFFFFFFFFFFFFFFE2
:1003F000FFFFFFFFFFFFFFFFFFFFFFFFFFFFFFFF0D
:10040000FFFFFFFFFFFFFFFFFFFFFFFFDEF9FFFF23
:1004100010B5054C237833B9044B13B10448AFF33E
:1004200000800123237010BD8833FF1F00000000EF
:10043000343A0400084B10B51BB108490848AFF323
:1004400000800848036803B910BD074B002BFBD0A0
:10045000BDE81040184700BF000000008C33FF1FAC
:10046000343A04008833FF1F00000000704700BFCB
:10047000704700BF034B586810B101680A68104705
:10048000704700BF7CDF0120034BD86810B10168C2
:100490000A681047704700BF7CDF0120034B1869D2
:1004A00010B101680A681047704700BF7CDF012067
:1004B000034B586910B101680A681047704700BFC4
:1004C0007CDF0120034B986910B101680A6810476E
:1004D000704700BF7CDF0120034BD86910B1016871
:1004E0000A681047704700BF7CDF0120034B186A81
:1004F00010B101680A681047704700BF7CDF012017
:10050000034B586A10B101680A681047704700BF72
:100510007CDF0120034B986A10B101680A6810471C
:10052000704700BF7CDF0120034BD86A10B101681F
:100530000A681047704700BF7CDF0120034B186B2F
:1005400010B101680A681047704700BF7CDF0120C6
:10055000034B586B10B101680A681047704700BF21
:100560007CDF0120034B986B10B101680A681047CB
:10057000704700BF7CDF0120034BD86B10B10168CE
:100580000A681047704700BF7CDF0120034B186CDE
:1005900010B101680A681047704700BF7CDF012076
:1005A000034B586C10B101680A681047704700BFD0
:1005B0007CDF0120034B986C10B101680A6810477A
:1005C000704700BF7CDF0120034BD86C10B101687D
:1005D0000A681047704700BF7CDF0120034B186D8D
:1005E00010B101680A681047704700BF7CDF012026
:1005F000034B586D10B101680A681047704700BF7F
:100600007CDF0120034B986D10B101680A68104728
:10061000704700BF7CDF0120034BD86D10B101682B
:100620000A681047704700BF7CDF0120034B186E3B
:1006300010B101680A681047704700BF7CDF0120D5
:10064000034B586E10B101680A681047704700BF2D
:100650007CDF0120034B986E10B101680A681047D7
:10066000704700BF7CDF0120034BD86E10B10168DA
:100670000A681047704700BF7CDF0120034B186FEA
:1006800010B101680A681047704700BF7CDF012085
:10069000034B586F10B101680A681047704700BFDC
:1006A0007CDF0120034B986F10B101680A68104786
:1006B000704700BF7CDF0120034BD86F10B1016889
:1006C0000A681047704700BF7CDF0120034BD3F856
:1006D000800010B101680A68104770477CDF012074
:1006E000034BD3F8840010B101680A6810477047C3
:1006F0007CDF0120034BD3F8880010B101680A6841
:10070000104770477CDF0120034BD3F88C0010B1F9
:1007100001680A68104770477CDF0120034BD3F85B
:10072000900010B101680A68104770477CDF012013
:10073000034BD3F8940010B101680A681047704762
:100740007CDF0120034BD3F8980010B101680A68E0
:10075000104770477CDF0120034BD3F89C0010B199
:1007600001680A68104770477CDF0120034BD3F80B
:10077000A00010B101680A68104770477CDF0120B3
:10078000034BD3F8A40010B101680A681047704702
:100790007CDF0120034BD3F8A80010B101680A6880
:1007A000104770477CDF0120034BD3F8AC0010B139
:1007B00001680A68104770477CDF0120034BD3F8BB
:1007C000B00010B101680A68104770477CDF012053
:1007D000034BD3F8B40010B101680A6810477047A2
:1007E0007CDF0120034BD3F8B80010B101680A6820
:1007F000104770477CDF0120034BD3F8BC0010B1D9
:1008000001680A68104770477CDF0120034BD3F86A
:10081000C00010B101680A68104770477CDF0120F2
:10082000034BD3F8C40010B101680A681047704741
:100830007CDF0120034BD3F8C80010B101680A68BF
:10084000104770477CDF0120034BD3F8CC0010B178
:1008500001680A68104770477CDF0120034BD3F81A
:10086000D00010B101680A68104770477CDF012092
:10087000034BD3F8D40010B101680A6810477047E1
:100880007CDF0120034BD3F8D80010B101680A685F
:10089000104770477CDF0120034BD3F8DC0010B118
:1008A00001680A68104770477CDF0120034BD3F8CA
:1008B000E00010B101680A68104770477CDF012032
:1008C000034BD3F8E40010B101680A681047704781
:1008D0007CDF0120034BD3F8E80010B101680A68FF
:1008E000104770477CDF0120034BD3F8EC0010B1B8
:1008F00001680A68104770477CDF0120F8B506469A
:10090000044690F8587000252DE0042B00F0C080BC
:10091000022B00F0B1800834A069013540B1227F7C
:10092000032A00F09D80042A00F08F80022A7CD0E8
:10093000206A6A1C38B194F82430032B69D0042B48
:100940005CD0022B4CD0A06AAA1C38B194F82C10B1
:1009500003293AD004292DD0022917D00335082DB8
:1009600004F1180425D0A0690028D4D0237F032BDC
:10097000CBD147FA05F1CB07CDD496F858202A41C0
:10098000D107C8D5036819688847C4E747FA02FC4D
:100990005FEACC71E2D596F8583043FA02F2D307F9
:1009A000DCD40368196888470335082D04F118045E
:1009B000D9D1F8BD96F85810794041FA02F3DB0717
:1009C000CCD5036819688847EEE747FA02F1C907F2
:1009D000C4D496F858C04CFA02F2D207BED5E0E76C
:1009E00047FA02F1C907AED596F858C04CFA02F2A0
:1009F000D307A8D401680B689847A4E796F8583045
:100A00007B4043FA02F1CB079DD501680B689847FC
:100A100099E747FA02FC5FEACC7194D496F8583013
:100A200043FA02F2D2078ED5E4E747FA05FC5FEA03
:100A3000CC727FF57DAF96F858302B41DB073FF540
:100A400077AF01680A68904772E796F858107940C6
:100A50002941C9077FF56CAF01680A68904767E7CD
:100A600047FA05F2D2073FF563AF96F858302B41AD
:100A7000DB077FF55DAFE4E747FA05F1CA077FF5CD
:100A80004AAF96F858202A41D3073FF544AF79E79B
:100A900096F858307B402B41D9077FF53CAF03686F
:100AA0001968884737E700BF30B48369164C027F66
:100AB00093F858302568016982B01341019503F01D
:100AC0000103019A81B14468551AA54209D3A3B91B
:100AD000826895424FF0010334BF0025012545751A
:100AE000037502B030BC7047002BFAD12468009423
:100AF000009D056102B030BC7047002101610175A5
:100B0000417502B030BC7047ACE00120F8B5D0F8B8
:100B10009032816900EBC30201330E2B0646A8BF59
:100B2000002300F52975D2F8C8020C69048006EB91
:100B3000C307C6F8903297F8C47200242B6847FAAE
:100B400004FC28469A680CF0010101349047042CFB
:100B500005F10805F2D10C4D307D4D2101FB005E01
:100B60009EF8437007F01F041F2C0BD0B66917F0D6
:100B7000800F16BFF168102121F0100144F04003EE
:100B8000F1603360F8BD00BF90330400F8B5002475
:100B900090F8C472C0F89042064600F529752B689B
:100BA00047FA04F128469A6801F0010101349047A0
:100BB000042C05F10805F2D1377D154BB06906EB21
:100BC000870C4D26DCF80C20046806FB073E55090F
:100BD000A9009EF8437001F1604302F01F0603F57F
:100BE000614C012207F01F0144F0400402FA06F5AF
:100BF0001F290460CCF8005009D03F064ABFC768DF
:100C0000102727F0100741F04003C7600360F8BDCC
:100C100090330400D0F8A012214AF8B54B1C03F021
:100C20000303047D1F4E00EB83054D27D5F88C523E
:100C300007FB042C84691CF80570202232602669A9
:100C4000C0F8A03207F01F031F2BB2B209D03D0637
:100C50004ABFE568102525F0100543F04007E56020
:100C60002760D0F89C02104C06683368A34212D16A
:100C7000C768FC070AD5456880687E10AC592358C0
:100C8000A8199847094920220A60F8BD4668836878
:100C900006EB6700F5E79847044920220A60F8BD93
:100CA0009033040084F00F40150E000088F00F40D0
:100CB000037D194970B4D0F8A052846900EB830217
:100CC00000EB8500D268D0F88C5220684D2606FBD8
:100CD000031C51098B001CF8055003F1604606F512
:100CE000614C02F01F02012105F01F0640F0400098
:100CF00001FA02F31F2E2060CCF8003009D02D0637
:100D00004ABFE568102525F0100546F04002E56071
:100D1000226070BC704700BF9033040010B4384BA1
:100D2000196883B029B10B6FC2785C782CB9162A88
:100D300042D003B05DF8044B7047197829B9162AE0
:100D40003DD003B05DF8044B704702F1FF3C0179E0
:100D5000BCF1160FEDD801A050F82CF0E70D000003
:100D6000CD0D0000330D0000330D0000330D0000E9
:100D7000330D0000330D0000330D0000330D000073
:100D8000330D0000330D0000330D0000330D000063
:100D9000330D0000330D0000330D0000330D000053
:100DA000330D0000330D0000330D0000330D000043
:100DB000BF0D0000C70D00001C78002CC5D101211B
:100DC00059701970B5E700201870B2E70D4A0E4847
:100DD0001468009445F6104C009A5A6000249C70E8
:100DE00040F80C10A5E7074A07481468019445F637
:100DF000144C019A5A6000249C7040F80C1098E73B
:100E00004074FF1FACE001204874FF1F704700BF13
:100E1000704700BF30B4C368DC0708D545688068F8
:100E20005B10EC582458E818A44630BC604784682E
:100E30004568A44605EB630030BC6047C368DA0729
:100E400006D55B1041688268C8588258C818104798
:100E50004168826801EB6300104700BF4368074A9E
:100E6000D8B211F0FF0F52F830304FF0010014BF2C
:100E700083F8800083F80001704700BF103504003C
:100E8000C9B200790FF094BF10B5102104460FF0DD
:100E900077FA204610BD00BF2DE9F04107EE902AF9
:100EA0009FED7E7AF8EEE76A2DED028B4FF48F63AB
:100EB000BEEE000A054644F2C81203FB0100A6EE8E
:100EC000870A8458D4ED050A30EE001AB7EE008A7E
:100ED00061EE201A82B0F4EEC81AF1EE10FA00F1B9
:100EE000C28094F8426094ED022A56B3DFED6C2A7A
:100EF0009FED6C5A94ED046ADFED6B5AB1EE043A43
:100F000062EE033A22EE224AF4EEC53A68EE064A51
:100F1000F1EE10FAB4EE654A58BFF0EE453AF1EE44
:100F200010FAF5EEC04A48BFB0EE654AF1EE10FA8D
:100F3000CBBF73EEC23A32EE444AA4EEA32AA4EE2B
:100F4000842A94F8417084ED032AF7EE007A5FB1A9
:100F500078EE278AD4ED046AB6EE007A28EE870A86
:100F600077EEE67AE6EE807A94F84360C4ED067A8E
:100F7000E6B1DFF84881D4ED048AD8F80030DB0709
:100F80007BD54A4FF0EE000ABFEE001AA8EEA01A79
:100F9000B4EEC18AF1EE10FA55D5D7ED001AB4EED1
:100FA000E11AF1EE10FA4ED887ED008A4FF48F6007
:100FB00000FB015C44F2C81284F840605CF8024017
:100FC00094F84430D3B3D4ED042A9FED395A394F05
:100FD000DFED395A22EE856A01EB4101BDEEC63ADA
:100FE000880013EE106A43F6FC0207EB860E2F18FA
:100FF000DEED003ABC5828EE258A04EE104AE2EEF7
:10100000883A05F563553C350544F8EEC44A07F5C2
:101010006458287A23EEA40A0FF0C4FDD8F8001013
:10102000287A012303FA01FC0CEBDC71194102B0B0
:10103000BDEC028BBDE8F0410FF0AABB02B0BDECE5
:10104000028BBDE8F081B4EEC18AF1EE10FA06DD44
:1010500097ED002AB4EEC21AF1EE10FAA4DA87ED89
:10106000008A0026A2E7BFEE008AF4EEC81AF1EE6D
:1010700010FAC8BFB0EE618A33E7404601910FF025
:101080003DF9019900283FF47CAF084F019140469B
:1010900087ED008A0FF038F9019973E7010880396C
:1010A000CDCC4C3E00005C4500005C41F833FF1F96
:1010B0000080F943A0D6FF1F0080BB45F433FF1F1B
:1010C00008B500790FF066FE08BD00BF90F86430E7
:1010D00063B310B48268284C92F802C027490CF020
:1010E000FE039370026E13792370046E22790A70E6
:1010F000816891F803C05FEA0C63FAD5046E204B57
:1011000022791A7081680224CC70826892F802C039
:101110000CF0C7039370836842F21071DC78A40668
:1011200005D400225DF8044B80F864207047DA781B
:101130009206F6D5DC78A406F3D593F803C05FEAEF
:101140008C62EED5DA789406EBD5DC78A206E8D589
:1011500093F803C05FEA8C64E3D5DA789206E0D5B1
:101160000839DBD1997000BF83688021997000BF76
:1011700001240473D5E700BF1F8000401A8000409F
:101180001C80004038B5437B85689C1E012CEA78A2
:10119000A97902D90223EB7038BD5FFA82FC5FEABD
:1011A000CC642AD45FEA4C632DD4CBB213F0500F39
:1011B000044612D0A87940F05002AA71A568A97916
:1011C00001F0DF03AB71A0680222C27025690DB186
:1011D000606DA8470221A5686173636D3F2B04D839
:1011E000581C606523442A791A75A97941F0500387
:1011F000AB71A4680225E57038BD1022EA705FEA81
:101200004C621CD5856800214165816595F806C052
:101210004CF02003AB718468C025A57081680A7901
:10122000530880F85C308C7944F050058D718168EA
:101230004222CA7084680323A279437338BD85684B
:10124000A97941F05002AA7180680224C47038BDA7
:101250000FB400B5C3B044ABFF2153F8042B019386
:1012600002A813F027FC02A813F04AFB014602A8CB
:1012700010F0CAFD43B05DF804EB04B0704700BF46
:101280000C4B986898B101680B4A0B6893420FD1D8
:10129000C368DA0706D55B1041688268C85882586F
:1012A000C81810474168826801EB63001047704717
:1012B000184700BF7CDF01203D0E0000D0ED047A0E
:1012C00090ED067A90ED056AD0ED036AD0ED025AF2
:1012D00030EE670AB0EE675AA7EE005AF6EE004A03
:1012E00075EE671A36EEE51A31EEC62AA2EE246ACA
:1012F00076EE052A80ED056AF4EEC12AF1EE10FAC9
:10130000C0ED042A24D572EEA56AC0ED036AD0EDC3
:10131000003A90ED074A90ED010AF0EE007AB0EE47
:10132000637AA5EEA77AF0EE635A76EEC76AE6EE28
:10133000845AF4EEC05AF1EE10FA08D5F4EEE53A0C
:10134000F1EE10FA54BFB0EE630AB0EE650A7047D2
:1013500036EEA53AF4EEC32AF1EE10FAC4BF72EEEF
:10136000E56AC0ED036AD2E72DE9F04F002A9DF847
:10137000244069DB002B67DB7F2865DC7F2963DC89
:101380007F2AA8BF7F2220EAE07E7F2BA8BF7F2391
:10139000724521EAE1789C4656DB5F1CC8EB0700EA
:1013A000DFF8A8A002F10109C7014FEAC81BC44534
:1013B00044DB0EEB0B028023A7F18001BB420AF84D
:1013C0000240C1F3C215524438D0EDB1012D17D0FF
:1013D000022D13D0032D0FD0042D0BD0052D07D0D7
:1013E000062D1CBF4FF4807382F88040D4548033A4
:1013F000D4548033D4548033D4548033D454803381
:10140000D4548033BB4219D003F1800103F58076B8
:1014100003F5C075D45403F500705454945503F586
:101420002071545503F5407603F5607503F580632C
:10143000BB421454545494555455E5D10EF1010E49
:10144000CE45B4D1BDE8F08FBDE8F08F4034FF1F2A
:10145000826810B442F210730446D17888060AD527
:10146000D078810607D592F803C05FEA8C6002D578
:10147000D17889062BD4B0239370A26842F21073FE
:1014800092F803C05FEA8C601BD4D178890618D427
:10149000D078800615D492F803C05FEA8C6110D42E
:1014A000D17888060DD4D07881060AD492F803C08A
:1014B0005FEA8C6005D4D178890602D4083BDFD17D
:1014C00015E0D478C4F340105DF8044B7047D07831
:1014D0008006D0D592F803C05FEA8C61CBD5D17875
:1014E0008806C8D5D0788106C5D5083BB5D193709C
:1014F00000BFA2688020907000BF012118462173B0
:101500005DF8044B704700BF01380B463A2800F2E3
:101510005C82DFE810F053024C0245023E023702C3
:101520003002290222021B02AE01A701A00199018B
:1015300092018B0184017D0176016F0168016101D7
:101540005A0153014C0145013E0137013001290187
:1015500022011B0113010B010301FB00F300EB004F
:10156000E300DB00D300CB00C300BB00B300AB0043
:10157000A3009B0093008B0083007B0073006B0033
:1015800063005B0053004B0043003B00BC48BD4977
:10159000C0F8EC201A463B200EF01CBFB848BA49F0
:1015A000C0F8E8201A463A200EF014BFB448B749F4
:1015B000C0F8E4201A4639200EF00CBFB048B449F8
:1015C000C0F8E0201A4638200EF004BFAC48B149FC
:1015D000C0F8DC201A4637200EF0FCBEA848AE4901
:1015E000C0F8D8201A4636200EF0F4BEA448AB4905
:1015F000C0F8D4201A4635200EF0ECBEA048A84909
:10160000C0F8D0201A4634200EF0E4BE9C48A5490C
:10161000C0F8CC201A4633200EF0DCBE9848A24910
:10162000C0F8C8201A4632200EF0D4BE94489F4914
:10163000C0F8C4201A4631200EF0CCBE90489C4918
:10164000C0F8C0201A4630200EF0C4BE8C4899491C
:10165000C0F8BC201A462F200EF0BCBE8848964920
:10166000C0F8B8201A462E200EF0B4BE8448934924
:10167000C0F8B4201A462D200EF0ACBE8048904928
:10168000C0F8B0201A462C200EF0A4BE7C488D492C
:10169000C0F8AC201A462B200EF09CBE78488A4930
:1016A000C0F8A8201A462A200EF094BE7448874934
:1016B000C0F8A4201A4629200EF08CBE7048844938
:1016C000C0F8A0201A4628200EF084BE6C4881493C
:1016D000C0F89C201A4627200EF07CBE68487E4940
:1016E000C0F898201A4626200EF074BE64487B4944
:1016F000C0F894201A4625200EF06CBE6048784948
:10170000C0F890201A4624200EF064BE5C4875494B
:10171000C0F88C201A4623200EF05CBE584872494F
:10172000C0F888201A4622200EF054BE54486F4953
:10173000C0F884201A4621200EF04CBE50486C4957
:10174000C0F880201A4620200EF044BE4C4869495B
:10175000C2671A461F200EF03DBE4948664982679F
:101760001A461E200EF036BE4548644942671A46A6
:101770001D200EF02FBE4248614902671A461C2008
:101780000EF028BE3E485F49C2661A461B200EF086
:1017900021BE3B485C4982661A461A200EF01ABEEA
:1017A00037485A4942661A4619200EF013BE34488B
:1017B000574902661A4618200EF00CBE30485549AB
:1017C000C2651A4617200EF005BE2D4852498265A3
:1017D0001A4616200EF0FEBD2948504942651A46A9
:1017E00015200EF0F7BD26484D4902651A46142013
:1017F0000EF0F0BD22484B49C2641A4613200EF089
:10180000E9BD1F48484982641A4612200EF0E2BD25
:101810001B48464942641A4611200EF0DBBD1848A9
:10182000434902641A4610200EF0D4BD14484149C1
:10183000C2631A460F200EF0CDBD11483E498263A7
:101840001A460E200EF0C6BD0D483C4942631A46AA
:101850000D200EF0BFBD0A48394902631A460C201C
:101860000EF0B8BD06483749C2621A460B200EF08A
:10187000B1BD0348344982621A460A200EF0AABD5F
:101880007CDF0120E9080000D5080000C108000045
:10189000AD080000990800008508000071080000EC
:1018A0005D0800004908000035080000210800001C
:1018B0000D080000F9070000E5070000D10700004F
:1018C000BD070000A9070000950700008107000080
:1018D0006D070000590700004507000031070000B0
:1018E0001D07000009070000F5060000E1060000E2
:1018F000CD060000B9060000A50600009106000014
:101900007D06000069060000550600004106000043
:101910002D0600001906000005060000F105000074
:10192000DD050000C9050000B5050000A1050000A7
:101930008D050000790500006505000051050000D7
:101940003D05000029050000150500001F4820493D
:1019500042621A4609200EF03DBD1C481D49026234
:101960001A4608200EF036BD18481B49C2611A46B7
:1019700007200EF02FBD1548184982611A4606202F
:101980000EF028BD1148164942611A4605200EF096
:1019900021BD0E48134902611A4604200EF01ABDFB
:1019A0000A481149C2601A4603200EF013BD0748C9
:1019B0000E4982601A4602200EF00CBD03480C4905
:1019C00042601A4601200EF005BD70477CDF012001
:1019D00001050000ED040000D9040000C50400006A
:1019E000B10400009D040000890400008112000081
:1019F0007504000008B5134640680A461946FFF70B
:101A000083FD08BD2DE9F04F7A4C0F78236895B01F
:101A100005460A930A9E22680B920B9B40696B61F4
:101A2000013F032F00F2FA84DFE817F0F102E6022B
:101A3000C30204009FED727A0023361A01EE106A89
:101A4000DFED6D6AF8EE411AA1EEE67A85ED047AD3
:101A5000A8682F7B002B40F0DB83012390F859907E
:101A600003FA07F729EA0706236880F85960069306
:101A7000069E91F809A020680790079F686E6F6620
:101A80000AF1FF3BBBF1030F00F2C084DFE81BF05B
:101A900086027B02580204009FED592A0023361A61
:101AA00004EE106A9FED545AF8EE444AA4EEC52A9B
:101AB00085ED182AA86D95F85C70002B40F0A28384
:101AC000012390F859E003FA07F72EEA0706236886
:101AD00080F859600293029E91F80A802068039072
:101AE000039F686F6F6708F1FF39B9F1030F00F2C8
:101AF0008F84DFE819F01A020F02EC010400DFED19
:101B0000405A0023361A00EE106A9FED3B1AF8EE99
:101B1000400AE0EEC15AC5ED1C5AA86E95F86C70EB
:101B2000002B40F06983012390F859B003FA07F7BE
:101B30002BEA0702DFED306ADFF8C0C080F85920D9
:101B40000E1D2B460020F2EE0E4A01274FF08C0EA0
:101B500022681292DDF8488011F801BFD4F8009095
:101B6000CDF84C90DDF84CA0D3F82490C3F824A015
:101B70000BF1FF32032A00F24D84DFE812F09C01E2
:101B8000910171010400DFED1E1A0022C9EB080B60
:101B900003EE10BAF8EE433AE3EEE61AC3ED081A84
:101BA000D3F8189093F81C80002A40F01A8399F813
:101BB00059A007FA08F22AEA0208226889F859802F
:101BC0000E92DDF8389016F801BFD4F80080CDF8F9
:101BD0003C80DDF83CA0D3F88480C3F884A00BF1EE
:101BE000FF32032A00F21884DFE812F02E012301ED
:101BF00003010C00ACE001206F12833A3BA8833A4A
:101C0000CDCCCC3E1FED024A0022C8EB090B06EEFC
:101C100010BAB8EE467AA7EE664A83ED204AD3F8AA
:101C2000789093F87C80002A40F0D38299F859A0EC
:101C300007FA08F22AEA02020130042889F859203A
:101C400003F1100384D12E68376896F85A4038465D
:101C5000FFF7FEFB002862D0B968887840F03003B7
:101C60008B70BA6842F21071D07880060FD492F867
:101C700003C05FEA8C630AD492F803E05FEA8E60E7
:101C800005D492F803905FEA896340F1C78264004B
:101C9000E1B21171BB6842F21072D878840708D49F
:101CA000DC78A00705D493F803C05FEA8C7040F19C
:101CB00017833268936842F21070DF78390600F1BA
:101CC000B081D9780F0600F1AC81DC78210600F1F3
:101CD000A881DF783F0600F1A48193F803C05FEA92
:101CE0000C6400F19E8193F803E05FEA0E6100F15D
:101CF000988193F803905FEA096700F1928193F865
:101D000003A05FEA0A6400F18C810838D5D198708D
:101D100000BF96688023B37000BF012111736D6806
:101D20002E6895F85A403046FFF792FB00285DD0A8
:101D3000B76897F8028048F03003BB70B26842F28F
:101D40001071D07887060DD4D778B8060AD492F8E7
:101D500003C05FEA8C6005D492F803E05FEA8E630B
:101D600040F177826400E3B21371B36842F21072FB
:101D7000D978890706D4D878870703D4DF78BF07D6
:101D800040F184822A68936842F21070DE7834064B
:101D900000F1B08193F803B05FEA0B6100F1AA8112
:101DA00093F803805FEA086400F1A481D9780906FA
:101DB00000F1A081DF783F0600F19C81DC782606E7
:101DC00000F19881DE78340600F1948193F803C025
:101DD0005FEA0C6100F18E810838D7D1987000BF9E
:101DE00094688025A57000BF0120107315B0BDE870
:101DF000F08F22680C92DDF830A04FEA9A0BACFB12
:101E00000BB2D2080EFB12A2462A8CBF002201227E
:101E100093ED204AB5EEC04AF1EE10FA7FF7FFAE1F
:101E200024EE245AFDEEC55A15EE90AA0AF00102DE
:101E3000EBE622680D920D9AC2F30802B2F5807F9C
:101E40008CBF00220122E3E793ED204AB5EEC04AA1
:101E5000F1EE10FAE4DCD3F8789093F87C80E5E6B4
:101E600022681092DDF840A04FEA9A0BACFB0BB24F
:101E7000D2080EFB12A2462A8CBF00220122D3ED0B
:101E8000081AF5EEC01AF1EE10FA7FF789AE21EECE
:101E9000A42AFDEEC22A12EE90AA0AF0010275E60B
:101EA00022681192119AC2F30802B2F5807F8CBFAA
:101EB00000220122E3E7D3ED081AF5EEC01AF1EE95
:101EC00010FAE4DCD3F8189093F81C806FE62268CF
:101ED0000092009FC74BBA08A3FB0232D2084FF012
:101EE0008C0A0AFB1273462B8CBF00230123D5ED0D
:101EF0001C5AF5EEC05AF1EE10FA7FF70EAEB2EEB4
:101F00000E6A25EE867AFDEEC77A17EE902A02F069
:101F10000103F7E527680197019BC3F30803B3F5B5
:101F2000807F8CBF00230123E1E7D5ED1C5AF5EE3D
:101F3000C05AF1EE10FAE2DCA86E95F86C70F2E58A
:101F400022680492049FAB4BBA08A3FB0232D2086A
:101F50004FF08C0C0CFB1273462B8CBF002301231B
:101F600095ED182AB5EEC02AF1EE10FA7FF7A2AD72
:101F7000F2EE0E2A22EE223AFDEEC33A13EE902A3A
:101F800002F001038BE527680597059BC3F308035F
:101F9000B3F5807F8CBF00230123E1E795ED182A7C
:101FA000B5EEC02AF1EE10FAE2DCA86D95F85C708F
:101FB00086E522680892089F8E4BBA08A3FB02327E
:101FC000D2084FF08C0808FB1273462B8CBF0023FD
:101FD000012395ED047AB5EEC07AF1EE10FA7FF7A1
:101FE00037ADF2EE0E7A27EE270AFDEEC00A10EEAC
:101FF000902A02F0010320E527680997099BC3F3A3
:102000000803B3F5807F8CBF00230123E1E795ED42
:10201000047AB5EEC07AF1EE10FAE2DCA8682F7B04
:102020001BE5022196F85900D970946894F802B023
:102030004BF01003A37097683871916842F21070EA
:10204000CC78A4070AD491F803805FEA887305D49A
:1020500091F803C05FEA8C7340F16C81CF78022065
:10206000FCB2C87014F0100140F0B981E70700F12C
:10207000C7819268D07031688E6896F8028008F047
:10208000C703B3708B6842F21070DF78BC067FF52F
:1020900046AEDC78A2067FF542AE93F803C05FEA55
:1020A0008C647FF53CAE93F803E05FEA8E627FF5C7
:1020B00036AE93F803905FEA89677FF530AE93F808
:1020C00003A05FEA8A667FF52AAE93F803B05FEA61
:1020D0008B647FF524AEDA7892067FF520AE08385F
:1020E000D3D1987000BF8E688023B37000BF0120E9
:1020F000087314E6022195F85900D970976897F88B
:1021000002E04EF01003BB7094682071916842F2B7
:102110001070CE78B3070DD4CF78BF070AD491F8EA
:1021200003905FEA897705D491F803A05FEA8A7685
:1021300040F12181CB780220DCB2C87014F010018C
:1021400040F03681E60700F144819268D07029683A
:102150008D68AE7806F0C707AF708B6842F21070DA
:10216000DC78A5067FF542AE93F803905FEA8964B8
:102170007FF53CAE93F803A05FEA8A627FF536AE46
:1021800093F803B05FEA8B677FF530AE93F8038076
:102190005FEA88667FF52AAE93F803C05FEA8C6534
:1021A0007FF524AE93F803E05FEA8E647FF51EAE00
:1021B000DA7892067FF51AAE0838D1D1987000BF50
:1021C0008D688026AE7000BF01270F7315B0BDE883
:1021D000F08F99F859B002FA08F84BEA0802D2B227
:1021E0002AE599F859B002FA08FA4BEA0A025FFAAE
:1021F00082F8E2E43BA8833A90F85960BB4033434D
:10220000DAB297E490F85920BB401343DEB25EE4A3
:1022100090F85920BB401343DEB225E492F803A0A6
:102220005FEA8A603FF533AD92F803B05FEA8B63F3
:102230003FF52DAD92F803805FEA88603FF527AD4A
:10224000D3789B063FF523AD08397FF40DAD91702F
:1022500068E092F803905FEA89673FF583AD92F8F2
:1022600003A05FEA8A603FF57DAD92F803B05FEAB4
:102270008B633FF577AD92F803805FEA88673FF59F
:1022800071AD08397FF45DAD91701FE0DC78A40773
:102290003FF578AD93F803C05FEA8C703FF572ADFF
:1022A00093F803E05FEA8E713FF56CAD93F803900D
:1022B0005FEA89773FF566AD93F803A05FEA8A7419
:1022C0003FF560AD083A7FF453AD9A7000BFB16836
:1022D00080278F7000BF0123337315B0BDE8F08FE6
:1022E00093F803E05FEA8E713FF5E3AC93F8039057
:1022F0005FEA89743FF5DDAC93F803A05FEA8A706A
:102300003FF5D7AC93F803B05FEA8B713FF5D1ACE2
:1023100093F803805FEA88743FF5CBAC083A7FF40A
:10232000BCAC9A7000BFB8688024847000BF0122E2
:102330003A73F4E491F803E05FEA8E773FF58EAEEE
:1023400091F803905FEA89743FF588AE91F803A095
:102350005FEA8A733FF582AE91F803B05FEA8B774C
:102360003FF57CAECB789C073FF578AE08387FF41C
:1023700067AE8870CCE491F803B05FEA8B743FF5E8
:10238000D9AE91F803805FEA88733FF5D3AE91F838
:1023900003C05FEA8C773FF5CDAE91F803E05FEACA
:1023A0008E763FF5C7AE08387FF4B3AE887016E579
:1023B00090681021C17000BF956803200021107340
:1023C000A97000BF96688027B77093680222DA7000
:1023D0000CE593680124DC7000BF9568EFE7936813
:1023E0001021D97000BF9668032000211073B170CE
:1023F00000BF90688027877094680222E2708EE4A4
:1024000097680124FC7000BF9668EFE70123A7E5F9
:1024100001236CE5012232E50122F9E40123D8E52C
:102420002DE9F0430668376896F85A4085B00546AE
:102430003846FFF70DF830B3BA68937843F03000B0
:102440009070BA6842F2107192F803805FEA886077
:102450000AD492F803905FEA896305D492F803C026
:102460005FEA8C6040F15881640044F00101CBB216
:102470001371BB6842F21072D878840703D4DC78F9
:10248000A00740F17E81002732688DF807709DF823
:102490000730936842F2107093F803C05FEA0C6152
:1024A00000F1E18093F803E05FEA0E6700F1DB8062
:1024B00093F803805FEA086100F1D58093F80390F8
:1024C0005FEA096700F1CF80D9780C0600F1CB8074
:1024D000DC78210600F1C780DF783F0600F1C38079
:1024E00093F803C05FEA0C6400F1BD800838D3D1D3
:1024F000987000BF94688023A37000BF01211173FE
:102500006E68376896F85A403846FEF7A1FF70B3F8
:10251000B868827842F030038370BA6842F2107172
:10252000D07880060FD492F803E05FEA8E630AD475
:1025300092F803805FEA886005D492F803905FEA1E
:10254000896340F1CA81640044F00101CBB2137188
:10255000BB6842F21072D878800708D4DC78A107F3
:1025600005D493F803805FEA887040F1CF8100279B
:1025700032688DF806709DF80630936842F210704C
:1025800093F803805FEA086700F1278193F80390CE
:102590005FEA096400F1218193F803C05FEA0C61EE
:1025A00000F11B8193F803E05FEA0E6700F11581EB
:1025B000D9780C0600F11181DC78210600F10D813B
:1025C000DF783F0600F1098193F803805FEA086431
:1025D00000F103810838D3D1987000BF946880233C
:1025E000A37000BF01211173D5F84841002C37D0EA
:1025F000B34FDFF8D08268354FF0000901260FE0B5
:102600006268411A914209D3002B40F05D81A368B2
:1026100026758B428CBF002101216175E468FCB1F5
:10262000A54200F0588120680268BA4240F0448117
:10263000A369227F93F85830D8F8000021690390ED
:10264000134103F0010303980029D9D1002BE5D1F0
:10265000D8F800000290029A2261E468002CDFD1D1
:1026600005B0BDE8F083987800F0E70199709368B1
:102670001C79E7B28DF80770987840F008019970DE
:1026800093680224DC70936842F21070DF78BC0714
:1026900009D493F803E05FEA8E7104D493F80380C1
:1026A0005FEA887157D5987800F0C70199709368F0
:1026B00042F21071DC78A70627D5DF78BC0624D556
:1026C00093F803E05FEA8E671FD593F803805FEA13
:1026D00088641AD593F803905FEA896015D593F85A
:1026E00003C05FEA8C6710D5D87884060DD5DC78F6
:1026F000A0060AD50839DDD1997000BF9368802102
:10270000997000BF012793681773187986F85800ED
:1027100096680222F270F3E692F803E05FEA8E63B5
:102720003FF5A2AED37898063FF59EAED0788306EB
:102730003FF59AAE92F803805FEA88603FF594AE69
:1027400092F803905FEA89633FF58EAE08397FF413
:102750007BAE917039E093F803905FEA8977A2D459
:1027600093F803C05FEA8C749DD4D97889079AD412
:10277000DC78A70797D4DF78BC0794D4083885D1D4
:10278000B6E693F803C05FEA8C703FF57CAE93F831
:1027900003E05FEA8E713FF576AE93F803805FEA5F
:1027A00088743FF570AE93F803905FEA89703FF547
:1027B0006AAED97889073FF566AED87884073FF5C9
:1027C00062AE083A7FF458AE9A7000BFBB688022B0
:1027D0009A7000BF01243C7355E6987800F0E70139
:1027E000997093681C79E7B28DF80670987840F07C
:1027F0000801997093680224DC70936842F21070AB
:10280000DF78B9071FD493F803905FEA89771AD469
:1028100093F803C05FEA8C7115D493F803E05FEA84
:102820008E7710D493F803805FEA88740BD4D9783C
:10283000890708D4DC78A70705D4DF78BC0702D461
:102840000838DDD1C8E6987800F0C7019970936820
:1028500042F21071DC78A40627D5DF78B80624D5BB
:1028600093F803905FEA89671FD593F803C05FEA86
:102870008C641AD593F803E05FEA8E6015D593F85F
:1028800003805FEA886710D5D87884060DD5DC7898
:10289000A0060AD50839DDD1997000BF9368802160
:1028A000997000BF012793681773187986F858004C
:1028B00096680222F27097E620469047AEE600BF87
:1028C000A90A0000ACE00120C4F8109084F814902C
:1028D00084F81590A2E600BFA5E692F803C05FEA6F
:1028E0008C603FF530AED3789B063FF52CAED078A8
:1028F00080063FF528AE92F803E05FEA8E633FF56D
:1029000022AE08397FF40CAE91701DE093F803906D
:102910005FEA89713FF52BAE93F803C05FEA8C74D0
:102920003FF525AE93F803E05FEA8E703FF51FAEEA
:10293000D97889073FF51BAED87884073FF517AEE5
:10294000083A7FF408AE9A7000BFBB6880229A7084
:1029500000BF01243C730AE6F8B5046894F86430BB
:1029600005460E46002B00F0EA80A36842F2107183
:10297000D878020623D4DF783F0620D493F803C02A
:102980005FEA0C601BD4DA78120618D4D8780706F0
:1029900015D4DF78380612D493F803C05FEA0C62CE
:1029A0000DD4DA7817060AD40839E1D1997000BF3E
:1029B000A16880228A7000BF0123237327E00221CF
:1029C000D970A068837843F010078770A16800224F
:1029D0000A71A26842F21071D078800707D492F889
:1029E00003C05FEA8C7302D4D378980746D5D078B9
:1029F00002215FFA80FCD1701CF0100240F02481AB
:102A00005FEACC7700F11481A4680220E0702868A6
:102A1000836842F21071DF783C0644D4DC782206E9
:102A200041D493F803C05FEA0C623CD4DA7817060D
:102A300039D4DF783C0636D4DC78220633D493F8D8
:102A400003C05FEA0C672ED4DA7814062BD4083959
:102A5000E1D1997000BF83688021997000BF012483
:102A6000047329688D68AE7806F0C702AA708B6877
:102A700042F21070DF78BC063FD4F8BDD778BB07B0
:102A8000B5D4D0788707B2D492F803C05FEA8C70CF
:102A9000ADD4D3789B07AAD4D778BF07A7D4083979
:102AA0009AD1917083E70221D9708768BB7843F08F
:102AB0001004BC7082681671826842F21071D67878
:102AC000B3070BD4D778BF0708D492F803C05FEAE6
:102AD0008C7603D4D3789C0740F19380D37802217D
:102AE000DCB2D17014F0100240F0B680E60700F1BD
:102AF000C18080680227C770B3E7DC78A206BCD526
:102B0000DD78AF06B9D5DE78B606B6D593F803C042
:102B10005FEA8C65B1D5DA789406AED5DF78BA066F
:102B2000ABD5DC78A706A8D50838A3D1987000BF2C
:102B30008B688020987000BF01250D73F8BD20467A
:102B40002F7BFEF785FC002859D0A268907840F0D2
:102B500030019170A26842F2107192F803C05FEAEE
:102B60008C601ED492F803E05FEA8E6319D4D378A8
:102B7000980616D4D078830613D492F803C05FEA7F
:102B80008C600ED492F803E05FEA8E6309D4D378A8
:102B9000980606D4D078830603D40839DDD1917025
:102BA00026E07F00F9B21171A36842F21072D87862
:102BB000800724D4DF78B90721D493F803C05FEAF3
:102BC0008C701CD493F803E05FEA8E7117D4D97827
:102BD0008F0714D4D878800711D4DF78B9070ED4C2
:102BE00093F803C05FEA8C7709D4083ADFD19A7072
:102BF00000BFA36880229A7000BF012121732C6856
:102C0000B3E6D478A3073FF569AFD678B7073FF5A9
:102C100065AFD778BE073FF561AF92F803C05FEAB2
:102C20008C743FF55BAF08397FF449AF917011E7C1
:102C3000A3680127DF7000BFA0682173827000BF06
:102C4000A36880279F70DFE6A1681022CA7000BFCA
:102C50000321A0680022F0E781681024CC7000BF37
:102C600083680321002201739A7000BF8668802266
:102C7000B2703EE786680127F77000BF8368F2E70D
:102C80002DE9F84F056895F864300446002B00F0F4
:102C90005A82AB6842F21071DF783E0629D4D878A8
:102CA000000626D4DE78370623D493F803E05FEAE3
:102CB0000E661ED493F803805FEA086019D493F877
:102CC00003905FEA096214D493F803A05FEA0A67ED
:102CD0000FD493F803B05FEA0B660AD40839DBD14E
:102CE000997000BFAF688020B87000BF01212973C0
:102CF00029E00222DA70A96891F802C04CF01003B2
:102D00008B70AF6800203871AB6842F21071DE78CA
:102D1000B2070AD493F803E05FEA8E7705D493F8FC
:102D200003805FEA887040F1E981D8780221C6B259
:102D3000D97016F0100340F09283F60700F1698312
:102D4000AD680222EA709F49022201F11B054FF093
:102D5000100E4FF0030C4FF0000880264FF0010BCF
:102D600029E0F87810F0800F2DD1F87810F0800F5E
:102D700029D1F87810F0800F25D1F87810F0800F65
:102D800021D1F87810F0800F1DD1F87810F0800F65
:102D900019D1F87810F0800F15D1B9F108090ED1CA
:102DA00087F8029000BF9868867000BF0131A94281
:102DB00083F80CB048D023689F6842F21079F87805
:102DC00010F0800FCDD091F80090FA709F6897F8BE
:102DD00002A04AF01000B8709F6887F804909F68BE
:102DE00042F2107A97F803905FEA89701BD4F87862
:102DF000800718D497F803905FEA897013D4F878A5
:102E0000800710D497F803905FEA89700BD4F878A4
:102E1000800708D497F803905FEA897003D4F878A4
:102E2000800740F1898197F803A0FA705FFA8AF76A
:102E300017F0100940F06082FF0700F151829B6893
:102E40000131A942DA70B6D121688A68957805F017
:102E5000C70696708B6842F21070DF78BE0600F1EC
:102E6000FB8000214FF40052A06811F0C9FA2568D8
:102E700095F86410002900F0C881AB6842F2107127
:102E8000DF78380638D4D878020635D493F8038032
:102E90005FEA086030D493F803B05FEA0B622BD48A
:102EA00093F803C05FEA0C6726D493F803E05FEA67
:102EB0000E6621D493F803A05FEA0A601CD493F84D
:102EC00003905FEA096217D40839D9D1997000BF1D
:102ED000AE688027B77000BF236893F864000121B3
:102EE0002973002838D064200DF0C2FF2046AF219E
:102EF000FFF732FDBDE8F88F0222DA70AE68B378D2
:102F000043F01001B170AF6840203871AB6842F2F5
:102F1000107193F803805FEA88770AD493F803B0BE
:102F20005FEA8B7605D493F803C05FEA8C7740F1B3
:102F3000C780DF780221F8B2D97010F0100340F09A
:102F40008082C00700F17182AD680222EA702368B6
:102F500093F864000028C6D1A56820699A68DD66E8
:102F6000186742F21076D77839062DD492F803808C
:102F70005FEA086728D492F803B05FEA0B6723D4AE
:102F800092F803C05FEA0C611ED492F803E05FEA96
:102F90000E6719D492F803A05FEA0A6114D492F87C
:102FA00003905FEA09670FD4D17809060CD4083E74
:102FB000D9D1967000BF9E688021B17000BF0127F3
:102FC0001F7390E770810100967946F05007977162
:102FD0009A681221D1709E68B778012847F01002D4
:102FE000B27000F09D811A6E11680026CE71D2F881
:102FF00000806F1C0F6001278F80C8F80870176869
:1030000001381FFA80FBA7F81EB012684142F96030
:10301000A2F816B01F6E9A68386804328671B2F151
:10302000804F026186823A6880F07381012191604D
:103030003A681F6EB94800269661397901709F6819
:1030400097F802C04CF00102BA7098682D780571AB
:10305000012683F8646046E793F803805FEA886599
:103060007FF5FFAE93F803B05FEA8B667FF5F9AEAC
:1030700093F803C05FEA8C657FF5F3AE93F803E045
:103080005FEA8E627FF5EDAE93F803A05FEA8A6790
:103090007FF5E7AE93F803905FEA89667FF5E1AECE
:1030A000DA7895067FF5DDAE08387FF4D6AE9870F5
:1030B00000BF8D688026AE7000BF01230B73D0E681
:1030C00093F803E05FEA8E763FF533AF93F803A001
:1030D0005FEA8A703FF52DAF93F803905FEA89723B
:1030E0003FF527AFDA7897073FF523AFDE78B607CD
:1030F0003FF51FAF08397FF40CAFE7E693F8039074
:103100005FEA89723FF511AE93F803A05FEA8A7710
:103110003FF50BAE93F803B05FEA8B763FF505AE53
:10312000DA7890073FF501AEDF78BA073FF5FDADDD
:1031300008397FF4ECADD3E5BAF1080A7FF452AE5A
:1031400087F802A02EE62846267BFEF781F90028A4
:1031500059D0AA68907840F030019170AB6842F283
:103160001072DF78BF061CD4D878800619D493F883
:1031700003805FEA886714D493F803905FEA89605C
:103180000FD493F803A05FEA8A610AD493F803B0DE
:103190005FEA8B6705D493F803C05FEA8C6040F167
:1031A00086817600F1B21971AB6842F21072DF7855
:1031B000B90728D4D878870725D4DE78B00722D479
:1031C00093F803805FEA88711DD493F803905FEA57
:1031D000897718D493F803A05FEA8A7613D493F81A
:1031E00003B05FEA8B700ED493F803C05FEA8C7172
:1031F00009D4083ADBD19A7000BFAB6880229A707C
:1032000000BF01212973256843E52846267BFEF788
:103210001FF9002862D0A868877847F030028270D2
:10322000AB6842F2107293F803805FEA88601BD4A7
:1032300093F803B05FEA8B6116D493F803C05FEA9A
:103240008C6011D493F803E05FEA8E610CD493F89C
:1032500003A05FEA8A6707D493F803905FEA896066
:1032600002D4D97889062CD57600F7B21F71AB68E5
:1032700042F2107293F803805FEA88772ED493F8B5
:1032800003B05FEA8B7629D493F803C05FEA8C77AA
:1032900024D493F803E05FEA8E761FD493F803A05A
:1032A0005FEA8A701AD493F803905FEA897115D4A3
:1032B000D9788F0712D4D87886070FD4083AD9D195
:1032C00004E0D8788706CFD4083AACD19A7000BF12
:1032D000AB6880229A7000BF01262E732568CCE56A
:1032E000986880F803B000BF9F681A7387F802904F
:1032F00000BF98688670A2E59F6887F803E000BF6A
:10330000986883F80CC080F8028000BF9F68BE7088
:1033100095E59668002E7FF48CAE87E61B80004012
:1033200028789A6842F21071D7783E0632D492F823
:1033300003E05FEA0E652DD492F803A05FEA0A6706
:1033400028D492F803905FEA096623D492F80380A8
:103350005FEA08651ED492F803B05FEA0B6719D4E0
:1033600092F803C05FEA0C6614D4D5782D0611D408
:103370000839D9D1917000BF9F688025BD7000BF0A
:1033800001201873986E00283FF4ADAD03681A68E9
:103390009047A8E50226D67099688A7842F010070F
:1033A0008F709D6828719A6842F21071D0788007FA
:1033B0001FD4D678B7071CD4D778BD0719D4D578D1
:1033C000A80716D492F803E05FEA8E7711D492F83A
:1033D00003A05FEA8A760CD492F803905FEA8975BD
:1033E00007D492F803805FEA887002D40839DDD1EF
:1033F000C0E792F803B002205FFA8BFCD0701CF09B
:10340000100246D15FEACC7637D49E680221F17073
:10341000B8E7AA680127D77000BFA868297383702E
:1034200000BFA96880268E708AE4AA680126D6703B
:1034300000BFAF682973BB7000BFA9688020887087
:1034400082E5AB681022DA7000BFAE680327002166
:103450002F73B17000BFA8688023837074E5AB68D8
:103460001022DA7000BFAF68032000212873B97002
:1034700000BFAE688023B37062E499680126CE7005
:1034800000BF9F681873BA7000BF9D688020A87045
:10349000BBE79A681021D17000BF9E680327002502
:1034A0001F73B57000BF986880228270ADE793F8F3
:1034B00003E05FEA8E613FF574AE083A7FF451AEE7
:1034C00099E600BF2DE9F04F42F292038046C05CBE
:1034D00083B0002840F0D38108F501513C310191BF
:1034E000DFF8AC95A8F1020A09F5804BD9F8047011
:1034F000D9F80860D9F80C50D9F8104009F1140C2B
:103500009CE807004FEA172E4FEA174C0CF4706C3A
:103510002EF47F6E4CEA0E0E07F0F0074FEA164CC1
:103520004EEA07074FEA162E0CF4706C2EF47F6EED
:103530004CEA0E0E06F0F0064FEA154C4EEA06066F
:103540004FEA152E0CF4706C2EF47F6E4CEA0E0EC2
:1035500005F0F0054FEA144C4EEA05054FEA142E2B
:103560000CF4706C2EF47F6E4CEA0E0E04F0F00436
:103570004FEA104C4EEA04044FEA102E0CF4706C23
:103580002EF47F6E4CEA0E0E00F0F0004FEA114C64
:103590004EEA00004FEA112E0CF4706C2EF47F6E90
:1035A0004CEA0E0E01F0F0014FEA124C4EEA010116
:1035B0004FEA122E59F8203FAAF802700CF4706CF2
:1035C0002EF47F6E4CEA0E0E02F0F0024FEA134C1E
:1035D0004EEA02024FEA132E0CF4706C2EF47F6E4A
:1035E0004CEA0E0E03F0F0034EEA030CD945AAF89C
:1035F0000460AAF80650AAF80840AAF80A00AAF837
:103600000C10AAF80E202AF810CF7FF46FAF42F208
:103610007C0758F8074094F86460002E00F0F180B1
:10362000A36842F21071DE78320627D4D8780706F4
:1036300024D4DD782E0621D4DF783D061ED493F8FD
:1036400003C05FEA0C6019D493F803905FEA096243
:1036500014D493F803A05FEA0A670FD493F803B079
:103660005FEA0B660AD40839DDD1997000BFA36800
:1036700080269E7000BF0120207327E00222DA70AE
:10368000A1688B7843F010068E70A0684025057104
:10369000A36842F21071DF78BE0709D493F803C023
:1036A0005FEA8C7504D493F803905FEA89774BD571
:1036B000DD780221EFB2D97017F0100340F0BE811F
:1036C000F80700F1AF81A4680227E77042F27C029C
:1036D00058F8023093F86450002D40F08F80019923
:1036E0009A688C6808691867DC6642F21075D778AA
:1036F00039063FD4D67837063CD492F803C05FEA47
:103700000C6737D492F803905FEA096632D492F8D6
:1037100003A05FEA0A612DD492F803B05FEA0B6759
:1037200028D4D1780E0625D4D778390622D4083D7E
:10373000DDD1957000BF9C688020A07000BF012182
:10374000197303B0BDE8F08F93F803A05FEA8A769F
:10375000AED493F803B05FEA8B75A9D4DA789007FA
:10376000A6D4DE78B207A3D4D8788707A0D40839C6
:1037700091D17AE7957945F0500696719A681221B1
:10378000D1709F68BD78012845F01006BE7000F02A
:10379000D1801A6E11680025CD711768661C0E6005
:1037A00001268E80BE60176801381FFA80F8A7F8DE
:1037B0001E8012684142F960A2F816801E6E9F6852
:1037C000306804378571B7F1804F076185823268B0
:1037D00078D20121916032681E6EAC4F002090615A
:1037E00035793D70996891F802C04CF001028A70F9
:1037F0009E6824783471012783F8647003B0BDE8B3
:10380000F08F019D20462D7BFDF722FE002856D02B
:10381000A068817841F030028270A26842F2107193
:1038200092F803905FEA896755D492F803A05FEAA3
:103830008A6650D492F803B05FEA8B604BD492F85A
:1038400003E05FEA8E6346D4D3789F0643D4D778EB
:10385000BE0640D4D678B0063DD4D07883063AD49C
:103860000839DDD1917000BFA16880238B7000BF43
:1038700042F27C070122227358F80740D0E608F58F
:10388000015242F2900614463C3418F80670019436
:103890002046812142F29109FFF75EF83946204621
:1038A000FFF75AF818F8093083B9A7210198FFF7F4
:1038B00053F842F29200002108F8001010E658F880
:1038C0000740ADE69568002D86D182E7A4210198D6
:1038D000FFF742F8EDE76D00E9B21171A36842F21B
:1038E0001072DF78B80720D4DE78B1071DD4D878FD
:1038F00085071AD4DD78A80717D493F803C05FEAC8
:103900008C7112D493F803905FEA89770DD493F801
:1039100003A05FEA8A7608D493F803B05FEA8B7558
:1039200003D4083ADDD19A709DE742F27C0458F83E
:10393000044075E69A6842F21070D5782E0620D4BD
:1039400092F803905FEA09651BD492F803A05FEA3E
:103950000A6516D492F803B05FEA0B6111D492F8AD
:1039600003805FEA08670CD4D1780E0609D4D678B4
:10397000350606D4D778390603D40838DDD19070DF
:1039800030E002252478D570986890F802C04CF099
:103990001002827099680C719A6842F21071D678A0
:1039A000B40727D4D778B80724D4D578AE0721D464
:1039B000D478A5071ED492F803905FEA897419D4CD
:1039C00092F803A05FEA8A7014D492F803B05FEA19
:1039D0008B770FD492F803805FEA88760AD408398F
:1039E000DDD1917000BF9E688027B77000BF0125B0
:1039F0001D730DE092F803C002205FFA8CF1D070C5
:103A000011F0100234D1CF0726D49A680221D17068
:103A1000986E00283FF4F2AE03681A6803B0BDE860
:103A2000F04F1047A2680126D67000BFA06821732E
:103A3000837000BFA5688021A97044E6A7681023A1
:103A4000FB7000BFA668032000222073B27000BF85
:103A5000A5688021A97036E69E680127F77000BF2F
:103A60009D681873AA7000BF9C688020A070CCE786
:103A70009A681021D17000BF9E68032700251F732C
:103A8000B57000BF9C688020A070BEE71B8000401E
:103A90003C34FF1F10B4036841681A7890F809C0DD
:103AA0000C78037A14EA0C0F02EA03021DD0847A20
:103AB00004F003010AB141F0040141F008039A1037
:103AC00003F1FF3C8272BCF10D0F0BD8DFE80CF064
:103AD00021071B070A152121150A071B0721C268A8
:103AE000531EC3605DF8044B7047817A01F00303F5
:103AF000002AE4D043F00403E1E7C3689C1EC460DD
:103B00005DF8044B7047C1685DF8044B0231C16039
:103B10007047C4680134C4605DF8044B704700BF4F
:103B200008B5034BD3F8EC00FFF7B4FF08BD00BFA6
:103B300074DE012008B5034BD3F8E800FFF7AAFFB5
:103B400008BD00BF74DE012008B5034BD3F8E400C4
:103B5000FFF7A0FF08BD00BF74DE012008B5034BCE
:103B6000D3F8E000FFF796FF08BD00BF74DE012028
:103B700008B5034BD3F8DC00FFF78CFF08BD00BF8E
:103B800074DE012008B5034BD3F8D800FFF782FF9D
:103B900008BD00BF74DE012008B5034BD3F8D40084
:103BA000FFF778FF08BD00BF74DE012008B5034BA6
:103BB000D3F8D000FFF76EFF08BD00BF74DE012010
:103BC00008B5034BD3F8CC00FFF764FF08BD00BF76
:103BD00074DE012008B5034BD3F8C800FFF75AFF85
:103BE00008BD00BF74DE012008B5034BD3F8C40044
:103BF000FFF750FF08BD00BF74DE012008B5034B7E
:103C0000D3F8C000FFF746FF08BD00BF74DE0120F7
:103C100008B5034BD3F8BC00FFF73CFF08BD00BF5D
:103C200074DE012008B5034BD3F8B800FFF732FF6C
:103C300008BD00BF74DE012008B5034BD3F8B40003
:103C4000FFF728FF08BD00BF74DE012008B5034B55
:103C5000D3F8B000FFF71EFF08BD00BF74DE0120DF
:103C600008B5034BD3F8AC00FFF714FF08BD00BF45
:103C700074DE012008B5034BD3F8A800FFF70AFF54
:103C800008BD00BF74DE012008B5034BD3F8A400C3
:103C9000FFF700FF08BD00BF74DE012008B5034B2D
:103CA000D3F8A000FFF7F6FE08BD00BF74DE0120C8
:103CB00008B5034BD3F89C00FFF7ECFE08BD00BF2E
:103CC00074DE012008B5034BD3F89800FFF7E2FE3D
:103CD00008BD00BF74DE012008B5034BD3F8940083
:103CE000FFF7D8FE08BD00BF74DE012008B5034B06
:103CF000D3F89000FFF7CEFE08BD00BF74DE0120B0
:103D000008B5034BD3F88C00FFF7C4FE08BD00BF15
:103D100074DE012008B5034BD3F88800FFF7BAFE24
:103D200008BD00BF74DE012008B5034BD3F8840042
:103D3000FFF7B0FE08BD00BF74DE012008B5034BDD
:103D4000D3F88000FFF7A6FE08BD00BF74DE012097
:103D500008B5024BD86FFFF79DFE08BD74DE012049
:103D600008B5024B986FFFF795FE08BD74DE012081
:103D700008B5024B586FFFF78DFE08BD74DE0120B9
:103D800008B5024B186FFFF785FE08BD74DE0120F1
:103D900008B5024BD86EFFF77DFE08BD74DE01202A
:103DA00008B5024B986EFFF775FE08BD74DE012062
:103DB00008B5024B586EFFF76DFE08BD74DE01209A
:103DC00008B5024B186EFFF765FE08BD74DE0120D2
:103DD00008B5024BD86DFFF75DFE08BD74DE01200B
:103DE00008B5024B986DFFF755FE08BD74DE012043
:103DF00008B5024B586DFFF74DFE08BD74DE01207B
:103E000008B5024B186DFFF745FE08BD74DE0120B2
:103E100008B5024BD86CFFF73DFE08BD74DE0120EB
:103E200008B5024B986CFFF735FE08BD74DE012023
:103E300008B5024B586CFFF72DFE08BD74DE01205B
:103E400008B5024B186CFFF725FE08BD74DE012093
:103E500008B5024BD86BFFF71DFE08BD74DE0120CC
:103E600008B5024B986BFFF715FE08BD74DE012004
:103E700008B5024B586BFFF70DFE08BD74DE01203C
:103E800008B5024B186BFFF705FE08BD74DE012074
:103E900008B5024BD86AFFF7FDFD08BD74DE0120AE
:103EA00008B5024B986AFFF7F5FD08BD74DE0120E6
:103EB00008B5024B586AFFF7EDFD08BD74DE01201E
:103EC00008B5024B186AFFF7E5FD08BD74DE012056
:103ED00008B5024BD869FFF7DDFD08BD74DE01208F
:103EE00008B5024B9869FFF7D5FD08BD74DE0120C7
:103EF00008B5024B5869FFF7CDFD08BD74DE0120FF
:103F000008B5024B1869FFF7C5FD08BD74DE012036
:103F100008B5024BD868FFF7BDFD08BD74DE01206F
:103F200008B5024B9868FFF7B5FD08BD74DE0120A7
:103F300008B5024B5868FFF7ADFD08BD74DE0120DF
:103F400001380B463A2800F25C82DFE810F0530299
:103F50004C0245023E0237023002290222021B02B5
:103F6000AE01A701A001990192018B0184017D019D
:103F700076016F01680161015A0153014C0145014D
:103F80003E0137013001290122011B0113010B0100
:103F90000301FB00F300EB00E300DB00D300CB00E8
:103FA000C300BB00B300AB00A3009B0093008B00D9
:103FB00083007B0073006B0063005B0053004B00C9
:103FC00043003B00BC4ABD49C2F8EC303B20042210
:103FD0000CF000BAB848BA49C0F8E83004223A20D8
:103FE0000CF0F8B9B44AB749C2F8E43039200422D9
:103FF0000CF0F0B9B048B449C0F8E03004223820E1
:104000000CF0E8B9AC4AB149C2F8DC3037200422E0
:104010000CF0E0B9A848AE49C0F8D83004223620E8
:104020000CF0D8B9A44AAB49C2F8D43035200422E8
:104030000CF0D0B9A048A849C0F8D03004223420F0
:104040000CF0C8B99C4AA549C2F8CC3033200422F0
:104050000CF0C0B99848A249C0F8C83004223220F8
:104060000CF0B8B9944A9F49C2F8C43031200422F8
:104070000CF0B0B990489C49C0F8C0300422302000
:104080000CF0A8B98C4A9949C2F8BC302F20042200
:104090000CF0A0B988489649C0F8B83004222E2008
:1040A0000CF098B9844A9349C2F8B4302D20042208
:1040B0000CF090B980489049C0F8B03004222C2010
:1040C0000CF088B97C4A8D49C2F8AC302B20042210
:1040D0000CF080B978488A49C0F8A83004222A2018
:1040E0000CF078B9744A8749C2F8A4302920042218
:1040F0000CF070B970488449C0F8A0300422282020
:104100000CF068B96C4A8149C2F89C30272004221F
:104110000CF060B968487E49C0F898300422262027
:104120000CF058B9644A7B49C2F894302520042227
:104130000CF050B960487849C0F89030042224202F
:104140000CF048B95C4A7549C2F88C30232004222F
:104150000CF040B958487249C0F888300422222037
:104160000CF038B9544A6F49C2F884302120042237
:104170000CF030B950486C49C0F88030042220203F
:104180000CF028B94C4A6949D3671F2004220CF06F
:1041900021B949486649836704221E200CF01AB9E8
:1041A000454A644953671D2004220CF013B9424864
:1041B0006149036704221C200CF00CB93E4A5F4998
:1041C000D3661B2004220CF005B93B485C4983668A
:1041D00004221A200CF0FEB8374A5A4953661920B7
:1041E00004220CF0F7B8344857490366042218201B
:1041F0000CF0F0B8304A5549D365172004220CF072
:10420000E9B82D4852498365042216200CF0E2B823
:10421000294A50495365152004220CF0DBB8264882
:104220004D490365042214200CF0D4B8224A4B49AE
:10423000D364132004220CF0CDB81F48484983648E
:10424000042212200CF0C6B81B4A464953641120C0
:1042500004220CF0BFB8184843490364042210201C
:104260000CF0B8B8144A4149D3630F2004220CF073
:10427000B1B811483E49836304220E200CF0AAB85D
:104280000D4A3C4953630D2004220CF0A3B80A48A0
:104290003949036304220C200CF09CB8064A3749C4
:1042A000D3620B2004220CF095B803483449836292
:1042B00004220A200CF08EB874DE0120213B00009D
:1042C000353B0000493B00005D3B0000713B0000B6
:1042D000853B0000993B0000AD3B0000C13B000066
:1042E000D53B0000E93B0000FD3B0000113C000015
:1042F000253C0000393C00004D3C0000613C0000C2
:10430000753C0000893C00009D3C0000B13C000071
:10431000C53C0000D93C0000ED3C0000013D000020
:10432000153D0000293D00003D3D0000513D0000CD
:10433000613D0000713D0000813D0000913D0000A5
:10434000A13D0000B13D0000C13D0000D13D000095
:10435000E13D0000F13D0000013E0000113E000083
:10436000213E0000313E0000413E0000513E000071
:10437000613E0000713E0000813E0000913E000061
:10438000A13E00001F4A20495362092004220CF07C
:1043900021B81C481D490362042208200CF01AB8F9
:1043A000184A1B49D361072004220CF013B81548A2
:1043B00018498361042206200CF00CB8114A1649F2
:1043C0005361052004220CF005B80E48134903611F
:1043D000042210460BF0FEBF0A4A1149D3600320A5
:1043E00004220BF0F7BF07480E4983600422022025
:1043F0000BF0F0BF034A0C495360012004220BF07C
:10440000E9BF704774DE0120B13E0000C13E0000EC
:10441000D13E0000E13E0000F13E0000013F0000FF
:10442000113F0000213F0000313F000070B5234BD9
:10443000036104460D46164600216FF00042C2603B
:10444000836181724561C6610221E8B20CF0B0FC63
:10445000207F02210CF0ACFC194850F835100122E5
:1044600001F500732360227250F83600627200F585
:104470000071616002200CF0FBFC226894F808C017
:10448000137813EA0C0F03D0A07A40F00101A17257
:10449000626894F809E0137813EA0E0F03D0A07A4B
:1044A00040F00201A17228462146FFF749FD30463F
:1044B0002146FFF745FD204670BD00BFA4800100E6
:1044C00010350400F0B486B072B6C36862B6BC4C56
:1044D000026A25680595059F466A9B08BD1A9E1BC2
:1044E000826A18BF0762012D4362B8BF0125B70277
:1044F00097FBF5F312B1002B40F0498102EB420229
:10450000D71848BF0337BB1083EAE375A5EBE37CFC
:10451000ACF10202012A836240F33F8197103B1FF6
:10452000A7F10B0523EAE37C002DA8BFAC440137BB
:104530006744012F00F03181013F7A00C36A02FB1A
:104540000636C662CE6272B6C56B62B62268049247
:10455000466D049F026DAB089E1BA7EB020518BFBA
:104560000765876D4365012DB8BF0125B20292FB37
:10457000F5F317B1002B40F0028107EB4707FA185B
:1045800048BF0332931083EAE375A5EBE37CACF1FB
:104590000207012F836540F3F880BA10131FA2F1C0
:1045A0000B0523EAE37C002DA8BFAC440132624432
:1045B000012A00F0EA80013A5700C36D07FB063676
:1045C000C6650E6372B6C56E62B62768D0F88460A1
:1045D0000397AB08039FD0F88020C0F884309E1B5F
:1045E000A7EB020518BFC0F88070D0F88870012DC5
:1045F000B8BF0125B20292FBF5F317B1002B40F0D2
:10460000B58007EB4707FA1848BF0332931083EAD7
:10461000E375A5EBE37CACF10207012FC0F888300D
:1046200040F3AB80BA10131FA2F10B0523EAE37C21
:10463000002DA8BFAC4401326244012A00F09D80E5
:10464000013A5700D0F88C3007FB0636C0F88C6072
:104650004E6372B6D0F89C5062B62768D0F8B4604A
:104660000297AB08029FD0F8B020C0F8B4309E1B70
:10467000A7EB020518BFC0F8B070D0F8B870012DD4
:10468000B8BF0125B20292FBF5F30FB1002B65D143
:1046900007EB4707FA1848BF0332931083EAE37524
:1046A000A5EBE37CACF10207012FC0F8B8305BDD6D
:1046B000BA10131FA2F10B0523EAE37C002DA8BF5B
:1046C000AC4401326244012A4ED0013A5700D0F87E
:1046D000BC3007FB0636C0F8BC608E6372B6D0F8FB
:1046E000CC7062B624680194D0F8E450019ED0F8F2
:1046F000E020BB085D1BA6EB020718BFC0F8E06016
:10470000D0F8E860C0F8E430012FB8BF0127AC0250
:1047100094FBF7F20EB1002A1CD106EB4606B41842
:1047200048BF0334A31083EAE37CACEBE372254F6C
:10473000961E87FB064CACEBE6770137D0F8EC40D1
:10474000C0F8E83007FB0545C0F8EC50CD6306B073
:10475000F0BC704726DD002EDFDC25E027DD002FD2
:1047600096DC0025C0F8B8500127B0E722DD002F05
:104770003FF747AF0025C0F88850012762E71CDDEE
:10478000002F3FF7FAAE00258565012715E706DD06
:10479000002A3FF7B3AE002585620122CEE6002A4B
:1047A000F9DCABE6002EB8DD01270023C6E7002FB9
:1047B000D7DC6DE7002FDDDC23E7002FE3DCDCE650
:1047C000ACE00120ABAAAA2A2DE9F04F854B854A1F
:1047D000DD6A196854689BB0002D1191064640F3BC
:1047E0008181032D57DC304610F08AF83278002A98
:1047F0005AD000284FF0000EACBF07466FF00047BC
:10480000F44606F1FF38012018F8013F33B99FB98B
:1048100018F8013F4FF0FF37002BF8D00A2B04D0D7
:104820001F2BF1D90EF1060EEEE7F445B8BFF446A2
:1048300001304FF0000EE7E76A4FB96A083100FB1C
:1048400001F06849F44505FB00F7C8686346B8BF46
:10485000734605FB03F3012816932CD0022800F0C1
:104860004481604B1969012930D0022908BFE41B3B
:104870005C4BDFF870B1D3F818E0196A119B01EBBB
:104880000E0843459C4603DA16998C44E64522DB24
:104890001BB0BDE8F08F53480325C562304610F0C9
:1048A0002FF83278002AA4D14E491692C868012800
:1048B0004FEAC507D2D11699119B01EBD179A3EB31
:1048C0006901484B119119690129CED107EBD77ABB
:1048D000A4EB6A04CCE7DBF81CE0DBF8243073447B
:1048E0009C42D5DA2744BE45D2DA002AD0D00996B8
:1048F000CDF864B00A2A099F00F0DB853E461346D6
:10490000002102E00A2B00F0A0831F2B16F8013FC4
:1049100088BF0131002BF5D101EB410E4FEA4E016A
:10492000179605FB01FE2F4EB76A083705FB07F9FE
:104930000128A9EBC50600F09283022800F0B1859A
:10494000119806902749087D002840F0D38009EB94
:1049500004032644022D0E93109600F08A83032D43
:1049600040F0FF80002A00F0AE810A2A00F0AB81FF
:104970001C4E109D1B4C316A776AD6F81890D6F8F9
:104980001CB0237A0293203AEE01D0B2AB1C09EBA3
:10499000010A01350BEB07016B2806F102070391B1
:1049A0000A970C930B9500F226830F4E56F8207051
:1049B0003E78069C0A990D4B059701EB04080022EE
:1049C000601CA11CDDF830E0DDF82CC0109F0492C3
:1049D00007909844089108462246079944460023C8
:1049E00035E000BF70D0FF1F80FD01004034FF1F85
:1049F000814500F37381824540F37081894540F31E
:104A00004782BB4505DC039DBD42C4BF9DF80850ED
:104A10002570E34506DC039D654503DD9DF80850E0
:104A200084F88050F34506DC039D754503DD9DF851
:104A3000085084F800510133062B02F1030204F1FF
:104A4000030401F1030100F1030000F0678146FA5D
:104A500003F5ED07EFD59145CADC824500F373817C
:104A6000814540F39681894500F37281924540F378
:104A70000582BB4500F38982039DBD4240F38582D8
:104A80009DF8085004F8025C8A4506DD9DF8085040
:104A900004F8015C924540F3E381E34500F3E081D3
:104AA000039D654540F3DC819DF8085084F87E50F5
:104AB0008A4540F3AE829DF8085084F87F509245B5
:104AC00040F32481F345B6DC039D7545B3DD9DF8C5
:104AD000085084F8FE508A45ADDD9DF8085084F8F2
:104AE000FF50A8E70125D5627DE6119B16995B1A58
:104AF0001193B6E6199A517D9069D2F81CA0136AF9
:104B0000576A0091069909EB04028946F14400EBCB
:104B1000030E0E920EF1FF3809F1FF3242450AEB07
:104B2000070B0E9FA8BF42468842B8BF08460BF14C
:104B3000FF3307F1FF3CA2455146B8BF214663450C
:104B4000A8BF6346FCF710FC3019099E1090022D97
:104B5000327800F08E82032D3FF404AF002A00F07B
:104B6000B2800A2A00F0AF80B94DB94FD5F81CB019
:104B7000387A6B6A109FA9692E6A069D07905B447C
:104B8000F80105350E44059306900837A2F1200A76
:104B90005FFA8AF36B2B96BFAE4AAF4C52F82340B4
:104BA000069AAE4B03955019013C05F1FF3E109A51
:104BB000CDF810E01844A5F1050AA5F10409A5F106
:104BC0000308A5F1020C0294029D15F8013F02951D
:104BD000DC070FD551450DDC56450BDD934509DC4F
:104BE000059C944206DD039D441B9DF81C5004F86F
:104BF0000A50A6469D070FD549450DDC4E450BDDF5
:104C0000934509DC059C944206DD039D441B9DF8F9
:104C10001C5004F80950A6465C070FD541450DDC31
:104C200046450BDD934509DC059C944206DD039D5A
:104C3000441B9DF81C5004F80850A6461D070FD5CC
:104C40008C450DDBB4450BDA934509DC059C944299
:104C500006DD039D441B9DF81C5004F80C50A6462D
:104C6000DC0611D5049DA9422C460DDCAE420BDDBD
:104C7000934509DC059C944206DD039C041BA64673
:104C80009DF81C400EF805409B060CD5039B9942ED
:104C900009DC9E4207DD934505DC059D9542C4BFB6
:104CA0009DF81C5005700132974200F180008BD1B5
:104CB0000998039D10F8012F099022B10A2A05F1E5
:104CC00006057FF463AF179E0E9C3278002A3FF4EE
:104CD000DFAD5F490996CD6AC8680BE689453FF7A5
:104CE000AAAE8A457FF7A7AEBB4506DC039DBD4251
:104CF00003DD9DF8085004F8015CE34506DC039DE4
:104D0000654503DD9DF8085084F87F50F3453FF773
:104D100092AE039D75453FF7E0AE8CE6049E0336E8
:104D2000182E049608F5C0780EF1030E07F103075C
:104D30000CF1030C00F04D81059A089812F8016FF0
:104D40000592069A49E6814551DD4945BFF68EAE8A
:104D500092457FF770AEBB4506DC039DBD4203DD87
:104D60009DF8085004F8025CE34506DC039D6545A8
:104D700003DD9DF8085084F87E50F3453FF75BAEA5
:104D8000039D75457FF757AE9DF8085084F8FE5097
:104D900051E68945DCDC924540F34281BB4500F396
:104DA0004A81039DBD4240F346819DF8085004F8B6
:104DB000025C8A4506DD9DF8085004F8015C9245C6
:104DC00040F31C81E34500F31981039D654540F3E1
:104DD00015819DF8085084F87E508A4540F32E8155
:104DE0009DF8085084F87F5092458FDD6AE68A4529
:104DF0007ADC924540F3D980BB450CDC039DBD4273
:104E000009DD9DF8085004F8025C9DF808502570F3
:104E1000924540F3D080E3450DDC039D65450ADDF6
:104E20009DF8085084F87E509DF8085084F8805012
:104E300092457FF7F7ADF3453FF7FDAD039D75450F
:104E40007FF7F9AD9DF8085084F8FE50EFE500BFFC
:104E500070D0FF1F80FD0100CC9C01004034FF1F7B
:104E60008A4507DDE3453FF72AAE039D65457FF799
:104E700026AE20E692457FF7DEAD23E68A45F9DDD2
:104E8000BB453FF707AE039DBD427FF703AEFDE58F
:104E90008A457EDDBB450BDC039DBD4208DD9DF8E8
:104EA000085004F8015C9DF8085025708A4575DDAE
:104EB000E3450DDC039D65450ADD9DF8085084F847
:104EC0007F509DF8085084F880508A457FF7AAAD3E
:104ED000F3453FF7B0AD039D75457FF7ACAD9DF849
:104EE000085084F8FF50A2E5924542DDBB4540DC06
:104EF000039DBD423DDD9DF8085004F8025C8945E4
:104F00003EDD039DBD4202DD9DF8085025709245AF
:104F10001FDDE3451DDC039D65451ADD9DF8085046
:104F200084F87E5089451BDD039D654503DD9DF8B2
:104F3000085084F88050924517DDF34515DC039D39
:104F4000754512DD9DF8085084F8FE508945C6DD90
:104F50006AE5894537DCE345EDDC039D6545EADD1F
:104F60009DF8085084F87F50E1E789453FF75AAD36
:104F7000AEE789452ADCBB45C9DC039DBD42C6DDE1
:104F80009DF8085004F8015CBEE78A453FF778AF0A
:104F900083E5BB4502DC039DBD4284DCE3453FF76E
:104FA00041AD039D65458CDC3CE5BB4503DC039DC1
:104FB000BD423FF72AAFE3453FF734AD039D65455A
:104FC0003FF732AF2EE5E345B5DCADE7BB459EDCF0
:104FD00097E70999069B11F8012F0991123306935F
:104FE000002A3FF470AE0A2A3FF46DAE203AD0B2E8
:104FF0006B287FF6DAAC9B4F0026DAE48A457FF710
:1050000039AFE3453FF7F0AE039D65457FF7ECAE62
:10501000E6E692453FF756AD8A453FF777AE0AE59B
:105020008A457FF727AFBB453FF7C9AE039DBD4219
:105030007FF7C5AEBFE68A45F5DCC3E692453FF78C
:1050400041AD8A457FF7F7AC60E601EB41077B0095
:10505000179605FB03FE37460137179763E416984A
:10506000119BCEEB000A0AEBDA7B03EB6B0706978A
:1050700068E4002A3FF427AE0A2A3FF424AE7A4FB0
:10508000069B796AFE693D6ABC69774898465F1C51
:1050900006EB010A0B334146093104EB050B0F9374
:1050A0004546434690F808900C910A35591D4046F4
:1050B000083003970D95DF1D9D1D0691203A10992C
:1050C00004900B97181DDF1C0A95C8469D1C994635
:1050D000D3B201316B2B089007970595189100F218
:1050E0004281624850F823703978109A189B0297D1
:1050F00000208CE0CD0711D5039DA542C0F29F8111
:10510000A14580F2E3815D4508DAB34206DB5345F1
:1051100004DA574F07EBC31C0CF805808D0713D535
:10512000079D059FAC4200F37581BC4240F3C881E6
:10513000079DAB4508DD9E4206DC9A4504DD4C4FD9
:1051400007EBC31C0CF805804F0713D5069D089F7D
:10515000AC4200F30B81BC4240F3BB81069DAB45E2
:1051600008DD9E4206DC9A4504DD414F07EBC31C77
:105170000CF805800D0713D50B9D0A9FA542C0F2C0
:105180000A81BC4240F3A9810B9D5D4508DA9E422D
:1051900006DC9A4504DD364F07EBC31C0CF805808E
:1051A000CF0613D50C9D049FAC4200F30981BC428D
:1051B00040F397810C9DAB4508DD9E4206DC9A4585
:1051C00004DD2B4F07EBC31C0CF805808D0613D5AF
:1051D0000F990D9DA142C0F20881AC4240F36D8150
:1051E0000F9F5F4508DA9E4206DC9A4504DD2049A0
:1051F00001EBC31505F807800130082802F102020F
:1052000003F102037DD0029F17F8011F0297964217
:105210003FF770AF924513DCCF077FF57FAF039D5B
:10522000A542C0F22A81A14580F24D815D45BFF6BD
:1052300075AF9E423FF772AF9A457FF76FAF68E751
:105240000B4DDDF80CC0CDF8509005EBC217084DA2
:10525000129705EBC3151395CE460027029D1592B4
:1052600022E000BFCC9C010070D0FF1F80FD010038
:105270004034FF1FDE4502DA129A02F80E806445C0
:105280001BDDDE4509DA9E4204DC9A45C4BF139A51
:1052900002F80E80644540F3EC800137062F0CF1D4
:1052A000020C0EF1020E21D041FA07F919F0010F9C
:1052B000F3D0A645DEDA6445EFDCE34540F3D38066
:1052C000129AA64502F80C8080F2D0809E42E4DC5F
:1052D0009A45C8BF139A07F10107C8BF02F80C80AE
:1052E000062F0CF1020C0EF1020EDDD1159ADDF83D
:1052F000509002950130082802F1020203F10203E6
:1053000081D1099810F8012F099009F10C09002AA0
:105310003FF4D9AC039B0F990D9D0C9F04980C335F
:1053200003930B9B0C310C350C370C300C330F9165
:105330000D950A99069D0C970490089F07980B936A
:10534000059B0C310C350C370C300C330A2A0A91B2
:1053500006950897079005933FF4B5AC203AD3B271
:105360006B2B7FF6BEAE614F0021BEE6BC423FF71D
:1053700001AFBB457FF7FEAE9E4207DC9A4505DDD7
:105380005B4D089F05EBC31C0CF80780069DAC42E3
:105390003FF7F0AEE2E6BC423FF702AFBB457FF716
:1053A000FFAE9E4207DC9A4505DD514D0A9F05EB95
:1053B000C31C0CF807800B9DA542FFF6F1AEE3E697
:1053C000BC423FF703AFBB457FF700AF9E4207DC0F
:1053D0009A4505DD464D049F05EBC31C0CF807807C
:1053E0000C9DAC423FF7F2AEE4E6AC423FF704AFAF
:1053F000AB457FF701AF9E4207DC9A4505DD3C4F88
:105400000D9907EBC31C0CF801800F9DA542FFF618
:10541000F3AEE5E6BC423FF797AEBB457FF794AEEF
:105420009E4207DC9A4505DD314D059F05EBC31C07
:105430000CF80780079DAC423FF786AE78E6A145A1
:10544000FFF66CAED945BFF669AE9E4206DC9A45C2
:1054500004DD274F07EBC31C0CF80980039DA54210
:10546000FFF65CAE4FE6A645FFF617AFDE45FFF64A
:105470000AAFE3453FF72AAF0FE7A145FFF64EAE6F
:10548000D945BFF64BAE9E4206DC9A4504DD184D69
:1054900005EBC31707F80980039DA542FFF63EAE52
:1054A000C4E6169B1199CEEB03070F440697FFF74E
:1054B00049BA17974FF0000ECEE5AB459BDC8FE65F
:1054C000BB45ADDC34E6D945DDDBAFE6D945BCDB19
:1054D00019E6BB453FF750AF40E6BB453FF761AF2C
:1054E00052E6BB453FF772AF64E600BFCC9C0100BB
:1054F0004034FF1F0FB410B582B004AB074C53F813
:10550000042B0193402120460FF0D4FA2046FFF7E8
:105510005BF902B0BDE8104004B07047FC33FF1FD8
:105520002DE9F04F8BB00B4605919946059B6E4ACD
:10553000D3F8986F6D4CDFF8D8816D4D029201F56C
:105540004B7000276B4900974FF0260B731C03909C
:10555000049101945F4600F0B4810098864214BF24
:105560007724FF240146634E99F8203056F831A085
:105570000A46CE00002B6BD0012B40F085835A48A1
:1055800099F822108259029EC8F82C307068C8F829
:1055900000200223012988F80840C8F80400C8F850
:1055A0000C3000F0C183C0F08483994240F07B83CB
:1055B000514A524E0AEBC71C624406F5D257A6F177
:1055C000C00396465968043309B18EF80040586804
:1055D0000EF1010B08B18EF80140996809B18BF802
:1055E0000140D86808B18BF80240196909B18BF8FD
:1055F0000340586908B18BF80440996909B18BF8E8
:105600000540D8691C3308B18BF80640B3420BF152
:10561000070ED7D103F1C006BE4202F18002CED1FF
:105620003748FFF7D1F8374A009E99F823700FCA20
:105630000DF1180A8AE80F005AF82660042F00F2CC
:105640002C83DFE817F0AF023702C5014101670084
:10565000264999F821B051F832302B4E2B49019848
:10566000C8F80030BBF1000F08BF31464268C8F8E7
:105670000420084601230221C8F80C1088F80840CD
:10568000C8F82C30FFF7A0F852461B49DDF80CC0D3
:1056900007F1230A02F1300B5CF8047F07F5004E96
:1056A000CEEB0E10470085FB07633B44FE17C6EBAD
:1056B000E3300230C0EB0A03981E5F1E5E1C01EB54
:1056C000C01E981C01EBC71701EBC61601EBC313F4
:1056D00001EBC0100EF80240BC549C54B4548454E6
:1056E00001329345D8D19EE730810100108101003D
:1056F00001800080508101004034FF1F4883010079
:10570000E0FF01008C810100CCFF0100D0FF01000F
:1057100070D0FF1FA54AA64B32440027186818B165
:1057200002F51B5B8BF82F40596819B102F51B5C21
:105730008CF83040986818B102F51B5E8EF8314045
:10574000D96819B102F51B5A8AF83240186918B1A4
:1057500002F51B5B8BF83340596919B102F51B5CEC
:105760008CF83440986918B102F51B5E8EF835400C
:10577000D96919B102F51B5A8AF83640186A18B16E
:1057800002F51B5B8BF83740596A19B102F51B5CB7
:105790008CF83840986A18B102F51B5E8EF83940D3
:1057A000D96A19B102F51B5A8AF83A40186B18B138
:1057B00002F51B5B8BF83B40596B19B102F51B5C82
:1057C0008CF83C40986B18B102F51B5E8EF83D409A
:1057D000D96B19B102F51B5A8AF83E40186C18B102
:1057E00002F51B5B8BF83F400137072F03F14403A1
:1057F00002F1800292D1009A059F88F8084002EBDE
:10580000820307EB830CC8F8006002240126C8F865
:105810000C40C8F82C60BCF82010664FB1F5807FB2
:105820000BD0D9F824206449644B65485924002AD8
:10583000C8BF19467C60FFF75DFE6322D9F82810C7
:105840006048C8F804205D4EFFF754FED9F82C20BC
:1058500059495B48002AC8BF31466E27C8F8047012
:10586000FFF748FE009CD9F83010574B049A554872
:10587000013403EB810A27460094039CDAED007A99
:1058800008320492164604F57172BDEEE70A029CD6
:105890000392019A7823083210EE101A0834029409
:1058A0000192C8F80430FFF725FE042F09F114090E
:1058B00000F0F081059B7768D3F8986F731C7FF434
:1058C0004CAEAA2400994EE6384A404B3244002799
:1058D000196819B102F51B5C8CF82F40586818B193
:1058E00002F51B5E8EF83040996819B102F51B5A1B
:1058F0008AF83140D86818B102F51B5B8BF832404A
:10590000196919B102F51B5C8CF83340586918B15C
:1059100002F51B5E8EF83440996919B102F51B5AE5
:105920008AF83540D86918B102F51B5B8BF8364010
:10593000196A19B102F51B5C8CF83740586A18B126
:1059400002F51B5E8EF83840996A19B102F51B5AB0
:105950008AF83940D86A18B102F51B5B8BF83A40D7
:10596000196B19B102F51B5C8CF83B40586B18B1F0
:1059700002F51B5E8EF83C40996B19B102F51B5A7B
:105980008AF83D40D86B18B102F51B5B8BF83E409E
:10599000196C19B102F51B5C8CF83F400137072FD9
:1059A00003F1440302F1800292D124E74034FF1F47
:1059B000EC02020070D0FF1F64000200D4FF01005F
:1059C000680002007000020024A00100A4FB010096
:1059D000714A724B32440027186818B102F51B5EF9
:1059E0008EF82F40596819B102F51B5A8AF83040D9
:1059F000986818B102F51B5B8BF83140D96819B172
:105A000002F51B5C8CF83240186918B102F51B5E78
:105A10008EF83340596919B102F51B5A8AF834409F
:105A2000986918B102F51B5B8BF83540D96919B13B
:105A300002F51B5C8CF83640186A18B102F51B5E43
:105A40008EF83740596A19B102F51B5A8AF8384066
:105A5000986A18B102F51B5B8BF83940D96A19B105
:105A600002F51B5C8CF83A40186B18B102F51B5E0E
:105A70008EF83B40596B19B102F51B5A8AF83C402D
:105A8000986B18B102F51B5B8BF83D40D96B19B1CF
:105A900002F51B5C8CF83E40186C18B102F51B5ED9
:105AA0008EF83F400137072F03F1440302F18002D3
:105AB00092D1A0E6384A3A4B32440027196819B10E
:105AC00002F51B5A8AF82F40586818B102F51B5B83
:105AD0008BF83040996819B102F51B5C8CF83140A5
:105AE000D86818B102F51B5E8EF83240196919B1F9
:105AF00002F51B5A8AF83340586918B102F51B5B4E
:105B00008BF83440996919B102F51B5C8CF835406B
:105B1000D86918B102F51B5E8EF83640196A19B1C2
:105B200002F51B5A8AF83740586A18B102F51B5B18
:105B30008BF83840996A19B102F51B5C8CF8394032
:105B4000D86A18B102F51B5E8EF83A40196B19B18C
:105B500002F51B5A8AF83B40586B18B102F51B5BE3
:105B60008BF83C40996B19B102F51B5C8CF83D40F9
:105B7000D86B18B102F51B5E8EF83E40196C19B156
:105B800002F51B5A8AF83F400137072F03F14403FF
:105B900002F1800292D12EE64034FF1F540702002A
:105BA000C8040200794A7A4B32440027186818B1B9
:105BB00002F51B5B8BF82F40596819B102F51B5C8D
:105BC0008CF83040986818B102F51B5E8EF83140B1
:105BD000D96819B102F51B5A8AF83240186918B110
:105BE00002F51B5B8BF83340596919B102F51B5C58
:105BF0008CF83440986918B102F51B5E8EF8354078
:105C0000D96919B102F51B5A8AF83640186A18B1D9
:105C100002F51B5B8BF83740596A19B102F51B5C22
:105C20008CF83840986A18B102F51B5E8EF839403E
:105C3000D96A19B102F51B5A8AF83A40186B18B1A3
:105C400002F51B5B8BF83B40596B19B102F51B5CED
:105C50008CF83C40986B18B102F51B5E8EF83D4005
:105C6000D96B19B102F51B5A8AF83E40186C18B16D
:105C700002F51B5B8BF83F400137072F03F144030C
:105C800002F1800292D1B6E5BE2242494248FBF7BA
:105C9000DFFAC8E40BB0BDE8F08FD9223F49404895
:105CA000FBF7D6FAA7E588223E493F48FBF7D0FA32
:105CB000B9E4364A3D4E0AEBC71A524406F5D25EA5
:105CC000A6F1C00393465968043309B18BF800402C
:105CD00058680BF1010C08B18BF80140996809B1C3
:105CE0008CF80140D86808B18CF80240196909B1F4
:105CF0008CF80340586908B18CF80440996909B1DF
:105D00008CF80540D8691C3308B18CF806409E42D7
:105D10000CF1070BD7D1C036764502F18002CFD106
:105D20002348FEF751FD7EE4184A224E0AEBC717BE
:105D30003A44A6F1C00310465968043301B1047017
:105D40005F68411C07B14470986800B14C70DF680F
:105D500007B18C70186900B1CC705F6907B10C7124
:105D6000986900B14C71DF691C3307B18C71B34283
:105D700001F10700E0D103F1C0060F4B9E4202F192
:105D80008002D6D10D48FEF71FFD4CE44034FF1FC2
:105D9000840902007CFF01000C000200A40602003E
:105DA00038000200F8060200E4FF010020E20100D2
:105DB000D8FF01001C0C02005C260200DCFF010081
:105DC0002DE9F04F8DB001F54B706B4E0791002718
:105DD00089466A4A6A49DFF8C8816A4C6A4D03916C
:105DE0004FF0260B04960590069202975E463946C0
:105DF000634899F8203050F831A0CF00002B6DD0C7
:105E0000012B40F086835D4899F82210C259069F05
:105E1000C8F800207868C8F82C30772202230129BE
:105E2000C8F80400C8F80C3088F8082000F0508545
:105E3000C0F01085994240F0E084544F0AEBC6163A
:105E4000A61907F5D25EA7F1C003B446B346596858
:105E5000043309B18CF8002058680CF1010A08B12C
:105E60008CF801209E680EB18AF80120D96809B12A
:105E70008AF80220186908B18AF803205E690EB119
:105E80008AF80420996909B18AF80520D8691C3379
:105E900008B18AF80620BB420AF1070CD7D103F1FA
:105EA000C0075E46774506F18006CCD13848FEF73C
:105EB0008BFC384A029F99F823600FCA0DF1200A23
:105EC0008AE80F005AF82770042E00F28D84DFE86C
:105ED00016F0AD023602C30140016900264899F868
:105EE00021C050F831102C4A2C48049FC8F80010EB
:105EF000BCF1000F08BF02467B68C8F804300221DD
:105F00004FF0770B10460127C8F80C1088F808B03E
:105F1000C8F82C70FEF758FC5246DDF814C05946FC
:105F200006F1230A02F1300B5CF8046F06F500431A
:105F3000C3EB0310470085FB076EBE44FE17C6EB9C
:105F4000EE330233C3EB0A03981E5F1E5E1C04EBA4
:105F5000C01E981C04EBC71704EBC61604EBC31352
:105F600004EBC0100EF80210B9549954B154815486
:105F700001329345D8D19CE71081010030810100A6
:105F8000508101004034FF1F0180008048830100E0
:105F9000E0FF01008C810100D0FF0100CCFF010077
:105FA00070D0FF1FA44BE21900204FF0770B1E6842
:105FB0001EB102F51B5C8CF82FB0596819B102F5BF
:105FC0001B5E8EF830B09E681EB102F51B5A8AF82F
:105FD00031B0D96819B102F51B5C8CF832B01E697A
:105FE0001EB102F51B5E8EF833B0596919B102F586
:105FF0001B5A8AF834B09E691EB102F51B5C8CF8FE
:1060000035B0D96919B102F51B5E8EF836B01E6A3B
:106010001EB102F51B5A8AF837B0596A19B102F558
:106020001B5C8CF838B09E6A1EB102F51B5E8EF8C0
:1060300039B0D96A19B102F51B5A8AF83AB01E6B09
:106040001EB102F51B5C8CF83BB0596B19B102F51F
:106050001B5E8EF83CB09E6B1EB102F51B5A8AF88F
:106060003DB0D96B19B102F51B5C8CF83EB01E6CCB
:106070001EB102F51B5E8EF83FB00130072803F118
:10608000440302F1800292D1029B079AC8F8007083
:1060900003EB8300022602EB800B77270121C8F86F
:1060A0000C6088F80870C8F82C10BBF820E0634E2C
:1060B000BEF5807F0BD0D9F824206149614B62483E
:1060C0005927002AC8BF19467760FFF713FA6322E1
:1060D000D9F828105D48C8F804205A4E5C4FFFF7E5
:1060E00009FAD9F82C2056495748002AC8BF31462A
:1060F0006E23C8F80430FFF7FDF9029AD9F8301082
:1061000052484E4E013207EB810A02921746039A1B
:10611000DAED007A08320392059A02F5717B069A4D
:10612000CDF814B00832BDEEE70A0692049A78233F
:10613000083210EE101A0492C8F80430FFF7DAF9AA
:10614000042F09F1140900F0F18103994E680299B6
:106150004EE6404BE21900204FF0770B196819B159
:1061600002F51B5A8AF82FB05E681EB102F51B5C5F
:106170008CF830B0996819B102F51B5E8EF831B019
:10618000DE681EB102F51B5A8AF832B0196919B1DE
:1061900002F51B5C8CF833B05E691EB102F51B5E24
:1061A0008EF834B0996919B102F51B5A8AF835B0E6
:1061B000DE691EB102F51B5C8CF836B0196A19B1A4
:1061C00002F51B5E8EF837B05E6A1EB102F51B5AEF
:1061D0008AF838B0996A19B102F51B5C8CF839B0AD
:1061E000DE6A1EB102F51B5E8EF83AB0196B19B16A
:1061F00002F51B5A8AF83BB05E6B1EB102F51B5CC0
:106200008CF83CB0996B19B102F51B5E8EF83DB06D
:10621000DE6B1EB102F51B5A8AF83EB0196C19B13B
:1062200002F51B5C8CF83FB00130072803F14403F2
:1062300002F1800292D127E7EC02020070D0FF1F2A
:1062400064000200D4FF0100680002007000020038
:1062500024A00100A4FB0100724BE21900204FF0C2
:10626000770B1E681EB102F51B5E8EF82FB05968C1
:1062700019B102F51B5A8AF830B09E681EB102F5BA
:106280001B5C8CF831B0D96819B102F51B5E8EF831
:1062900032B01E691EB102F51B5A8AF833B0596933
:1062A00019B102F51B5C8CF834B09E691EB102F581
:1062B0001B5E8EF835B0D96919B102F51B5A8AF800
:1062C00036B01E6A1EB102F51B5C8CF837B0596AF5
:1062D00019B102F51B5E8EF838B09E6A1EB102F548
:1062E0001B5A8AF839B0D96A19B102F51B5C8CF8CF
:1062F0003AB01E6B1EB102F51B5E8EF83BB0596BB7
:1063000019B102F51B5A8AF83CB09E6B1EB102F51A
:106310001B5C8CF83DB0D96B19B102F51B5E8EF891
:106320003EB01E6C1EB102F51B5A8AF83FB0013018
:10633000072803F1440302F1800292D1A4E63A4B0C
:10634000E21900204FF0770B196819B102F51B5CB8
:106350008CF82FB05E681EB102F51B5E8EF830B06F
:10636000996819B102F51B5A8AF831B0DE681EB17E
:1063700002F51B5C8CF832B0196919B102F51B5E8D
:106380008EF833B05E691EB102F51B5A8AF834B03C
:10639000996919B102F51B5C8CF835B0DE691EB144
:1063A00002F51B5E8EF836B0196A19B102F51B5A58
:1063B0008AF837B05E6A1EB102F51B5C8CF838B003
:1063C000996A19B102F51B5E8EF839B0DE6A1EB10A
:1063D00002F51B5A8AF83AB0196B19B102F51B5C29
:1063E0008CF83BB05E6B1EB102F51B5E8EF83CB0C4
:1063F000996B19B102F51B5A8AF83DB0DE6B1EB1DC
:1064000002F51B5C8CF83EB0196C19B102F51B5EED
:106410008EF83FB00130072803F1440302F18002F7
:1064200092D131E654070200C80402003C4BE21945
:1064300000204FF0770B1E681EB102F51B5A8AF838
:106440002FB0596819B102F51B5C8CF830B09E680A
:106450001EB102F51B5E8EF831B0D96819B102F594
:106460001B5A8AF832B01E691EB102F51B5C8CF80B
:1064700033B0596919B102F51B5E8EF834B09E69CC
:106480001EB102F51B5A8AF835B0D96919B102F567
:106490001B5C8CF836B01E6A1EB102F51B5E8EF8CE
:1064A00037B0596A19B102F51B5A8AF838B09E6A9A
:1064B0001EB102F51B5C8CF839B0D96A19B102F52E
:1064C0001B5E8EF83AB01E6B1EB102F51B5A8AF89D
:1064D0003BB0596B19B102F51B5C8CF83CB09E6B5C
:1064E0001EB102F51B5E8EF83DB0D96B19B102F5F5
:1064F0001B5A8AF83EB01E6C1EB102F51B5C8CF86C
:106500003FB00130072803F1440302F1800292D129
:10651000BAE5BE2203490448FAF79AFEC9E400BF6F
:10652000840902007CFF01000C000200B74C002728
:10653000FF2500971F235322F7600E2135722E206E
:10654000FAF712FF04F5206AAC46A346234683F807
:10655000ADC683F82DC783F8ADC783F82DC883F87F
:10656000ADC883F82DC983F8ADC983F82DCA83F867
:10657000ADCA83F82DCB03F5A0635345E7D128229C
:10658000FF21A3480DF03CFFA24800F5C079FF228F
:10659000CA4584F8D42680F8D42680F8542780F899
:1065A000D42713D089F8D42689F8542789F8D4271A
:1065B00089F8542889F8D42889F8542989F8D429E5
:1065C00089F8542A09F58069CA45EBD12822FF21B0
:1065D0009148924E0DF014FF079F9148D7F8884FCD
:1065E000D7F8843F56F8242056F8231010250226A9
:1065F0002E24C8F82C60C8F80450C8F80040FEF7F4
:1066000079FF8848884902680892089BD7F88C7FF0
:10661000C3EB0316A1FB06350120C5F34016C8F8ED
:106620002C00002F00F0E680002E15BFFF20002078
:106630000024FF240090312349222921372041F2F0
:106640003655FAF791FE41F2B66241F2367141F2E7
:10665000B64C41F236630BF8054041F2B65941F2AF
:10666000B67A41F6360741F6B6050BF802400BF84C
:106670000140152221466D480BF80C400BF80940EB
:106680000BF803400BF80A400BF807400BF80540E5
:106690000DF0B6FE41F24A4C41F24A5041F2CA6254
:1066A00041F24A7141F24A630BF80C4041F2CA4987
:1066B00041F6CA0C41F2CA5A41F2CA7541F64A077C
:1066C0000BF800400BF802400BF801401522214660
:1066D00057480BF803400BF80C400BF809400BF837
:1066E0000A400BF805400BF807400DF089FE2A23FD
:1066F0003722504888F8084088E80C00FEF764F814
:106700000798D0F8903F002B7ED0002E0BBF0023BF
:10671000FF23FF2400240093492243233B213720F9
:1067200041F63665FAF720FE41F6367742F2360139
:106730000BF8054042F2B61342F2B60C41F6B659D8
:1067400041F6B66641F6B67A42F236150BF80740C6
:106750000BF801401522214641F6CA5736480BF87E
:1067600003400BF809400BF806400BF80A400BF801
:106770000C400BF805400DF043FE41F64A5241F63D
:106780004A6042F24A010BF8074042F2CA1C41F645
:10679000CA6941F64A7541F6CA7A42F2CA0742F21C
:1067A0004A160BF802400BF800400BF80140152286
:1067B000214622480BF80C400BF809400BF8054025
:1067C0000BF80A400BF807400BF806400DF018FED6
:1067D0003A223C231A4888F8084088E80C00FDF764
:1067E000F3FF0DB0BDE8F08FD92216491648FAF72D
:1067F0002FFD49E43846FF241CE78822134914483A
:10680000FAF726FDFFF755BBFF2484E74034FF1F4E
:10681000ED3AFF1FC034FF1F6D44FF1F9022FF1F82
:1068200074000200ACE001201F85EB517648FF1F89
:10683000764DFF1F7C0002007651FF1F7656FF1F2A
:1068400080000200A406020038000200F8060200E0
:10685000E4FF01003C4F0AEBC613E61807F5D25ED1
:10686000A7F1C003B446B3465968043309B18CF8A4
:10687000002058680CF1010A08B18CF801209E68CC
:106880000EB18AF80120D96809B18AF80220186986
:1068900008B18AF803205E690EB18AF8042099696C
:1068A00009B18AF80520D8691C3308B18AF8062096
:1068B000BB420AF1070CD7D103F1C0075E46BE45C3
:1068C00006F18006CCD12148FDF77EFFFFF7F1BA33
:1068D0000AEBC6131E4FE118A7F1C0038A46586899
:1068E000043308B18AF800205E680AF1010B0EB18A
:1068F0008AF80120986808B18BF80120DE680EB193
:106900008BF80220186908B18BF803205E690EB17C
:106910008BF80420986908B18BF80520DE691C33D8
:106920000EB18BF80620BB420BF1070AD7D103F159
:10693000C007084B9F4201F18001CDD10648FDF709
:1069400043FFFFF7B6BA00BF20E20100D8FF010005
:106950001C0C02005C260200DCFF01002DE9F04F58
:10696000C04FC14C0D460FCF91B008AE0FC697E88F
:106970000F00802786E80F000023E36023614FF0BB
:1069800001083A46FF21B948A36223756375A361E4
:10699000E361237295F89C6FC4F82C80C4F80080E2
:1069A000276267620DF02CFD3A46FF21B0480DF0DA
:1069B00027FD3A46FF21AF480DF022FD3A46FF2160
:1069C000AD480DF01DFD3A46FF21AC480DF018FD15
:1069D0003A46FF21AA480DF013FD3A46FF21A94887
:1069E0000DF00EFD3A46FF21A7480DF009FD3A468D
:1069F000FF21A6480DF004FDA548A649C4F804806F
:106A0000FEF778FDD5ED017AF5EEC07AFF20F1EEC4
:106A100010FA207200F1C5816946EE46BDEEE77AB4
:106A20000EF1FF3CB8EEC70A17EE103A002077EEE1
:106A3000C00ADFF8648200E0384688FB0329DA17D1
:106A4000C2EBA90A0AEB8A0BA3EB4B07303753467C
:106A50000CF8017F471C002BEED15FEA670800F0BD
:106A6000A6800EEB0702734612F801AD9EF8009067
:106A700003F801AB08F1FF3BF044984582F8009021
:106A80000BF0070C00F09380BCF1000F4BD0BCF171
:106A9000010F3ED0BCF1020F33D0BCF1030F28D060
:106AA000BCF1040F1DD0BCF1050F12D0BCF1060FD4
:106AB00007D093F800A012F8019D03F8019B82F81B
:106AC00000A093F800B012F801CD03F801CB82F8D2
:106AD00000B093F800A012F8019D03F8019B82F822
:106AE00000A093F800B012F801CD03F801CB82F8B2
:106AF00000B093F800A012F8019D03F8019B82F802
:106B000000A093F800B012F801CD03F801CB82F891
:106B100000B012F801AD93F8009003F801AB98456E
:106B200082F8009043D09C4612F801BC93F800A074
:106B30000CF801BB02F801AC93F8019012F802BC0A
:106B400083F801B002F8029C9CF8019012F803ACA3
:106B50008CF801A002F8039C93F803C012F804BC5F
:106B600083F803B002F804CC93F804A012F8059C53
:106B700083F8049002F805AC93F805C012F806BC3F
:106B800083F805B002F806CC93F806A012F8079C2B
:106B900083F8069002F807AC12F808BD93F807C016
:106BA00083F807B00833984582F800C0BBD1B2EE35
:106BB000041A60EE811A384ADFF8AC80BDEEE12A93
:106BC000704412EE103A82FB032ADA17C2EBAA09CC
:106BD00009EB890BA3EB4B034FF02E0A0EF807A02D
:106BE00030334FF0000C0B27837080F803C06760D0
:106BF000002E67D1294A2A48FEF77CFCE968142256
:106C0000C8F80420002900F09A8026492648274A1F
:106C1000FEF770FCEF691D206060002F00F0BF8060
:106C20002349022E67D11D4A22480F4FFEF762FC0E
:106C3000A8686F220528626040F298801B4A1E49AE
:106C40001E48FEF757FC2C69184A10AD05EB840668
:106C50007820786056F8201C1948FEF74BFC11B0DC
:106C6000BDE8F08F9C81010070D0FF1F4034FF1FF2
:106C7000C034FF1F4035FF1FC035FF1F4036FF1FC8
:106C8000C036FF1F4037FF1FC037FF1F4038FF1FB0
:106C9000B0000200A800020067666666A400020059
:106CA000BC0002008C000200D00002006400020060
:106CB00094000200E40002009C000200F8000200C0
:106CC0000C0102003C4A3D48FEF714FCE8683C4BCE
:106CD0003C491422002818BF1946012EC8F8042088
:106CE00094D1394A3948FEF705FCE9691D276760E8
:106CF000002930D1364937482F4AFEF7FBFBA868F8
:106D00006F230528636031D9032E334933D02A4AD3
:106D10003248FEF7EFFB2F69274A2B4D0DF1400853
:106D200008EB87097820606059F8201C2C48042E55
:106D300008BF2A46FEF7DEFB11B0BDE8F08F2149FF
:106D40001D4A2248FEF7D6FBEB691D21C8F8041046
:106D50002BB32449CFE71F48174A2249FEF7CAFB45
:106D6000A8686F230528C8F8043023D81E49032ECD
:106D700051F82010CBD1144A1848FEF7BBFB2E69FE
:106D80000D4A17480DF1400B0BEB860A78235AF891
:106D9000201C6360FEF7AEFB11B0BDE8F08F0C491C
:106DA0003FE72D218DF80010F1EE677A0DEB080E0C
:106DB000694633E60849AAE764000200BC00020005
:106DC0008C00020084000200A4000200D000020037
:106DD00098000200E40002009C000200F80002009B
:106DE0000C01020094000200D40202002DE9F043DD
:106DF000C3B001AC804625460DF582792B462A1B8F
:106E000003F8012BEF1C2E1D681DA91DEA1D03F1BF
:106E1000010EC4EB0E0EC4EB030C3F1B361B001B14
:106E2000091B121B85F801C083F801E0083505F83D
:106E3000057C05F8046C05F8030C05F8021C05F840
:106E4000012C4D45DAD10DF105077B1BFF20DE43F8
:106E500084F800010DF030FB06F003092E462D1BCF
:106E600016F8013D90FBF5F101FB150CBE4214F83C
:106E70000C20327004F80C3071D0B9F1000F2FD013
:106E8000B9F1010F1CD0B9F1020F0BD00DF014FBBA
:106E9000351B90FBF5F101FB150016F8013D225C56
:106EA000327023540DF008FB351B90FBF5F101FB0C
:106EB000150916F8010D14F80930337004F80900AB
:106EC0000DF0FAFA351B16F8012D90FBF5FC0CFBC2
:106ED0001509BE4214F80910317004F809203ED09B
:106EE0000DF0EAFA331B90FBF3F505FB130016F8DF
:106EF000011C14F800C006F801CC21540DF0DCFA96
:106F0000721E131B90FBF3F505FB130916F8020C18
:106F100014F8091006F8021C04F809000DF0CCFA68
:106F2000B21E151B90FBF5FC0CFB150916F8033C73
:106F300014F8090006F8030C04F809300DF0BCFA47
:106F4000F11E0D1B16F8043D90FBF5F202FB150C2B
:106F5000BE4214F80C00307004F80C30C0D1214649
:106F60004FF48072404609F0E9F8214608F5807038
:106F70004FF4807209F0E2F843B0BDE8F08300BF3F
:106F80002DE9F04F2DED088B544DDFED558A2B6820
:106F9000544E9FED558A8FB004460C930C98C4F85C
:106FA0000402C4ED808A8B460DF07CFA2046FFF780
:106FB0001DFF4FF086482A68C4F83C8204F58E6CA9
:106FC0000A924A484A49C4F80C02012204F2544782
:106FD00004F58B6A04F2744800234FF00009C4F8EA
:106FE000146284F84922DDF828E0424AC4F8081205
:106FF0004FF07E5604F50270C4F8443284F84832EB
:1070000084F84A3284F84B3284F84C32C4F82C228B
:10701000C4F83422C4F85002C4F81892C4F8249278
:10702000C4F84092C4F81C62C4F83062C4F83862F4
:107030002046C7F80090CAF80090C4F868E4C4F885
:107040005C34C4F8603484F8643484F8653484F8BB
:107050006C34CCF80090C8F8009008F0FFFD204692
:1070600008F0DCFD204608F00FFE642009F02CF843
:1070700007EE900A29680B91B8EE670A0B9860EE4C
:10708000080AA0EEA88A10B92D680D950D98C4F8CD
:1070900004020DF007FA2046FFF7A8FEB5EEC08AFD
:1070A000F1EE10FA04F51570D2BFD4ED802A84ED0C
:1070B000808AF0EE482A0390DFED0F9A9FED0FAA29
:1070C00082460026B1EE089AFAEE0EBAF2EE048A73
:1070D000B5EE00BAF7EE00AA1EE000BFACE001205A
:1070E0000AD7A33C00005C410AD7233CA0D2FF1F73
:1070F00070DE0020000080BF00000000FFFF7F7FE7
:107100006666E63F6666663F00FEFF4600F07F4526
:1071100000008046D4ED802A01EE106AF8EEC11A14
:10712000013621EEA22A12EE100A0CF025FA894649
:10713000804649EC108B0BF0FBFF53EC102B10EE4C
:10714000100A1946CDE900230CF01AFDDDE90023F1
:10715000C5B2494640460CF0AFF80CF059FD14F8A2
:107160000590254409F00303697803EE103A5FEABD
:10717000097201F0030202EE900AF8EEC33A08EE3B
:10718000102AB0EE6B7AF0EE6A5AE3EE8B5AA2EE5A
:10719000897AB8EEC80AF0EE6A0AE0EE0B0AB0EEA1
:1071A000686AF0EE654A72EEEA7A62EEA26AA2EED0
:1071B000876A4CBF65EEE24A62EEA44A0B074CBFF9
:1071C00060EEE77A67EEA07A26EEA24A77EEE41A3E
:1071D00024EE065AE5EE214AF4EECA4AF1EE10FA20
:1071E000F4EE694AD8BFB0EE64AAF1EE10FAC8BF57
:1071F000F0EE649A802EEAEC014A8BD103985FEDA1
:1072000040BA90ED009A5FED418A39EE4ABA79EEC4
:10721000CA9A6BEE2BAA06468AEEA97A3D1A2B1F54
:10722000C3F3810177EE686AE6EC016AB7425ED08B
:1072300049B3012919D002290BD096ED006A36EE28
:107240004A3A63EE2B3A83EEA94A74EE685AE6ECAA
:10725000015AD6ED004A34EECA5A25EE2B8A88EE42
:10726000290A70EE687AE6EC017AD6ED000A30EE73
:10727000CA1A61EE2B1A81EEA92A72EE682AE6EC90
:10728000012AB74233D096ED009A39EE4ABAB64693
:107290006BEE2BAA10368AEEA97A77EE686AEEECCE
:1072A000016A16ED036A36EE4A3A63EE2B3A83EE34
:1072B000A94A74EE685A46ED035ADEED014A34EEEF
:1072C000CA5A25EE2B8A88EE290A70EE687ACEED2E
:1072D000017A56ED010A30EECA1A61EE2B1A81EEE0
:1072E000A92A72EE682A46ED012AB742CBD1039A49
:1072F0005FED7BBA1346B3EC01AA6AEE2B8AB81A8B
:10730000FDEEE89A0022CDED009A061FBDF900506F
:10731000C4F85C249F42C4F86024C6F38201DA46B4
:10732000CBF8005000F0C980002962D0012952D06A
:10733000022944D0032936D0042928D005291AD09F
:1073400006290CD0B3EC019A29EE2BBADA46FDEEF1
:10735000CBAACDED00AABDF900004AF8040FB3ECAA
:10736000017A67EE2B6ABDEEE66A8DED006ABDF923
:1073700000604AF8046FB3EC013A63EE2B3ABDEEBD
:10738000E34A8DED004ABDF900504AF8045FF3EC82
:10739000015A65EEAB4ABDEEE45A8DED005ABDF9D7
:1073A00000204AF8042FB3EC018A28EE2B0AFDEEE8
:1073B000C07ACDED007ABDF900104AF8041FF3EC55
:1073C000010A20EEAB1AFDEEC11ACDED001ABDF98F
:1073D00000004AF8040FB3EC012A62EE2B2A9F4208
:1073E000BDEEE2AA8DED00AABDF900604AF8046F77
:1073F00063D09C46FCEC018AD3ED019A93ED03BA6D
:10740000D3ED04AA93ED056AD3ED066A93ED077AEE
:107410009CED019A28EEAB3A29EE2B4A69EEAB4A75
:107420002BEE2B5A6AEEAB5A26EE2B8A26EEAB0ACF
:1074300067EE2B7AFDEEC33AFDEEC40ABDEEE41A08
:10744000FDEEC51ABDEEE52AFDEEC82ABDEEC0AAC6
:10745000FDEEE78ACDED003ACDED040A8DED031A7D
:10746000CDED051A8DED062ACDED072A8DED08AA82
:10747000CDED098A2033BDF91090BDF90080BDF92A
:107480000CC0BDF914E0BDF91820BDF91C50BDF9C0
:107490002000BDF92410CAF80C909F42CAF804805D
:1074A000CAF808C0CAF810E0CAF81420CAF8185080
:1074B000CAF81C004AF8201F9BD104F58A67D7ED53
:1074C00000BA5FEDEE9A5FEDEEFA9FED1AFADFED8E
:1074D0001AEA9FED1AEADFED1ADA9FED1ADAB7EE33
:1074E000009A3BEE89BAF6EE00AA2BEE296A2046F6
:1074F00066EE2A6A0122BCEEE67A00268DED007A5D
:10750000BDF80040CBF8806303EE104AB8EE434A62
:107510000023CBF884338BEDEF4A8BF8C0638BF8F4
:1075200098238BF899238BF8B9230FB0BDEC088B07
:10753000BDE8F08F1F91EE3DB704CD4333333346A2
:10754000000034420000803C2DE9F04F4B8C2DEDC3
:10755000028B00EE103A0D468046ADF20C4D00F560
:107560009870B8EE400A1446F9F7A8FEA88C98ED7A
:10757000587A98ED595AD8ED577AD8ED566A88ED71
:107580006C0A06EE100AF8EE460A77EEE65A30EE7E
:10759000C71AA5EE017AB4EEE57AF1EE10FA88ED9D
:1075A000587A40F1958677EE267AC8ED577A98EDAD
:1075B000542AD8ED5A2A98ED553A76EE823AF0EEF2
:1075C000424A37EEE34AE4EE224AF4EEC34AF1EED1
:1075D00010FAB0EE648A40F11687B4EE642AF1EE38
:1075E00010FA58BFB0EE428A04F57D619FEDF32A90
:1075F0000A68DFEDF32A9FEDF33ADFEDF33A9FEDF2
:10760000F34AC8F8B42188ED6B8A05F10E0E4246A4
:1076100008F5DC7705F11606C14643460020F6EE74
:10762000004AB7EE005A3EF8021F92ED300AD2ED42
:10763000326AD2ED315A92ED2F7A92ED2E6A08EE2F
:10764000901AF8EE687AF0EE400A77EEC01A37EE3C
:10765000461AE6EEA10A70EEC08A38EEE50AE0EEC0
:10766000245AF0EE656A70EEA55AC2ED316AF4EE66
:10767000C15AF1EE10FAC2ED305A40F1198635EEDA
:10768000867A82ED2F7AD2ED2C6AD2ED330A92ED12
:107690002D8AF0EE001AB0EE661AA6EE211AF0EE70
:1076A000668A37EE417AE7EE208AF4EEC88AF1EE78
:1076B00010FA40F1F985F4EE686AF1EE10FA48BF6D
:1076C000F0EE686A36F8021FE7EC016A05EE901AE0
:1076D000D3ED087AD3ED090A93ED0A8AB8EE651A5C
:1076E00071EE671A31EE606AE1EE827AE6EE220A06
:1076F000C3ED087A37EEE07AC3ED090AF0EEC78AE7
:10770000F4EE488AF1EE10FAD8BFF0EE488A68EE3F
:10771000837AF4EEC57AF1EE10FA40F3EE85DFEDF0
:10772000AC5ADFEDAC0AB6EE000AF7EE007A93ED44
:107730000F8AD3ED0D6AC3ED0A7A75EE885A31EEE1
:10774000661A75EEA01AF0EE667AC5EEA10A93ED00
:107750000B6A93ED0C7AC3ED0E0AE0EE817A76EEB9
:10776000478A35EE608AF4EEE87A68EE256AF1EE33
:1077700010FAC3ED0F6AC3ED0D7A07D577EE875A7D
:1077800035EEC61A36EE016A83ED0B6A77EE061AFD
:10779000F4EEE17AF1EE10FA07DD37EEC77A77EE14
:1077A000468A36EE286A83ED0B6A0130042883EDA1
:1077B000106A83ED0A0A02F12002A9EC016A03F1C2
:1077C00024037FF430AF04F57C6A9AED002A2A8CFA
:1077D000DFED872A03EE102A72EE023ABFEE004A6E
:1077E000A3EEA24A04F6BC7BF8EE434A9BED005A96
:1077F00024EEA20AF7EE000A24EE008AA5EE228A01
:10780000B4EEE08AF1EE10FA00F18D85DFED727AC8
:1078100094ED0B1AD8ED005ADFED741ADFED748A7F
:10782000266B6E4F9FED6E2A9FED6E7AC8ED797ACA
:10783000B8EEC16A65EEA82A26EE213A07EB860C5F
:1078400063EE223A9CED004AA3EE824A04F22449F8
:1078500004F5FD6304F6AC30B4EEC74A04F5776175
:10786000F1EE10FAC9ED007AC3ED007AC0ED007AAE
:10787000C1ED007A40F153859FED5B5AB4EEC54AE5
:10788000F1EE10FAC8BFB0EE445AD4ED106A84EDA0
:10789000FE5A98ED010ADFED560A9FED548A626C9C
:1078A0009FED4F1ADFED4F7AF8EEE61A60EE205AA0
:1078B00061EE888A07EB820A28EEA52A9AED007A03
:1078C000A2EE017AB4EEE77AF1EE10FA08D5DFED18
:1078D000467AB4EEE77AF1EE10FAC8BFF0EE477AD6
:1078E000D4ED152ADFED423A9FED404AA66DDFED5B
:1078F0003C4ADFED3C1A04F2BC7BCBED007A98EDFC
:10790000023AB8EEE25A23EE230A65EE040A07EBC8
:10791000860C20EE808A9CED001AA8EE241AB4EEA4
:10792000E11AF1EE10FA08D5DFED2F1AB4EEE11AE4
:10793000F1EE10FAC8BFF0EE411AD4ED1A8A9FEDAD
:107940002C7ADFED2A2AE36EDFED255ADFED257A6A
:1079500004F53869C9ED001A98ED032AB8EEE83A43
:1079600022EE076A63EE223A07EB830723EE864A8C
:10797000D7ED004AE4EE254AF4EEE74AF1EE10FABC
:10798000B0EE645A40F1C7849FED170AF4EEC04A86
:10799000F1EE10FAD8BFB0EE405A94ED0A8A208C6E
:1079A000DFED120AB8EEC81A04F64471B0F5807F14
:1079B00061EE207A81ED005A42D021E06666663F92
:1079C0009A99993E0AD7A33B9A99D93F0AD7233C63
:1079D000AE47813FD0CC4C3E295C0F3E24A0010035
:1079E00000245B4500005C4500005C41B57E253C01
:1079F0000108803917B7D13800000000ABAAAA40AF
:107A00002A8A94ED092A94F823605FED071A06EE9E
:107A1000902AF8EEC22AF8EE668A042E28EEA17AA1
:107A200022EEA03A00F00985E7EE037AF7EE003A7D
:107A3000F4EEE37AF1EE10FA00F1F484F0EE637AFA
:107A400094ED0F5AB4F834A05FED184AC4EDFF7AF4
:107A5000B8EEC50ABAF5807F60EE245A20D0B5F89A
:107A600012B0D4ED0E6A94F837301FED1F8A00EE85
:107A700090BAF8EEE61AB8EE601A042B61EE088AA6
:107A800021EEA42A00F06584E2EE285AB7EE003A0F
:107A9000F4EEC35AF1EE10FA00F15084F0EE435ABE
:107AA000D4ED147AB4F848705FED303AB8EEE74A96
:107AB00004F5F86CB7F5807FCCED005A64EE232A0C
:107AC0001FD0A88AD4ED130A94F84B101FED385A32
:107AD00004EE900AB8EEE08AB8EE640A042920EEBB
:107AE000051A68EE236A00F06984E6EE812AB7EE93
:107AF000002AF4EEC22AF1EE10FA00F15484F0EEFE
:107B0000422AD4ED195AB4F85C201FED483AB8EE79
:107B1000E56A04F68439B2F5807FC9ED002A66EE85
:107B2000037A1FD0ED8A94ED185A94F85F601FED28
:107B3000504A03EE905AB8EEC50AF8EE634A042E96
:107B400064EE840A20EE038A00F05084E8EE207A86
:107B5000F7EE001AF4EEE17AF1EE10FA00F13B8450
:107B6000F0EE617A04F6487ACAED007A5FED602A99
:107B700098ED6B2A04F6C47322EE227A93ED003A54
:107B8000A3EE227AB7EE006AB4EEC67AF1EE10FAEE
:107B900000F13D8404F57E6BDBED003A1FED6B4A8E
:107BA000E76976EE634AB0EEE45AB4EEC45AF1EEF9
:107BB00010FACCBF01230023002F40F02F8394F84C
:107BC0002150012D00F0EC8394F823105FED766ACC
:107BD000042918BFF0EE466A04F20C4C94F8357094
:107BE000CCED006A94F80904012F40EA030084F800
:107BF000090400F07F8394F837205FED811A042A8E
:107C000018BFF0EE461A04F5FA6994F84960C9ED18
:107C1000001A94F8CD57012E45EA030584F8CD5794
:107C200000F0658394F84B105FED8D7A042918BF3E
:107C3000F0EE467A04F6943A94F85D70CAED007A54
:107C400094F8910B012F40EA030084F8910B00F0A7
:107C50003C8394F85F205FED988A042A18BFF0EE09
:107C6000468A04F6587CCCED008A94F8556F33436D
:107C700084F8553F00238BED006A1FEDA08ACDF8F4
:107C8000048004F51B7B5E46984696F89C51002DB7
:107C900000F0F680C8EB0811D6F8840108EB011259
:107CA00001AB0DF58161B34600F07F06471C164419
:107CB00007F07F051C36C71C07F07F09071D00F180
:107CC000020E54F826605E6007F07F0C471D41F8F5
:107CD000046C0EF07F0AC61D07F07F0E871D07F0AB
:107CE0007F0706F07F0615449244914494449644DD
:107CF000174416441C350AF11C0A09F11C090CF141
:107D00001C0C0EF11C0E1C371C3654F8255054F870
:107D10002AA054F8299054F82CC054F82EE054F8B6
:107D2000277054F826609D6041F8085CC3F80CA0E9
:107D300041F80CACC3F8109041F8109CC3F814C083
:107D400041F814CCC3F818E041F818ECDF6141F8B1
:107D50001C7C43F8206F81ADAB4200F1080041F874
:107D6000206DA1D13F495E4600205F4601254FF0BE
:107D700000090BF02DFFB0F5807F28BF4FF4807015
:107D8000814580F0B28200F1804202AB511E03EBCC
:107D9000890B0DF1080A0AEB810CABF1040101F12A
:107DA000040ECBEB0C02E645C2F382024B683ED0D8
:107DB0001AB3012A1CD0022A17D0032A12D0042A8F
:107DC0000DD0052A08D0062A18BF5EF8042F5EF8E9
:107DD000041F18BF9B180B445EF8042F13445EF871
:107DE000041F0B445EF8042F13445EF8041F0B4479
:107DF0005EF8042FE645134419D0DEF80420DEF8BF
:107E000008101344DEF80C201944DEF81030114439
:107E1000DEF814201944DEF8183011440B44DEF863
:107E20001C205EF8201F1344E6450B44E5D10135C4
:107E3000312DC9EB000293FBF2F147F8041F1BD070
:107E400002EE105AF8EEC22A814622EE887A17EE28
:107E5000100A0BF091FB41EC100B0BF069F951EC9F
:107E6000100B86E700001440000000C700FEFF462C
:107E700000010038000000344FF0000086F89C013B
:107E800008F10108B8F1040F06F571767FF4FDAE34
:107E900004F59155DDF804801FED0D5A5FED0D5A84
:107EA0001FED0C6A1FED0E0A1C3504F54B724FF0E6
:107EB000000B92F8DD70002F00F06581DFF8D8E547
:107EC000A2F1C00117464FF0004C6FF00043DEED09
:107ED000013A92ED383A4868B8EEE34A64EE034A54
:107EE000FDEEE40A10EE90AA50447860DEED026ADE
:107EF00092ED381A8E68F8EEE61A834261EE817AC6
:107F0000A8BF0346FDEEE78A8445B8BF8446E14634
:107F100018EE90CAB444C7F808C09EED032A92ED4B
:107F2000388AF8EEC22A634522EE887AA8BF6346F3
:107F3000BDEEC73AE145B8BFE1469A4613EE10CA16
:107F4000CB680CEB0306FE609EED044AD2ED383A96
:107F50000B69F8EEC44A504664EEA30AB245BDEE82
:107F6000E01AA8BF304611EE10AAB145B8BFB1461D
:107F70000AEB03063E61DEED051AD2ED386A4B6965
:107F8000F8EEE17AB04267EEA68AA8BF3046BDEEB1
:107F9000E88ACC46B14518EE109A9944C7F8149077
:107FA000B8BFB4465EF8186FD2ED382A02EE106AF8
:107FB000B8EEC27A4B4627EE223A9842FDEEC33A1B
:107FC000A8BF184651F8189F824613EE900A9C45A8
:107FD0004844B8BF9C4682455346A8BF03468445E3
:107FE000B8BF8446914247F8180F7FF470AF04EE93
:107FF000103A04EE90CAF8EEC40AB8EEE41AD2EDD4
:10800000381A75EE606A75EEC17AF0EE608AA1EEFC
:10801000A71AC3EB0C0E02F1C007E1EEA68A1146C7
:10802000FDEEC12ABDEEE82A12EE900A12EE106AA9
:1080300008EE10EA801BB8EEC87A03EE100A77EE5D
:10804000064AF8EEC33AB8EEC21A83EEA44A4E6866
:10805000F01A01F1040C06EE900AF8EEE61AF0EEC2
:10806000417AE4EE217ABDEEE78A18EE106A06F353
:108070000F004860DCF80460F01A02EE100AF8EE17
:10808000C22AB0EE417AA4EE227AFDEEC73A13EE90
:10809000906A06F30F00CCF80400CE68F01A04EEE4
:1080A000900AF8EEE46AF0EE411AE4EE261AFDEECC
:1080B000E18A18EE906A06F30F000E69C860F01AA4
:1080C00008EE100AB8EEC82AF0EE412AE4EE022AC1
:1080D000BDEEE23A13EE106A06F30F004E69086136
:1080E000F01A03EE900AF8EEE36AF0EE414AE4EE8D
:1080F000264AFDEEE47A17EE906A06F30F008E69C9
:108100004861F01A08EE900AB8EEE88AB0EE412A0B
:10811000A4EE082ABDEEC27A17EE10EA0EF30F069F
:10812000C8698E61C61A03EE106AF8EEC33AF0EE23
:10813000416AE4EE236AFDEEE61A11EE909A09F325
:108140000F00C86151F8206FF01A07EE900AF8EEA0
:10815000E78AB0EE418AA4EE288AFDEEC82A12EE24
:10816000906A06F30F008F4208607FF470AF60EEF4
:10817000800A21EE001AC2ED3A0A82ED3C1A82ED25
:10818000394A82F8DDB002F5717295427FF491AE02
:1081900094F8235098F8DC31AB4207D0042B00F060
:1081A0006181042D00F0568188F8DC5194F8370085
:1081B00098F8DD21824207D0042A00F0608104286B
:1081C00000F0558188F8DD0194F84B1098F8DE61D5
:1081D0008E4207D0042E00F0D680042900F0CA8019
:1081E00088F8DE1194F85F5098F8DF2195420AD0A4
:1081F000042A04BF98F8E32184F85D20042D00F0E0
:10820000C78088F8DF51D8F8B01104F6DC7421601B
:108210000DF20C4DBDEC028BBDE8F08F94F82300FD
:108220009FED990A94F8372094F84B6094F85F50CA
:1082300004280CBFF0EE400AF0EE460A04F20C4CA3
:10824000CCED000A94F80914042A0CBFB0EE408A61
:10825000B0EE468A194304F5FA6984F8091489EDE9
:10826000008A94F8CD77042E0CBFB0EE401AB0EE21
:10827000461A1F4304F6943A84F8CD778AED001A23
:1082800094F8910B042D40EA030018BFB0EE460AA3
:1082900004F6587284F8910B82ED000A94F8556F39
:1082A000334384F8553FE5E4F0EE486AFFF70ABA35
:1082B00077EE067AF4EEE75AF1EE10FAC4BF35EE27
:1082C000C67A82ED2F7AFFF7DEB9DFED6F8AC8E458
:1082D00077EEA61AB4EEE17AF1EE10FAC4BF77EEAB
:1082E000667AC8ED577AFFF762B900239FE5DFEDA4
:1082F000667A9FE4DFED641A85E4B7EE080AF0EED3
:10830000630AF0EE445AE7EEC00AE7EEA75A27EEFA
:10831000A40AFFF70CBAB0EE675AFFF73EBBB0EE07
:10832000475AFFF7B2BAB5EEC08AF1EE10FA1DDD7A
:10833000DFED566A68EE267AFFF76ABAF5EEC05AA4
:108340009FED516AF1EE10FAD8BFF0EE465AFFF7F2
:10835000A7BBDFED4F2A9FED4C7AF4EE628AF1EE77
:1083600010FA48BFF0EE478AFFF78EBBDFED467A82
:10837000FFF74EBA94F849B088F8E2B14FF0000A1E
:1083800084F849A02CE798F8E20184F8490024E732
:1083900094F85D3088F8E331002784F85D7030E7A9
:1083A000DFED396A18E4F5EEC02A9FED377AF1EE79
:1083B00010FAD8BFF0EE472AFFF7A3BBDFED341A5F
:1083C000DFED318AB4EE611AF1EE10FA48BFB0EE7B
:1083D000681AFFF78ABBF5EEC07ADFED2B8AF1EE63
:1083E00010FAD8BFF0EE687AFFF7BCBB9FED281AF1
:1083F000DFED256AF4EE410AF1EE10FA48BFF0EE27
:10840000660AFFF7A3BBB0EE438AFFF7EDB89FED16
:10841000216AB4EEC67AF1EE10FAC8BFB0EE476A30
:10842000FFF7B8BBF5EEC07A9FED174AF1EE10FAF0
:10843000D8BFF0EE447AFFF703BBDFED155A9FED8E
:10844000126AB4EE657AF1EE10FA48BFB0EE467AE1
:10845000FFF7EABA94F8211088F8E011002684F8B2
:108460002160A1E698F8E07184F8217099E694F80B
:10847000353088F8E131002784F83570A2E698F8A5
:10848000E15184F835509AE600000000295C0F3E67
:108490000AD7233C000000349C22FF1F0B8D00EE06
:1084A000103A70B5B8EE400A0446006E0E46154606
:1084B000F8F704FFD4ED1C7A84ED1E0A70EE676AAB
:1084C000F5EEC06AF1EE10FA00F1258140F33D812E
:1084D00094ED1A7A94ED1B5ADFEDB04A94ED196AC7
:1084E00077EE670A77EE455AF4EEE40AF1EE10FAF9
:1084F00025EEA61AD8BFF0EE640AC1EE201A31EEBE
:10850000852AB4EEC72AF1EE10FA08D5B4EEC62AD1
:10851000F1EE10FAD4BFB0EE467AB0EE427A728D28
:1085200084ED1C0A02EE902A05F6BC7084ED1B7ADD
:10853000B8EE620A80ED007AE06FF8F7BFFE94EDC6
:10854000233A84ED250A70EE433AF5EEC03AF1EE97
:1085500010FA00F1D38040F3FF8094ED211A94EDDE
:10856000224ADFED8E6A94ED205A71EE437A71EE65
:10857000444AF4EEE67AF1EE10FA24EEA36AD8BF8C
:10858000F0EE667AC6EE270A70EE845AB4EEE51A6B
:10859000F1EE10FA08DDB4EEE55AF1EE10FA54BF30
:1085A000B0EE451AB0EE651A95F8D41FF68C84ED3E
:1085B000230A05F57C6C84ED221A00EE106A8CED1E
:1085C000001A002952D0D4F8B400B8EE400AF8F7E7
:1085D00075FED4ED311A84ED330A30EE612AB5EE22
:1085E000C02AF1EE10FA00F1A38040F3BC8094EDB4
:1085F0002F7AD4ED302A9FED693AD4ED2E3A37EE3A
:10860000614A77EE626AB4EEC34AF1EE10FA26EEE2
:10861000825AD8BFB0EE434AC5EE047A77EEA24A3A
:10862000B4EEE47AF1EE10FA08DDF4EEE43AF1EE9D
:1086300010FA54BFB0EE637AB0EE647A05F6D87ED5
:1086400084ED307A84ED310A05F57D638EED007A94
:10865000D4F8CC201A6005F6C87EA66FCEF800606C
:1086600005F6CC75D4F894402C6070BDD4F8980011
:10867000B8EE400AF8F722FED4ED2A0A84ED2C0A5F
:1086800030EE601AB5EEC01AF1EE10FA72D47EDD4B
:10869000D4ED286AD4ED291A9FED402A94ED276A7B
:1086A00076EEE02A76EEE15AF4EEC22AF1EE10FA06
:1086B00025EE813AD8BFF0EE422AC3EE223A33EEDD
:1086C000A14AF4EEC46AF1EE10FA08DDB4EEC46A11
:1086D000F1EE10FA54BFF0EE466AF0EE446A05F689
:1086E000C470C4ED296A84ED2A0A05F57D6CC0EDDD
:1086F000006AD4F8B010CCF80010ACE794ED205A22
:1087000094ED224ADFED256A94ED211A73EE457A45
:1087100074EE454A2DE794ED196A94ED1B5ADFED8E
:108720001F4A94ED1A7A77EEC60A75EE465ADBE6D2
:10873000D4ED2E3AD4ED302A9FED183A94ED2F7AED
:1087400031EEE34A72EEE36A5DE794ED196A94ED67
:108750001A7A94ED1B2AD4E694ED205A94ED211A4E
:10876000D4ED225A12E7D4ED2E3A94ED2F7AD4EDBF
:10877000304A55E794ED276AD4ED291A9FED072A70
:10878000D4ED286A70EEC62A71EEC65A8CE794EDD5
:10879000276AD4ED286A94ED294A92E7BD378635D9
:1087A0002DE9F041437D012B8CB062D0046EC26D87
:1087B000944208D300239C4601F1FF3898450CD021
:1087C0000CB0BDE8F081651C0444056694F81CC03B
:1087D00001F1FF3863469845F2D1457D8DF808C018
:1087E000012D00F0A781076EC36D9F42C0F0DF80AE
:1087F00000228DF809209F4280F05B827E1C074496
:1088000006663A7F37468DF80A209F4280F04A82FA
:108810007E1C074406663B7F8DF80B3004290DF162
:10882000080E20D00EEB08010DF10B0200250224EA
:108830008027012609E008F101038044036698F8C7
:108840001C3002F8013F91420DD0437D012B00F016
:10885000B480D0F86080C36D9845ECD3002302F853
:10886000013F9142F1D14168704688470CB0BDE8A4
:10887000F08100268DF803609DF80330036942F211
:108880001074DF783D0625D493F803805FEA086210
:1088900020D493F803C05FEA0C651BD4DA78120683
:1088A00018D4DD782F0615D4DE78360612D4DF789A
:1088B0003D060FD493F803805FEA08620AD4083CAF
:1088C000DFD19C7000BF036980229A7000BF012431
:1088D00004756FE79C7804F0E7029A7003691D79CC
:1088E000EEB28DF803609F7847F008049C7003692E
:1088F0000222DA70036942F21074DD78AF071BD4EC
:10890000DE78B60718D4DF78BF0715D493F803C014
:108910005FEA8C7610D493F803805FEA88750BD4F5
:10892000DA78920708D4DD78AF0705D4DE78B60789
:1089300002D4083CE1D1C4E79C7804F0C7079F70DB
:10894000026942F21073D578AD0640F1AD81D67858
:10895000B40640F1A98192F803C05FEA8C6540F14A
:10896000A38192F803805FEA886440F19D81D47806
:10897000A70640F19981D778BE0640F19581D57858
:10898000AD0640F19181D678B40640F18D81083B67
:10899000D9D1937000BF02698024947000BF012573
:1089A0000669057502273579F7709C4604E77E1C39
:1089B000074406663A7F37461BE78DF807509DF857
:1089C0000730036942F2107893F803C01CF0800F5F
:1089D0002ED193F803C01CF0800F29D193F803C067
:1089E0001CF0800F24D193F803C01CF0800F1FD11E
:1089F00093F803C01CF0800F1AD193F803C01CF049
:108A0000800F15D193F803C01CF0800F10D193F89C
:108A100003C01CF0800F0BD1B8F10808D4D183F843
:108A2000028000BF03699F7000BF0023067516E730
:108A300093F8028008F0E70C83F802C0036993F80A
:108A400004805FFA88FC8DF807C093F8028048F034
:108A5000080C83F802C00369DC70036942F21078E5
:108A600093F803C01CF0020F23D193F803C01CF04D
:108A7000020F1ED193F803C01CF0020F19D193F816
:108A800003C01CF0020F14D193F803C01CF0020FB6
:108A90000FD193F803C01CF0020F0AD193F803C062
:108AA0001CF0020F05D193F803C01CF0020F00F078
:108AB000738193F8028008F0C70C83F802C0D0F8E5
:108AC000108042F2107C98F803309B062DD598F860
:108AD00003309B0629D598F803309B0625D598F8D6
:108AE00003309B0621D598F803309B061DD598F8D6
:108AF00003309B0619D598F803309B0615D598F8D6
:108B000003309B0611D5BCF1080CDCD188F802C0FB
:108B100000BF03699F7000BFD0F8108006756346E0
:108B200098F804C088F803408BE698F8043088F879
:108B3000034086E600248DF806409DF80630036960
:108B400042F21075DF783F0600F1B580DA7816063C
:108B500000F1B180DE78340600F1AD8093F803E0D7
:108B60005FEA0E6700F1A78093F803C05FEA0C6626
:108B700000F1A180DC78240600F19D80DF783F06BB
:108B800000F19980DA78160600F19580083DD9D178
:108B90009D7000BF036980249C7000BF0127427D47
:108BA00007750023012A8DF8093040F0D481002593
:108BB0008DF805509DF80530036942F2107293F864
:108BC00003C05FEA0C6700F11E8193F803E05FEADF
:108BD0000E6600F11881DC78270600F11481DF7839
:108BE0003E0600F11081DE78340600F10C81DD785C
:108BF0002F0600F1088193F803C05FEA0C6600F1CC
:108C0000028193F803E05FEA0E6400F1FC80083A09
:108C1000D5D19A7000BF036980279F7000BF0125DE
:108C2000447D05750023012C8DF80A3040F09081B9
:108C300000228DF804209DF80430036942F210757B
:108C400093F803C05FEA0C6700F1AB8093F803E090
:108C50005FEA0E6600F1A580DC78270600F1A180AE
:108C6000DF783E0600F19D80DE78340600F19980C1
:108C7000DA78170600F1958093F803C05FEA0C6676
:108C800000F18F8093F803E05FEA0E6400F18980C1
:108C9000083DD5D19D7000BF036980269E7000BF3E
:108CA000012202750023B7E5137902279C46D7708D
:108CB00082E50022A7E59D7805F0E7069E7003692E
:108CC00093F804E05FFA8EFC8DF806C09C7844F0BF
:108CD00008079F7002690225D570036942F210757A
:108CE000DE78B4071DD493F803E05FEA8E7718D4DA
:108CF00093F803C05FEA8C7413D4DC78A70710D410
:108D0000DF78BE070DD4DA7894070AD4DE78B70787
:108D100007D493F803E05FEA8E7602D4083DDFD1F2
:108D200036E79D7805F0C7049C70026942F2107323
:108D3000D778BE0640F10281D678B50640F1FE80B4
:108D400092F803C05FEA8C6740F1F88092F803E084
:108D50005FEA8E6640F1F280D578AD0640F1EE8094
:108D6000D478A70640F1EA80D778BE0640F1E680C5
:108D7000D678B50640F1E280083BD9D1937000BFA8
:108D800004698027A77000BF0126026906750225C5
:108D90001679D570427D05E7B8F108087FF460AE1A
:108DA0003DE69D7805F0E7049C7003691F79FEB2EB
:108DB0008DF804609A7842F008059D7003690224DA
:108DC000DC70036942F21075DF78BC074DD4DE78A1
:108DD000B7074AD4DA78970747D493F803C05FEA15
:108DE0008C7642D493F803E05FEA8E743DD4DC784D
:108DF000A7073AD4DF78BE0737D4DE78B40734D477
:108E0000083DE1D146E79A7802F0E7049C700369D7
:108E10001F79FEB28DF805609D7845F008029A70C2
:108E200003690224DC70036942F21072DF78BC0728
:108E30004DD4DE78B7074AD4DD78AF0747D493F82E
:108E400003C05FEA8C7642D493F803E05FEA8E7445
:108E50003DD4DC78A7073AD4DF78BE0737D4DE7874
:108E6000B40734D4083AE1D1D3E69D7805F0C702BF
:108E70009A70046942F21073E778BE065AD5E67814
:108E8000B50657D594F803C05FEA8C6752D594F8BD
:108E900003E05FEA8E664DD5E578AD064AD5E27807
:108EA000970647D5E778BE0644D5E678B50641D59E
:108EB000083BE1D1A37000BF04698022A27000BF0B
:108EC00001270469077502252679E570A4E49A78DC
:108ED00002F0C7059D70046942F21073E778BE0680
:108EE00031D5E678B5062ED5E27897062BD594F8DD
:108EF00003C05FEA8C6626D594F803E05FEA8E65CE
:108F000021D5E578AF061ED5E778BE061BD5E678F5
:108F1000B50618D5083BE1D1A37000BF07698025CD
:108F2000BD7000BF01260269067502241679D4704F
:108F3000447D78E602252379E5706DE402251379F6
:108F4000D570427D2EE602222379E270447D6AE6E6
:108F5000076EC36D59E4076EC36D4CE408B5044B4E
:108F60001A681AB101461046FFF71AFC08BD00BF87
:108F700070DE01204FF47A72704B02FB01F19942CE
:108F8000F0B400F2AF806E4CA14200F2AF806D4DA4
:108F9000A94200F2AD806C4EB14200F2AE806B4F40
:108FA000B94200F2AE806A4B994200F2B080694C3F
:108FB000A14200F2AE80684DA94200F28A804AF6D2
:108FC000A836B14288BF4FF4807200F28380634FAD
:108FD0004FF400464FF48072B94280F08B8053000A
:108FE0005F4FB7FBF3FC614580F089801344B7FB0A
:108FF000F3F5A94280F087801344B7FBF3F4A14254
:1090000080F083801344B7FBF3FC614580F08380DC
:109010001344B7FBF3F5A9427FD21344B7FBF3F433
:10902000A1427CD21344B7FBF3FC614579D21344CF
:10903000B7FBF3F5A94276D21344B7FBF3F7B94275
:1090400073D21344464CB4FBF3FC61456FD2134416
:10905000B4FBF3F5A9426CD21344B4FBF3F7B94265
:109060003ED21344B4FBF3FC614564D21344B4FB19
:10907000F3F5A94229D21344B4FBF3F2914228BF7D
:10908000102223D2F024374D3549374A4FF47A77EE
:1090900007FB03F3B1FBF3F34360286820F00807F4
:1090A0002F60296821F47F2C2CF47F6343F4602027
:1090B00030432043286016683307FCD5294C2568C7
:1090C00045F008022260F0BC70470F22511E0C01CF
:1090D000D9E780225308224CB4FBF2F71E027BE74B
:1090E0000D22F3E71E4F0026012275E70222F1E769
:1090F0000422EFE713460024C5E70822EAE702222C
:10910000E4E71022E6E70322E0E70422DEE720227C
:10911000E0E74022DEE70522D8E70622D6E707226D
:10912000D4E70822D2E70922D0E70A22CEE70B22B1
:10913000CCE70C22CAE70E22C8E700BF4FA9AB005C
:10914000A7D4550053EA2A002975150094BA0A00DD
:10915000495D0500A4AE02005157010095BA0A000E
:109160000095BA0A2C100B4024100B402DE9F04159
:109170000746884607F058FE194C1A4E054604E08B
:1091800007F052FE431BB34226D82368DB07F7D40F
:10919000154A1648C2F80080076007F045FE144CD7
:1091A000104F064604E007F03FFE851BBD4213D872
:1091B0002568104B0E492B40002BF4D00E480A684E
:1091C00002600A6006680B4C3440A4F10104B4FA52
:1091D00084F77809BDE8F0810020BDE8F08100BF88
:1091E00024100B4040420F0008100B400C100B40A5
:1091F00030100B4001000F0098E001202DE9F04FE6
:1092000085B03F4F01900291039207F00DFEDFF809
:109210002CA13C4EBB468146DAF800803A4D07F05F
:1092200003FE044604E007F0FFFD011BA94225D818
:109230003368D907F7D4354A3548C2F80080506002
:1092400007F0F2FD304C054604E007F0EDFD401B51
:10925000A04213D839682F4B0B40002BF5D02E4C71
:10926000DBF800002060CBF800002268294B134097
:10927000012B03D1294D2968CA050FD407F0D4FD6D
:10928000214BC9EB00049C42C6D9019840F233122D
:10929000292105B0BDE8F04F06F02CBE204D214F2E
:1092A0002B701A48039B2049029E002222603B60DB
:1092B0001E4A1F4B06600A601E481F49B8631960AA
:1092C00007F0B2FD104E074604E007F0ADFDC21BEB
:1092D000B2420BD82B78002BF7D12468154D2540CE
:1092E000022D03D1012005B0BDE8F08F019840F2B6
:1092F0003D12232105B0BDE8F04F06F0FBBD00BFD5
:1093000030100B4024100B4040420F0008100B405F
:1093100000001A0D01000F0098E0012010100B4012
:109320009CE0012000100B4004100B4040000100A5
:109330000C100B4002007F1111003A06A0E0012042
:109340002DE9F04F93B0804607F06EFD8B4C8C4EAC
:10935000054605E007F068FD431BB34200F2DC80E0
:10936000236813F00100F5D18649874A0860106030
:1093700007F05AFD854C824D064605E007F054FD86
:10938000871BAF4200F2C8802068814B7F4F0340AB
:10939000002BF3D0DFF81C923968C9F8001039604F
:1093A000D9F800207A4E1640012E40F0B580734E59
:1093B000BB464FF00A0A07F037FD714D044604E042
:1093C00007F032FD021BAA4225D83068C007F7D447
:1093D0006C496D4D6F4B6A4C4FF4D5720A602B602F
:1093E00007F022FD054604E007F01EFD401BA042E9
:1093F00011D83868664A0240002AF5D0DBF8003000
:10940000C9F80030CBF80030D9F80010604D0D409D
:10941000012D00F08181BAF1010ACCD198F8111028
:109420005D4B002908BF4FF44013019307F0FCFC8B
:10943000564F524CDFF84CB10090BA4607F0F4FC9E
:109440004F4E054604E007F0EFFC421BB24258D8ED
:10945000206810F00101F6D14B4B504ACBF80010B8
:109460001A6007F0E1FC464D064604E007F0DCFC1C
:10947000811BA94245D83868454901400029F5D0EB
:10948000DAF80020C9F80020CAF80020D9F80060F6
:109490003F4B3340012B34D107F0C6FC384E054614
:1094A00004E007F0C1FC401BB0422AD82068C10785
:1094B000F7D4354B019A3A49CBF80020196007F0F0
:1094C000B3FC2F4D064604E007F0AEFC831BAB4215
:1094D00017D838682E4901400029F5D0DAF8002065
:1094E000C9F80020CAF80020D9F80030284E1E40E4
:1094F000012E06D107F098FC0099214D401AA84290
:1095000015D9404640F29112432106F0F3FC04467F
:10951000204613B0BDE8F08F40464FF4BF722021C3
:1095200006F0E8FC0446204613B0BDE8F08F1D4B62
:109530001A68002A82DA1C4D1968296018680F4CD5
:10954000420044BF1948067007F06EFC0C4E0746F7
:1095500005E007F069FCC51BB54200F2E78023680F
:1095600013F00105F5D10748074A1149056011605C
:1095700007F05AFC054F024C064623E024100B402E
:1095800040420F0008100B400C100B4030100B40F5
:1095900001000F0000001A080000304000001A37D8
:1095A0000000022910100B4090E001208CE0012007
:1095B0000000090298E0012007F036FC821BA2425D
:1095C00000F2B4803D689E4B9E482B40002BF3D0A8
:1095D0000268C9F800200260D9F80010984E0E40C9
:1095E000012E40F0A38000219748FFF7BFFD00281F
:1095F00000F0AC80954D964C2F6896483B0C1A04B1
:1096000011462260FFF7B2FD002800F0A780DFF8C6
:1096100078A2DFF878922B688F4FDAF80010D9F82B
:109620000020386888F82C100E0A4FEA114C4FEAD7
:10963000116E88F82B60110C160A4FEA102B88F86F
:10964000240088F82820000C88F8303088F82AC0D8
:10965000120E4FEA132C88F8276088F8261000268F
:10966000190C1B0E88F8220088F82E1088F829E0C3
:1096700088F8252088F823B088F82FC088F82D3086
:1096800088F8316021687548FFF770FD002875D0B3
:109690002968DAF80020D9F80030386888F82160A5
:1096A0000D0C0F0A160A88F81E50150C88F81400C5
:1096B00088F8201088F81C20090E88F8183088F8DF
:1096C0001F70120E1F0A88F81B6088F81A501E0CB3
:1096D000050A1B0E000C88F81D1088F8120088F887
:1096E000192088F8177088F8166088F8153088F8FF
:1096F000135021685A48FFF739FDB8B3216859481B
:10970000FFF734FD002841D1404640F2AB12402122
:1097100006F0F0FB044606E74C4F3C68B4F5D57FF5
:109720000CD1514E88F8115001967FE6404640F228
:109730009912212106F0DEFB0446F4E640464FF480
:10974000C272252106F0D6FB0446ECE640464FF4F3
:10975000CE72222106F0CEFB0446E4E6404640F2FB
:10976000A112262106F0C6FB0446DCE6404640F284
:10977000A712242106F0BEFB0446D4E640464FF46F
:10978000D272272106F0B6FB0446CCE60221374808
:10979000FFF7ECFC04460028B6D0354F35493A684F
:1097A00022F006063E603B684FF0101543F00200C1
:1097B000386002AA0D6040466FF07F41FFF71EFD42
:1097C00018B19DF81570BB0729D446F2A811DFF82F
:1097D000C0B0DFF8C0A0DFF8C090274F274E284D5B
:1097E0000023CBF800304046CAF80030C9F80030FA
:1097F0003B6033602B60FFF7BDFB40F243404FF40A
:1098000088614FF0010CCBF80000CAF80000C9F8DD
:10981000001038603060286088F810C083E602AA23
:1098200018494046FFF7EAFC0028CED09DF81810F2
:1098300001F00F02012AC8D14CF25031C7E700BF36
:1098400001000F0030100B4000001A0310100B40F5
:10985000A0E00120000009091C100B400000090ACB
:1098600000001B0700001A370000304000001A06F5
:1098700028100B4044100B400CD0044010D0044082
:1098800014D00440F1FFFF8014100B4018100B405F
:1098900000D0044004D0044008D004402DE9F04F2B
:1098A00085B08DE80E003C4FDFF82C91DFF800A169
:1098B0003A4E0390BB46D9F80080394D07F0B4FA10
:1098C000044604E007F0B0FA031BAB42F3D8336858
:1098D000D907F7D4334A3448C2F80080506007F003
:1098E000A3FA2F4C054604E007F09EFA411BA14263
:1098F000E1D839682D4B0B40002BF5D0DBF8000088
:10990000CAF80000CBF80000DAF80020274D2849FB
:109910001540012DCFD1274C2368DA05CBD5264F32
:1099200026483D70264D00222E780A60019901607C
:1099300036BB009C6202029B1A4D224E2A601C0418
:109940002148224A2249234D44F4007333600560C4
:10995000116007F069FA124C064604E007F064FA59
:10996000851BA5420ED838780028F7D1DAF80070A8
:10997000184A3A40022A05D1012005B0BDE8F08F0F
:10998000009AD8E703984FF40272332105B0BDE87E
:10999000F04F06F0AFBA00BF30100B4024100B4060
:1099A00040420F0008100B4000001A0D01000F008C
:1099B00098E0012010100B409CE0012000100B40AB
:1099C0008CE0012004100B4038100B400C100B40B1
:1099D00027003A1902007F11A0E001202DE9F04F85
:1099E000ADF6140D01238C00019011461C4402A811
:1099F0005C2200948DF80C383D4FDFF83891DFF889
:109A000008A13C4E06F09AFBBB46D9F800803A4DBF
:109A100007F00AFA044604E007F006FA001BA84221
:109A2000F3D83068C107F7D4344A3549C2F800800A
:109A3000516007F0F9F9304C054604E007F0F4F9FD
:109A4000431BA342E1D838682E4B0340002BF5D0CE
:109A5000DBF80010CAF80010CBF80010DAF800208C
:109A6000284D29481540012DCFD1284C2368DA050F
:109A7000CBD5274F274A3D70274D00212E78016016
:109A800002A8106026BB009C63021C48234D244999
:109A9000244A0360244E254B254C2E600C60136035
:109AA00007F0C2F9144E054604E007F0BDF9421B69
:109AB000B2420FD838780028F7D1DAF800701C4984
:109AC0003940022906D100200DF6140DBDE8F08FB3
:109AD000009BDAE701984FF40272332106F00AFA8C
:109AE0000028F0D105200DF6140DBDE8F08F00BF61
:109AF00030100B4024100B4040420F0008100B4068
:109B000000001A0D01000F0098E0012010100B401A
:109B10009CE0012000100B408CE0012004100B4061
:109B200038100B400C100B400002040027003A19BB
:109B300002007F11A0E001202DE9F04F0123ADF6D6
:109B40001C0D424FDFF84491DFF818A1404E0390FE
:109B500089001944019102928DF81438BB46D9F856
:109B600000803C4D07F060F9044604E007F05CF922
:109B7000031BAB42F3D83068C107F7D4364A3749E4
:109B8000C2F80080516007F04FF9324C054604E0FE
:109B900007F04AF9401BA042E1D83868304B034037
:109BA000002BF5D0DBF80010CAF80010CBF800103D
:109BB000DAF800202A4D2B481540012DCFD12A4C30
:109BC0002368DA05CBD5294F294A3D70294D00215C
:109BD0002E78016004A8106046BB019C63021E4AF7
:109BE00025492648264D274E274C13600D601663E5
:109BF000046007F019F9174E054604E007F014F960
:109C0000411BB14214D83B78002BF7D1DAF8007031
:109C10001C4A3A40022A0BD104A902985C2206F0A1
:109C20008DFA00200DF61C0DBDE8F08F019BD6E7E4
:109C300003984FF4F472312106F05CF90028EBD15F
:109C400005200DF61C0DBDE8F08F00BF30100B4055
:109C500024100B4040420F0008100B4000001A0D6A
:109C600001000F0098E0012010100B409CE0012043
:109C700000100B408CE0012004100B400C100B4036
:109C80000002040002007F1137003A12A0E0012018
:109C90000EB42DE9F04F82B00BAB064653F8042BFF
:109CA00071480093402106F5BB570AF003FF1837AF
:109CB00042F2900242F2910142F292033068B854AB
:109CC0000125002406F55F567C54DFF8B481FD546D
:109CD0003436664D02E0012007F0CAF8326892F887
:109CE00064100029F7D14FF4804260480AF088FBE5
:109CF0005F4800F17B0E00F510698346DA460AF8EA
:109D0000804B8BF880408AF880408BF800448BF8B9
:109D100080418BF800428BF880428BF800438BF82F
:109D200080430BF5906BCB45E8D101308645E2D1FD
:109D30000023FF2203F5D85C03F5DC5003F5E05166
:109D40000CF1020E0230023105F80E2003F5E45B3F
:109D50002A5403F5E85A6A5403F5EC5903F5F05C0C
:109D600003F5F45E03F5F85003F5FC510BF1020B1B
:109D70000AF1020A09F102090CF1020C0EF1020EBD
:109D80000230023103F5A063B3F5206F05F80B2014
:109D900005F80A2005F8092005F80C2005F80E2022
:109DA0002A546A54C6D17D22FF2132480AF028FB8A
:109DB0000023FF2203F5DB5C03F5DF5003F5E351DD
:109DC0000CF11E0E1E301E3105F80E2003F5E75B68
:109DD0002A5403F5EB5A6A5403F5EF5903F5F35C83
:109DE00003F5F75E03F5FB5003F5FF510BF11E0B76
:109DF0000AF11E0A09F11E090CF11E0C0EF11E0ECD
:109E00001E301E3103F5A063B3F5206F05F80B205B
:109E100005F80A2005F8092005F80C2005F80E20A1
:109E20002A546A54C6D17D22FF2113480AF0E8FA69
:109E3000124A10680190019BC3F3080001224021DF
:109E4000B0F5807FC8F80010C8F80410C8F80C20DE
:109E5000C8F81020C8F82C2002D90348FAF7B4FC3F
:109E60003846F9F72FFB36E7B433FF1F4034FF1FA6
:109E7000C34FFF1F424FFF1FC258FF1FACE001201E
:109E800070D0FF1F2DE9804800F5BB5808F1180875
:109E900042F29004056808F8045042F2910742F239
:109EA00092034FF00109002400F55F5608F80740BF
:109EB00083B008F80390684D684F8946924634365F
:109EC00002E0012006F0D4FF306890F86410002909
:109ED000F7D14FF4804260480AF092FA604800F1EE
:109EE0007B0E00F5106183465A4602F8804B8BF8D2
:109EF000804082F880408BF800448BF880418BF8DA
:109F000000428BF880428BF800438BF880430BF5BE
:109F1000906B8B45E8D101308645E2D10023FF22CA
:109F200003F5D85101F1020B03F5DC5C03F5E05EAB
:109F300003F5E45003F5E8510CF1020C0EF1020EAA
:109F40000230023105F80B2005F80C2003F5EC5B1C
:109F500005F80E2003F5F05C2A5403F5F45E6A540C
:109F600003F5F85003F5FC510BF1020B0CF1020C58
:109F70000EF1020E0230023103F5A063B3F5206F3B
:109F800005F80B2005F80C2005F80E202A546A5419
:109F9000C6D17D22FF2133480AF032FA0023FF2286
:109FA00003F5DB5B03F5DF5C03F5E35E03F5E750E8
:109FB00003F5EB510BF11E0B0CF11E0C0EF11E0EF6
:109FC0001E301E3105F80B2005F80C2003F5EF5B61
:109FD00005F80E2003F5F35C2A5403F5F75E6A5486
:109FE00003F5FB5003F5FF510BF11E0B0CF11E0C9A
:109FF0000EF11E0E1E301E3103F5A063B3F5206F67
:10A0000005F80B2005F80C2005F80E202A546A5498
:10A01000C6D17D22FF2114480AF0F2F9134A3C61AF
:10A02000106801900199C1F3080B012340203821E9
:10A03000BBF5807F87E80300FB60FB6202D94846DE
:10A04000FAF7C2FB4122514609487A60FBF752FAFF
:10A050004046F9F737FA34E74034FF1F70D0FF1F4E
:10A06000C34FFF1F424FFF1FC258FF1FACE001202C
:10A07000200102002DE9F04FBC4C2DED0A8BD4EDF0
:10A08000007A41F22403E1B0F5EE407A8346011DE7
:10A09000C55C00915030F1EE10FA05900BF2744758
:10A0A00009D197ED000AB5EE400AF1EE10FA02D0A0
:10A0B000AF4E024608E0002D00F04981AC4E3178E9
:10A0C000002940F04981059A00990BF56F5808F175
:10A0D00038094846FEF7E2F90BF5805A0AF11808EC
:10A0E0000BF5855E724610323F68357002F5BA7026
:10A0F000276003920BF59157F8F792F90BF59251FF
:10A100000BF5965097F820C091F820603D460BF56E
:10A1100093520BF594530BF595540C300C370C31CE
:10A1200097F815A0497D077D92F820008BF804C0B0
:10A130008BF8056093F820C094F820600C320C3343
:10A140000C345B7D527D647D8BF807C08BF8086012
:10A1500095F8E0C095F820618BF80970043595F802
:10A16000FC7095F83C518BF80E40009C8BF8060073
:10A170000BF560508BF80AC08BF812308BF80B701F
:10A180008BF80FA08BF810108BF811200C302146A3
:10A190008BF80C608BF80D50FAF794F9059A21466C
:10A1A0004846FEF77BF90BF1490A00218BF8441071
:10A1B00004225046DBF8E87F0AF022F9CBEB0A01D3
:10A1C0000BF14403A1F145020BF14500002102937C
:10A1D0000AF016F97B1C01F0718307EB87060BEB85
:10A1E000860570350FCD0DF17C0AD646AEE80F001E
:10A1F0005F44BAF800002A68CEF80020012487F8EE
:10A200004940002801F04E8341F224011BF801600F
:10A21000A0F580700025B0FA80F254098BF8445004
:10A2200087F84540002E00F0AF86DBF85C70012611
:10A23000002F40F0A9864FF0030C0BF58053043338
:10A240005D788BF84DC041F2040E002D00F09F8622
:10A250001BF80E00002801F099839A78002A0CBFA1
:10A26000012202228BF84E209BF8D07F7B1E0BF53B
:10A270007354012B04F10C0440F27C8621460F221A
:10A2800000980AF027F8DBF83020216BDBF8343037
:10A29000E56A94ED105AD8ED006A94ED116A98EDD4
:10A2A000017AD4ED125A98ED022A551B5A1A636BA3
:10A2B000DBF838101543C91A0D43DBF83C30A16BAD
:10A2C000E26B76EEC52A5B1A37EE463ADBF84010B1
:10A2D000B7EE004AF0EEE23A72EE654A2B43F4EE36
:10A2E000C43A8D1AB0EEC3AAF1EE10FA43EA0503A0
:10A2F000B4EEC4AAF0EEE4AAC8BF43F00103F1EE45
:10A3000010FAF4EEC4AAC8BF43F00103F1EE10FA4C
:10A31000C8BF43F00103034340F02C861549089160
:10A320000D68129541F20800129B5BF80020991A03
:10A33000B1F5FA7FC1F0A4810F4D0195032F01F211
:10A340002983DFE817F0F200CF02C1001B00084E9E
:10A350003278002A41F0A1830BF56F590BF5805A32
:10A3600009F138090AF11808BAE600BFAC33FF1F3B
:10A37000B033FF1FACE001203C34FF1F0F22214609
:10A38000009809F0A7FF98ED00BAD4ED10BAE66A7C
:10A3900098ED01CAD4ED11CA636BD8ED027A94ED41
:10A3A000120ADBF83010276B04937BEE6B8A35467C
:10A3B000DBF83420DBF8383006963CEE6CAAB7EEBA
:10A3C000001A491BF0EEE80A37EEC08A049DD4F863
:10A3D00038C0DBF83C60D4F83CE00797F4EEC10AE3
:10A3E000D21BF0EECA1A5D1BF1EE10FA41EA02012F
:10A3F000F4EEC11AF0EEC89ADBF84020CCBF01237E
:10A4000000232943F1EE10FACCEB0606F4EEC19AD4
:10A41000C8BF43F001033143F1EE10FACEEB020561
:10A42000C8BF43F0010341EA05063343034300F08C
:10A4300095829BF80450D5B99BF80500B8B99BF8F4
:10A440000670A7B99BF807308BB99BF8081071B953
:10A450009BF809205AB99BF80A6046B99BF80B0093
:10A4600028B99BF80C7017B99BF80D3013B1012176
:10A4700084F8511004F12C070FCF0BF130060FC6F2
:10A480003A68069FDBF838100346DBF83400326088
:10A49000DE1B079BDBF83C209BF8D17F8BF8D07F3D
:10A4A000C01A3043049EDBF84030891B0843CCEBD4
:10A4B00002020243CEEB0300002384F8583042EA44
:10A4C0000006DBF858304DE243F61D551BF80560D9
:10A4D000CEB99BF8077037B943F6CF411BF801207E
:10A4E000002A42F0E0819BF8080060B943F6D043AF
:10A4F0001BF803503DB19BF8EC6F0136042ED8BF1A
:10A50000F0B28BF8EC0FE36BDBF84020D51A01F0CA
:10A510007E849BF8EC0F042802F21B81DFE810F028
:10A52000180FFE0ED40E9C0E4C0E9BF80A202AB972
:10A53000A7791FB1E56C002D01F047879BF80B1040
:10A5400039B9E07928B1E36C012B04BF4FF0FF3338
:10A55000E3649BF80CE0BEF1000F07D1277A2FB11E
:10A56000E56C022D04BF4FF0FF35E5649BF80DC08C
:10A57000BCF1000F07D1607A28B1E36C032B04BF54
:10A580004FF0FF33E36494F8C030002B41F06B834D
:10A590009BF80950DBF85C7004971DB160790028C6
:10A5A00001F0DA8543F61D501BF800009BF870702F
:10A5B00027B99BF87130B3FA83F77B099BF8847055
:10A5C00027B99BF88570002F08BF01239BF898706E
:10A5D000002F41F03E849BF89970002F41F03984A0
:10A5E000002841F04A830498002841F0D38535B112
:10A5F000677927B9089805681695169B6365DBF897
:10A60000E83F002A41F04D85A07958B194F85050A8
:10A610002DB9002B02F0BE81CBF8E82F13460022A3
:10A6200084F85020E279002941F03C8762B194F827
:10A63000501031B9012B14BF01234FF0FF33CBF879
:10A64000E83F002684F85060217ABEF1000F41F007
:10A650003F8761B194F8506036B9022B14BF0223D2
:10A660004FF0FF33CBF8E83F002784F85070BCF17F
:10A67000000F01F00487607A88B9E26C002AC2F208
:10A680004D81032A02F04A81032601274FF0FF354E
:10A69000CBF8D42FCBF8D86F8BF8D07FE5649BF83C
:10A6A00007E0BEF1000F01F09586E078002841F048
:10A6B00091869BF805705FB141F2240600254FF0AA
:10A6C000020C01210BF806508BF8D0CF84F8511002
:10A6D000591C01F072879BF80800002841F0A18600
:10A6E000267906B3A57A002D42F038819800C21869
:10A6F0000BEB820C9CF87360042E02F01E819CF818
:10A700007050002D42F012819CF871204FF4717648
:10A71000B2FA82F506FB03B069098CF871104FF0AC
:10A72000010C80F859C49BF80E20002A41F07E8667
:10A730002279002A42F01781E16C4A1C01F0B787A8
:10A740009BF80F309BF80620BBB1E67A8EB994F8DF
:10A75000BE5075B941F205011BF80130002B02F023
:10A76000128141F2040C1BF80C1081F001030BF86C
:10A770000C30E16C4B1C01F03C869BF80450EDB9A9
:10A7800043F6CC461BF80600C0B1E37AB3B901EB3F
:10A7900081060BEB860C0120DCF88030CBF8803092
:10A7A000DCF88060CBF89460DCF88030CBF8A8301F
:10A7B000DCF88060CBF8BC6084F85000D7B96078D2
:10A7C000C0B1237BB3B901EB81060BEB860C0120F2
:10A7D000DCF87C30CBF87C30DCF87C60CBF8906027
:10A7E000DCF87C30CBF8A430DCF87C60CBF8B860C7
:10A7F00084F85000002A41F00E86A078C0B1637B37
:10A80000B3B901EB81060BEB860C0120DCF8783044
:10A81000CBF87830DCF87860CBF88C60DCF87830F6
:10A82000CBF8A030DCF87860CBF8B46084F8500046
:10A83000BEF1000F41F0E085E078002801F0848748
:10A84000A37BABBBBBF87060B6F5807F07D001EB94
:10A8500081000BEB800CDCF87430CBF87430BBF863
:10A860008460B6F5807F07D001EB81000BEB800C94
:10A87000DCF87430CBF88830BBF89860B6F5807F90
:10A8800007D001EB81000BEB800CDCF87430CBF8C7
:10A890009C30BBF8AC60B6F5807F06D001EB81013F
:10A8A0000BEB8100436FCBF8B030012684F8506089
:10A8B000002A01F0A1854FF0000E84F8BDE01FB919
:10A8C00063780BB184F8BF70002D41F0D88143F656
:10A8D000CC471BF80760002E01F0D18184F8BE50F0
:10A8E00001F0CDB99BF80770002F01F057819BF85C
:10A8F00005301BB96078002841F055839BF8E42FA0
:10A90000002A42F04D80DBF83060E26A216BDBF810
:10A910003430DBF83850676B98ED00CAD4ED10CABC
:10A9200098ED010AD4ED110AD8ED027A94ED121ACD
:10A93000B01A5B1ADBF83C60A16BDBF840200343E4
:10A94000ED1B701AE66B2B430343921B7CEE6C8A63
:10A9500030EE60AA37EEC18A42EA0306DBF85830CF
:10A960009BF80450042B25D8C34A52F823200AB37D
:10A970000899C2480B681193119BDBF8F41F5B1A0E
:10A980009A4217D29BF8D0CF0CF1FF32022A11D98C
:10A990000168109141F201004FF0010E109A8BF8FE
:10A9A000D1CF0323CBF8F02F0BF800E08BF8D03F8A
:10A9B00084F858E00F222146009809F08BFCB0EE95
:10A9C000E86AF7EE008AB4EEE86AB0EECAAAF1EEE1
:10A9D00010FAB4EEE8AACCBF01210021F1EE10FA82
:10A9E000CCBF01220022B0EEC88AB4EEE88A0A4346
:10A9F000F1EE10FA46EA0206C8BF46F0010656EA32
:10AA0000000305D1019E3068431C0F28336008DD28
:10AA100098E8070004F1400E8EE80700019900262F
:10AA20000E60FDB99BF80550E5B99BF80620CAB940
:10AA30009BF80700B0B99BF808309BB99BF80960F8
:10AA400086B99BF80A1069B99BF80B5055B99BF869
:10AA50000C203AB99BF80D0020B943F61D5C002389
:10AA60000BF80C3098E80700009E04F1400E3546C4
:10AA70008EE807000FCD0FC40FCD0FC40FCD0FC44C
:10AA800095E80F0084E80F000BF576503146059AE3
:10AA90001030FCF759FD039C029904F53070F6F76D
:10AAA000B1FF43F2F4715BF8012092F86460C6B91B
:10AAB00041F201051BF80510002901F0E781DBF8E0
:10AAC00060706F48032FCCBFFF2100214FF48042FC
:10AAD00009F096FC0BF5BB501830F8F7F3FC0BF8B7
:10AAE000056045F610440BF581535BF80450002DCA
:10AAF00003F1180380F2AC85099345F614455BF821
:10AB00000510002979DB099C0BF5A34022464C3047
:10AB1000FFF712F82146059805F0C2F80BF57051C1
:10AB200041F20602D9F810008B6A8E6CBBF82C70CB
:10AB300000244FF0000C0BF802C0C9F80C00C9F853
:10AB400014404B620BF5715330334E64CC62CC64CD
:10AB50000BF572501968C8F800100C300BF5725CD8
:10AB60000268C8F8042005EE907ADCF82810C8F8CE
:10AB700008100BF58053B8EE650A4846D3F80C80F0
:10AB8000404EF6F79BFBBBF82E200BF5715702EEFB
:10AB9000102A0BF5805C87ED0A0AC7F8248009F1BA
:10ABA0002000FC613E62B8EE420ADCF81080F6F745
:10ABB00085FBBBF82A100BF5715302EE901A0BF5CA
:10ABC000725709F140000BF5805983ED110A9C631F
:10ABD000DE63B8EE620AC7F80080D9F81480F6F791
:10ABE0006DFB0BF572504FF0FF3380ED080A4461A6
:10ABF0008661C0F81C804BF805300BF5B8450BF5A5
:10AC000064570BF56356DFED20AA9FED20BADFED08
:10AC100020BADDF81490173504373C36D8465C4628
:10AC200094F8733015F8011F994200F0848194F86C
:10AC30007020002A40F0718157ED023A307A032BE0
:10AC4000B8EEE33A00F0748123EE2B0A05F0AAFF78
:10AC50007268307A0121914001EBD173591005F0EF
:10AC600097FD94F87300287094F872202A7294F873
:10AC70007010297112E000BF30090200ACE0012021
:10AC80004034FF1F00F07F4500A00C4600007A45CD
:10AC900000409C466666E63F6666663F14344C4557
:10ACA00007F10C0706F10C06BAD10BF583452F46C8
:10ACB00007F120041C3507F14C0300201FED0B9A0F
:10ACC0005FED0B8A019502940393D9460490CDF869
:10ACD00018B0069A9BF8707092ED158A09F57D55AB
:10ACE0003835002F40F0F38098F87874D06E0790D4
:10ACF000002F40F07B8109F58347079BA84C039800
:10AD00003C6001267860FE6323B99BF87120B24253
:10AD100000F01F819BF87370042F00F01A8108F275
:10AD20005C4C0199DCF800500D6008F58C6E0298BF
:10AD3000DEF80040046008F2644609F58343326897
:10AD40005A6208F26C4709F5834C3D68CCF82C50E8
:10AD500009F58743934F1D6E934CDFED940A9FEDE9
:10AD6000941ADFED941A9FED945A9FED946A9448DB
:10AD70009FED8FAADFED939A9FED93BA07FB05F540
:10AD80002C44C4F30E4C07EE90CAF8EEE76A1C663A
:10AD900066EEA0CA08F2744EECEE811A09F58741FE
:10ADA00068319EED002AD1ED005A71EE82AA09F5B4
:10ADB0008347EAEE855A3B46F4EEC65AF1EE10FAA6
:10ADC000A8BF75EEC65ABDEEE5CAC1ED005A1CEE2D
:10ADD000106A00EB8602D2ED00BAF1EE6B2AE2EEC9
:10ADE0008A9AA2EE8ABAC7ED0D9A83ED0EBA08F5DB
:10ADF000896509F5834C2C68019E9BF87370CCF82B
:10AE0000084008F24C4E09F58342DEF80030136129
:10AE100006F58F64029E0194B7FA87F306F58F64F6
:10AE20005809039E82F8410094461146A7F1010299
:10AE3000049D029406F58F64B2FA82F6A7F103032B
:10AE400003947409A7F10206A7F1040781F84240B0
:10AE5000B3FA83F00135B6FA86F4B7FA87F74209F8
:10AE60007B096009042D049508F571780BF1140B2A
:10AE70008CF843208CF844008CF8453009F58F6934
:10AE80008CED058A7FF425AF05990998DDF81880C7
:10AE900004F036FF20B141F20605012108F8051043
:10AEA00008F24C49DFED498A99ED008A28EE280A1C
:10AEB00008F0CEF980EE289AB5EE409AF1EE10FA3D
:10AEC00040F0EA8361B0BDEC0A8BBDE8F08F09F574
:10AED00083459BF872103E4E394C2C6056F8213059
:10AEE0009FED3C4A019E0299DFED3B4A9FED39CA36
:10AEF0006B6009F5834E394C00204FF07E55CEF83B
:10AF00003C0086ED004A0D60CEF82440CEF82C407F
:10AF1000CEED0D4A8EED0ECA69E717ED027A94F870
:10AF20007230307AB8EEC73A13B923EE0B0A8DE6C9
:10AF300023EE2A0A8AE6287A94F872E094F87020C0
:10AF400070457FF476AE95F804C094457FF471AEF9
:10AF5000A4E609F5834E019E9FED1E0A02981F4A42
:10AF600086ED000A4FF07E510160CEF82420CEF825
:10AF70002C20EDE61A48089002681392139BCBF838
:10AF8000F43F0899FFF7CCB9B446FFF756B9997862
:10AF900000290CBF002102218BF84E10FFF764B985
:10AFA00070DEFF1FFD430300C39E26008000803734
:10AFB000CDCCCC3D8FC2753D6F12834100008046E1
:10AFC00070DE00200000FE4233334B4100007A4423
:10AFD0008422FF1F0000000000000043000080BF2B
:10AFE000ACE001200AD7233C0AD7A33C642005F03B
:10AFF0006BF80CEE900A5FED050A089A1FED061A31
:10B0000016681D96B8EE6C0A1D9BE34960EE207A27
:10B01000E7EE810AF0EE609A13B90C681E941E9B4D
:10B0200009F5824E1846CEF87C3009F03BFA5646B8
:10B030000DF5BE7C3046CAEB060700F8017BF41C18
:10B04000421CCAEB0203CAEB0001CAEB0407717091
:10B05000321D4370701DF770B31DF71DCAEB02045B
:10B06000CAEB0001CAEB0302CAEB0700347171712D
:10B07000B271F07108366645DCD10DF17D04A31B79
:10B08000D943FF2201F003078AF8002109F014FADE
:10B09000CAEB060C90FBFCF303FB1C0016F8012C1A
:10B0A0001AF8001006F8011C013EA6420AF800201A
:10B0B00077D097B3012F1FD0022F0ED009F0FCF9E3
:10B0C000CAEB060790FBF7F303FB170C16F8010D0C
:10B0D0001AF80C2032700AF80C0009F0EDF9CAEBEE
:10B0E000060190FBF1F707FB110316F8010D1AF8A2
:10B0F000032032700AF8030009F0DEF9CAEB0601FA
:10B1000090FBF1F707FB110316F8010D1AF8032065
:10B110003270A6420AF8030043D009F0CDF9CAEB19
:10B12000060190FBF1F707FB110C16F8013C1AF829
:10B130000C0006F8010C0AF80C3009F0BDF9721E7B
:10B14000CAEB020190FBF1F707FB110C16F8023C69
:10B150001AF80C0006F8020C0AF80C3009F0ACF9E9
:10B16000B21ECAEB020190FBF1F707FB110C16F8B7
:10B17000033C1AF80C0006F8030C0AF80C3009F02E
:10B180009BF9F21ECAEB020116F8043D90FBF1F7A1
:10B1900007FB110CA6421AF80C0030700AF80C30AC
:10B1A000BBD128464FF48072514604F0C7FF09F521
:10B1B00080404FF480725146783004F0BFFF049A0B
:10B1C0000699039B9FED77CADFED74CACDF82880FE
:10B1D00009F58244F5EEC09A4FF48F65783405FB8B
:10B1E0000217F1EE10FAC8BFC4ED009ACDF82C900A
:10B1F00000970025F1EE08AABAEE0EAAF2EE049A24
:10B20000B5EE00BAF7EE00BA9846CDF830B0A146D8
:10B21000CDF834A005EE105AD9ED001AF8EEC56A43
:10B22000013526EEA16A16EE100A08F0A5F90646C9
:10B230000F4647EC106B07F07BFF5BEC10AB10EE9A
:10B24000100A594608F09CFC52465B465FFA80FAA9
:10B250003946304608F030F808F0DAFC02EE100A01
:10B26000009882440AF57D5BF0EE4A5A9BF838401C
:10B270009BF8391004F0030603EE106A01F0030294
:10B28000B8EEC34A07EE902AB0EE6B0AE2EE2A5AF5
:10B290002607A4EE0B0AF8EEE71AF0EE6B6AE1EE71
:10B2A0008B6AF0EE692AF0EE400A32EE6B5AE2EE5B
:10B2B000252A62EE023A4CBF60EE420A62EE200A94
:10B2C0000C0763EE824A4CBF26EEC55A25EE265A7D
:10B2D00024EEA21A35EE602AE1EE020AF4EEEC0A40
:10B2E000F1EE10FAB4EE60CAD8BFF0EE60CAF1EE2B
:10B2F00010FA48BFB0EE60CA802DE8EC010A89D18F
:10B30000039FDDF834A0D7ED00AA3AEEECAA3CEE9C
:10B310006CCA6AEE099A0DF1280E89EE8CBA9EE885
:10B32000000B09F587403B464C30C51B2C1FC4F36E
:10B3300081067BEE68BAE3EC01BA83426AD0AEB311
:10B34000012E19D0022E0BD0D3ED002A32EEEC7A6A
:10B3500027EE093AC3EE0C3A33EEE84AA3EC014A71
:10B36000D3ED004A34EEEC0A60EE090A80EE8C1A46
:10B3700071EE687AE3EC017AD3ED001A31EEEC5A03
:10B3800065EE096A86EE8C6A36EE682AA3EC012A1D
:10B3900083423FD00AE000BFACE00120FFFF7F7F87
:10B3A00000FEFF460000000000F07F45D3ED005A8C
:10B3B00075EEECAA9C462AEE89AA1033CAEE0C9AC6
:10B3C00039EEE8BAACEC01BA53ED03BA7BEEEC2AE5
:10B3D00022EE893A83EE0C7A77EE683A43ED033A2F
:10B3E0009CED014A74EE6C4A24EE890AC0EE0C0A08
:10B3F00030EEE81A8CED011A53ED017A77EEEC1A73
:10B4000021EE895AC5EE0C6A36EEE86A03ED016A50
:10B410008342CBD109F5874E039F1FED1FCA002140
:10B42000CEF85410CEF858103B46F3EC01CA2CEE7F
:10B430008C2AC41BFDEEC25A261FCDED005ABDF961
:10B440000020C8F8C0208342C6F3820108F1C00C76
:10B4500000F0CA80002963D0012953D0022945D0C9
:10B46000032937D0042929D005291BD006290DD05E
:10B47000F3EC01AA2AEE8CAA08F1C40CFDEECA9ADC
:10B48000CDED009ABDF90070C8F8C470B3EC01BAF4
:10B490006BEE0CBAFDEEEB2ACDED002ABDF90050A3
:10B4A0004CF8045FB3EC013A23EE0C7AFDEEC73A98
:10B4B000CDED003ABDF900404CF8044FB3EC014A21
:10B4C00064EE0C4ABDEEE40A8DED000ABDF90060A1
:10B4D0004CF8046FF3EC010A20EE8C1AFDEEC17AF1
:10B4E000CDED007ABDF900204CF8042FF3EC011AE1
:10B4F00021EE8C5AFDEEC56ACDED006ABDF9001053
:10B500004CF8041FB3EC016A66EE0CCA8342BDEE30
:10B51000EC2A8DED002ABDF900704CF8047F63D051
:10B520009E46FEEC015A65EE8CAA2033BDEEEAAAD7
:10B530008DED00AABDF90050CCF8045053ED079AE8
:10B5400029EE8CBAFDEECBBACDED00BABDF90040C4
:10B55000CCF80840DEED012A22EE8C3ABDEEC37A2B
:10B560008DED007ABDF90060CCF80C6053ED053A22
:10B5700023EE8C4AFDEEC44ACDED004ABDF9002011
:10B58000CCF8102013ED040A60EE0C0ABDEEE01AB0
:10B590008DED001ABDF90010CCF8141053ED037AAC
:10B5A00067EE8C1ABDEEE15A8DED005ABDF90070C0
:10B5B000CCF8187053ED026A26EE8C6AFDEEC6CA0E
:10B5C000CDED00CABDF90050CCF81C5013ED012A96
:10B5D00062EE0C5A8342FDEEE5AACDED00AABDF95C
:10B5E00000404CF8204F9BD11FED92CA5FED929A1C
:10B5F000002008F2444CC8F8400409F587438CED5C
:10B6000000CA93ED12AAB7EE00BA7AEE0BBAF6EEC4
:10B61000002A2BEEA93A012223EE227A08F27C4E70
:10B62000FCEEC73ACDED003ABDF8006004EE106ABA
:10B63000F8EE444ACEED004A88F8800488F8780491
:10B6400088F8582488F8592488F87924FFF753BBE0
:10B650001846059909931F4604F0E0FB41F2060CD9
:10B6600000260BF5A3403A4629460BF80C604C30F7
:10B67000FEF7B4F94FF0FF324BF80420FFF73DBA64
:10B6800098E8070004F1400C8CE80700DE480190C0
:10B6900000230360FEF752BEB5EEC08AF1EE10FA49
:10B6A00000F14C845546BDEEC87A05F1FF3EF8EE38
:10B6B000C73A17EE103A002038EE634AD34E00E046
:10B6C000084686FB0327D917C1EBA70B0BEB8B02B0
:10B6D000A3EB420330330EF8013F5B46411C002BC5
:10B6E000EED15FEA61087FD06A182B4612F8014D4F
:10B6F0002F7803F8014BA844EE43464443451770A6
:10B7000006F0070470D0BCB3012C2DD0022C25D03C
:10B71000032C1DD0042C15D0052C0DD0062C05D0E3
:10B720001E7812F801CD03F801CB16701C7812F8C0
:10B73000019D03F8019B14701E7812F801BD03F8F7
:10B7400001BB16701C7812F801ED03F801EB1470C0
:10B750001E7812F8017D03F8017B16701C7812F830
:10B76000016D03F8016B147012F801CD1F7803F816
:10B7700001CB4345177037D0994612F8014C1E781B
:10B7800009F8014B02F8016C5F7812F8024C5C700A
:10B7900002F8027C99F8016012F8037C89F80170C4
:10B7A00002F8036C93F803B012F8044CDC7002F852
:10B7B00004BC1E7912F8057C1F7102F8056C93F821
:10B7C00005E012F8064C5C7102F806EC9E7912F85E
:10B7D000077C9F7102F8076C12F8086DDC79DE7146
:10B7E000083343451470C7D1F2EE044A24EE240A0C
:10B7F000DFF8188260EE240ABDEEC01A60EEA41ACB
:10B8000011EE103ABDEEE06A88FB032621EEA45A41
:10B81000DA1716EE107AC2EBA609FDEEE17AFDEE1C
:10B82000C56A09EB890B2E18A3EB4B0288FB073086
:10B83000FB1716EE904A17EE90CAC3EBA00E0EEB64
:10B840008E00A7EB40074FEAEC7388FB0C0988FBDE
:10B850000408E017C3EBA90BC0EBA8090BEB8B0E98
:10B8600009EB8908ACEB4E0CA4EB48032E2068547E
:10B8700030320CF13004303300213037B270737144
:10B88000B1715046F770347109F03AF801465046EC
:10B8900006F0BAFA5E4804F0F1FB61B0BDEC0A8B29
:10B8A000BDE8F08F41F224031BF80360002E40F046
:10B8B000A8808BF844403446FEF7B2BC41F2240025
:10B8C0000BF1700E1BF80060BEE80F000DF17C0A52
:10B8D000D446ACE80F00DEF80020BAF80050CCF8EF
:10B8E0000020002E40F09C80B5F5807F00F0BC85E4
:10B8F0008BF845601DB94FF0010E8BF844E00BF159
:10B9000084050FCD54460FC4BAF800302868206073
:10B91000B3F5807F00F0A38500228BF8462013B991
:10B9200001278BF844700BF1980EBEE80F00D44647
:10B93000ACE80F00BAF80050DEF80040CCF8004048
:10B94000B5F5807F00F0EB8500238BF8473015B903
:10B9500001208BF844000BF1AC070FCFD646AEE8C0
:10B960000F00BAF800103D68CEF80050B1F5807FA6
:10B9700000F0D08500248BF8484019B94FF0010C35
:10B980008BF844C04FF0000CFEF757BC8BF84E000C
:10B99000FEF76ABC40F213321E491F48F5F758FC07
:10B9A000DBF83060E06ADBF83470216BDBF838508C
:10B9B00098ED001AD4ED101AD8ED019A94ED115AB1
:10B9C00098ED029AD4ED126A7B1A321A676BDBF893
:10B9D0003C60A16BE81B1A43DBF84050731AE66B1E
:10B9E00002431A43A81B71EE618A39EEC5AA39EEEB
:10B9F000668ADBF858309BF8045042EA0006FEF7EE
:10BA0000B1BF2646FEF704BC3C34FF1F676666667E
:10BA10002029FF1F30FF01002401020000F07F45B4
:10BA20000BF184060FCE54460FC40BF1980E31680B
:10BA30002160BEE80F00D446BAF80070ACE80F00F1
:10BA4000B5F5807FBAF80030DEF80000CCF80000D1
:10BA50000CBF01250025B7F5807F0CBF012700270B
:10BA6000B3F5807F0CBF012300238BF845500BF109
:10BA7000AC058BF847300FCD56468BF846700FC695
:10BA8000BAF800402A683260B4F5807F00F0F28492
:10BA900000278BF84870FEF7C8BB0BF56F590BF504
:10BAA000705809F138094FF0000AD9F81030D8F869
:10BAB0002810D8F848E0C9F80C30C9F814A0C8F824
:10BAC0002CA0C8F84CA0C8F844E0C8F82410BBF873
:10BAD0002C801FED2E8A0BF5805C0BF5715000EE6B
:10BAE000908A0CF11808026BC8F800200BF572530D
:10BAF0000BF5725ED968C8F80410DEF82800C8F8A3
:10BB000008000BF58052B8EE600A4846D2ED038A71
:10BB1000F5F7D4FBBBF82E100BF5715C01EE101A93
:10BB20000BF58053CCED098A8CED0A0ACCF81CA0E9
:10BB30008CED088A09F12000B8EE410A93ED049AD1
:10BB4000F5F7BCFBBBF82A100BF5715C01EE901AFF
:10BB50000BF572528CED110ACCF838A08CED0F8ADF
:10BB60000BF5805382ED009A09F14000B8EE610AAE
:10BB7000D3ED059AF5F7A2FB0BF57250844680EDE4
:10BB8000080AC0F814A080ED068A059ACCED079A41
:10BB900048460099FCF782FCFEF7A2BAE17800293A
:10BBA0003EF4A5AEDBF8D43F0898DBF8D85F076811
:10BBB0001A9703EB83020BEB820670360FCE05EB70
:10BBC000850C0BEB8C0570350FC5012331681A9E6F
:10BBD0002960CBF8DC6F8BF8E43F002E00F0468143
:10BBE000089807681897189A961BB6F5C87F40F210
:10BBF0003D81E06A216BDBF83070DBF83430DBF834
:10BC00003850DBF83C60D8ED001AD4ED109A98ED6E
:10BC1000015A94ED119AD8ED026A94ED126A3A1A1B
:10BC20005B1A676BA16BE81B1343DBF84050721A79
:10BC3000E66B034313430020A91B43EA010671EEA0
:10BC4000E98A35EE49AA36EEC68A8BF8E40FCBF8BE
:10BC5000DC0FCBF8E00F8BF8D00FDBF858309BF8F7
:10BC60000450FEF77FBE002643F61D5784F8C060DF
:10BC70001BF8070000283EF4C2AC9BF80450DBF828
:10BC8000E83F5F1C00F0C281DBF83010E26A8A1ADC
:10BC900026D003EB8300E76C059B860006F1300E8F
:10BCA000781C9E4400F01182059807EB870600EB94
:10BCB000860E01210EF1300E84F85010DEF800706F
:10BCC00040F6FE7C3A446245D4BF22EAE27240F676
:10BCD000FF72CEF80020DBF8E83F581C00F010841B
:10BCE0004FEA830E0EEB03020BEB820643F608517C
:10BCF00096F870005BF80170DBF84020002840F0F7
:10BD0000268104208446D61B0CD0059F0EEB030130
:10BD100007EB81022032D1780E44664540F3BB81A7
:10BD20000020D0700EEB03060BEB860CBCF8707095
:10BD3000B7F5807F05D0DBF83C10A26B8A1A40F083
:10BD40001284DBF83810606B0A1A40F07881DBF857
:10BD50003460216BB6EB010C40F03281DBF830200F
:10BD6000E76AD61BDBF85C30002B40F0F38043F62B
:10BD700020505BF80070791C00F0D6830BF57452EC
:10BD8000D2ED052A98ED027A37EE628AB7EE003AD4
:10BD9000F0EEC83AF4EEC33AF1EE10FA05DD089F72
:10BDA00039681591159F4BF80070089B186814901E
:10BDB000149940F2DC5ECA1B724500F238810137EB
:10BDC00018BF0127606BDBF83C30A16BDBF8382033
:10BDD00098ED004AD4ED104AD8ED01AA94ED11BABD
:10BDE000121A581ADBF84030E16B10435A1A02431A
:10BDF00041F22400164346EA0C060BF8007074EE7C
:10BE0000648A3AEECBAADBF85830FEF7ABBDDBF81C
:10BE10003070E26ADBF83400266BDBF8385098EDBE
:10BE200000CAD4ED10CA98ED010AD4ED110AD8ED7C
:10BE3000027A94ED121AB91A626BDBF83C70831B1C
:10BE4000AE1AA56B41EA030040EA06037A1BFEF72F
:10BE50007DBD9BF8AC7027B99BF8AD70002F3EF408
:10BE6000BFAB002B3FF406AFFEF7BABBDBF8E05FD9
:10BE7000002D3EF448AD08990B6817931798471B9F
:10BE8000B7F5C87F3FF6B5AEFEF73DBD4FF4804233
:10BE9000C84808F0B5FA9BF8D03F0BF5735008304E
:10BEA000032B00F25183DFE813F01B00F200EE00D9
:10BEB0000400089B41F208011C681C941C9A5BF862
:10BEC0000160951BB5F5FA7F80F080839BF8D13F28
:10BED000002B40F07B830BF5805C01268CF8006022
:10BEE0000599F9F71DFB9BF8D05F032D00F05B84EB
:10BEF0000BF55F564FF4005272643436304615210C
:10BF0000F6F72AFD30460021F6F726FD30463F21A0
:10BF1000F6F722FD30467521F6F71EFD304600216A
:10BF2000F6F71AFD0BF5BB5530467F211835F6F7AD
:10BF300013FD2846F7F7C6FAFEF7D3BD2D22B1EE62
:10BF4000488A8AF800200DF17D05FFF7ACBB03207D
:10BF50008446D8E6DBF83870626BDBF83C30A16BC6
:10BF6000D8ED02BA98ED00CAD4ED10CA98ED010AD6
:10BF7000D4ED110AB81A5A1AE76BDBF840301043B7
:10BF8000DF1B0BF5745E3843DEED057ADBF85830C5
:10BF9000064346EA0C063BEEE78A7CEE6C8A30EEFE
:10BFA00060AAFEF7DFBC089DDBF8DC6F2F681997ED
:10BFB0001999CBF8E01F4FF0010E8BF8E4EF0CE677
:10BFC0009BF80500002840F0BD8067460EEB03009B
:10BFD0000BEB800EDEF87C103944622900F3BB8243
:10BFE00011F1620FC0F2D683133304EBC307CEF80E
:10BFF0007C107960002940F02285002104EBC30306
:10C00000DBF830601972E06A361AABE6E76C7E1C2A
:10C0100000F07682DBF83020E36AD21A7FF444AE77
:10C02000DBF83410236B1646C3EB010C9AE643F69B
:10C0300020574FF0FF334BF807300027C2E69BF83C
:10C0400006603EB143F68857012102EB82020BF8ED
:10C0500007108A400EEB030C0BEB8C00866F32440A
:10C06000622A40F39280002663220EEB030C03F158
:10C070000B010BEB8C0004EBC10782677A6004EBC9
:10C08000C102167263E60599FAF768FC2BE7059979
:10C09000F9F796FE27E7002EFFF643AEF0B2D07018
:10C0A00040E6A679002E7EF4BDAAE76C002F40F38F
:10C0B000628401254FF0FF30CBF8D47FCBF8D86FE6
:10C0C0008BF8D05FE064FEF7ADBA5E44002D00F05F
:10C0D000A783D6F8800000282FDBB0F5007F40F35F
:10C0E000D884B0F5806F40F3CF84B0F5C06F40F3D3
:10C0F000C684B0F5006FC0F2BD8440F2FE7C60459E
:10C100001BDDB0F5206FC0F2B08440F6FE1188420E
:10C1100013DDB0F5406FC0F2A38440F6FE37B8429D
:10C120000BDDB0F5606FC0F2968440F6FE53984286
:10C1300003DDB0F5805FC0F285840022012784F81A
:10C14000BE70BBE543F68B5101260CEB8C020BF85D
:10C15000016002FA06F739E7E06C471C3EF422AAB8
:10C1600000EB80070BEB870797F87070002F7EF4C9
:10C1700019AA4FF4717707FB00B0012780F8787493
:10C18000284684F85170FEF711BA002A40F3BC83A8
:10C1900001266AE7002D7EF432AA6579002D3EF46F
:10C1A0002EAA41F2240386F001060BF80360FEF785
:10C1B00026BA00BF4034FF1FDBF860703D44062DF7
:10C1C00000F3D483DD4925EAE57501EBC50C2E4665
:10C1D0009CF80400DA4ACBF8605043F6080701EBFC
:10C1E000C60ED055E76ADBF83050206B9EF805602C
:10C1F000D8ED008A98ED019A98ED026A94ED105AF4
:10C20000D4ED116A94ED128AED1BDBF8347043F61D
:10C210000901381A45EA000743F60A0CDBF83850E2
:10C22000606B5654012602F80C602D1ADBF83C2096
:10C23000A06BDBF840103D43161A2E43CB1A1E4369
:10C240009BF80450DBF8583078EEC58A39EE66AAC0
:10C2500036EE488AFEF786BBDBF85870DBF83020F4
:10C26000DBF83400D8ED005A94ED102AD8ED012AFD
:10C2700094ED117A98ED023AD4ED123A2F44042F3E
:10C28000CABF052327EAE7771F46CBF85870E16A53
:10C29000266BD8BF3B46571A3D43DBF83820676B07
:10C2A000811BA66BDBF83C000D43D21B2A43851B88
:10C2B00042EA050675EEC28A32EEC7AA33EE638AF9
:10C2C0009BF80450FEF74EBBDBF86C10DBF83060D7
:10C2D000DBF8343098ED00CAD4ED10CA98ED010AAD
:10C2E000D4ED110AD8ED027A94ED121A29440029EE
:10C2F000D4BF00210121CBF86C10E26A206BB11A87
:10C300000D43DBF83820616B1E1AA06BDBF83C3064
:10C310003543521A2A431B1AFEF718BBDBF85C00A0
:10C3200098ED00CAD4ED10CA98ED010AD4ED110AB7
:10C33000D8ED027A94ED121ADBF83060DBF8343075
:10C3400028440028D4BF00200120CBF85C00D4E7AB
:10C3500004EE105A9FED7BAADBED15AAF8EEC44A55
:10C36000F1EE04BAE4EE8AAAF4EEEBAAF1EE10FACA
:10C3700008D5F7EE00BAF4EEEBAAF1EE10FAC8BF5A
:10C38000F0EE6ABAE66ADBF83010DBF83420DBF84E
:10C390003830CBED15BA881B216B98ED00CAD4ED6F
:10C3A00010CA98ED010AD4ED110AD8ED027A94ED85
:10C3B000121A561A626BA16B0543DBF83C009B1AFC
:10C3C00035432B43421AFEF7C1BA4FF0FF31E16407
:10C3D000FEF7B4B89BF80570002F3EF479A9627897
:10C3E000002A7EF475A9BEF1000F3EF471A9FEF794
:10C3F00063B99BF8045022B9A27812B1002184F8E5
:10C40000BC10BEF1000F7EF45AAAE07800283EF47A
:10C4100056AAFEF750BABEF1000F7EF450AAFEF7FE
:10C420000BBA9BF80E20002A3EF486A9A67A002EAD
:10C430007EF482A903EB83050BEB850C9CF873005B
:10C44000042800F08582002A3EF476A99CF870103A
:10C45000B1FA81F256098CF87060FEF76DB90121CE
:10C460008BF84610FFF75FBA4FF0010C8BF845C010
:10C47000FFF745BA01218BF84810FDF7D6BE667A62
:10C48000002E3EF40CA994F8507037B9032B0CBF62
:10C490004FF0FF330323CBF8E83F002584F85050DA
:10C4A000FEF7FDB8002A7EF4CFA8E76C002FC0F29B
:10C4B0003982012F00F0368201204FF0FF32CBF895
:10C4C000D47FCBF8D80F8BF8D00FE264FEF7BCB85E
:10C4D00000297EF4CCA8E56C002DC0F20782022D65
:10C4E00000F0048202224FF0010E4FF0FF31CBF832
:10C4F000D45FCBF8D82F8BF8D0EFE164FEF7B7B854
:10C50000DBF83000E76ADBF83420216BC61BC1EB97
:10C51000020C27E401238BF84830FFF733BA0122DD
:10C520008BF84720FFF717BA0BF5745EDEED055A5E
:10C5300098ED022A1F4632EE658A43E44409020060
:10C540004874FF1FCDCCCC3D40F2F312B049B14846
:10C55000F4F77EFEC7E4133304EBC3076326CEF87B
:10C560007C607E6049E59BF8070038B143F6895648
:10C57000012702EB82020BF80670BA400EEB0301B2
:10C580000BEB810CDCF874000244622A00F3378163
:10C5900012F1620FC0F2AE8103F10F0104EBC1068C
:10C5A000CCF874207260002A40F0FE81002704EB72
:10C5B000C10C8CF80870FFF7C4BB9BF806209BF8F1
:10C5C0000F0000283EF4D5A8FEF7BFB8089CDBF8A2
:10C5D000600021681B910428DBF8F03F8E4D1B9C06
:10C5E000B4BF0027FF27A4EB03043946B4BFFF23E1
:10C5F000002380222846009307F002FF3946874F28
:10C60000802205F1800007F0FBFEA7FB0420C0F3A9
:10C610008601C0F346239DF800206A54CBF8FC1F26
:10C62000CBF8F83F089F38680F900F998B1BB3F534
:10C63000FA7F7FF65DACDBF8FC4F0BF580571CB141
:10C640003E78002E00F0B480DBF8606072484FF452
:10C6500080420BF55F55032ECCBFFF21002107F070
:10C66000CFFE4FF400506864343528461521F6F7A4
:10C6700073F928460021F6F76FF928463F21F6F7AF
:10C680006BF928467521F6F767F90BF5BB54284678
:10C690000021F6F761F918347F212846F6F75CF996
:10C6A0002046F6F70FFF00213970FEF71ABABEF1E7
:10C6B000000F10D1E67876B1A57B65B994F8BD007E
:10C6C00048B903EB830C0BEB8C014A6F002A40F056
:10C6D0006D8163224A6797B9617881B1257B75B90D
:10C6E00094F8BF605EB99D00E8180BEB800CDCF895
:10C6F0007C20002A40F061816325CCF87C509BF8B7
:10C700000620002A7FF45BAFA678002E3FF457AFD7
:10C71000617B00297FF453AF94F8BC0000287FF4BC
:10C720004EAF4FEA830C0CEB03050BEB8500816FDA
:10C73000002900F08281632900F06D811146634475
:10C740000BEB830399673AE7002A3FF455AEFEF7F7
:10C75000B6B8DBF83060E26ADBF83430216B98ED74
:10C7600000CAD4ED10CA98ED010AD4ED110AD8ED33
:10C77000027A94ED121AB01A0543DBF83820606B88
:10C780005E1ADBF83C30A16B3543121A2A435B1A60
:10C79000FEF7DCB8133304EBC3006FF06202CEF88F
:10C7A0007C20426029E441F208045BF8046039E728
:10C7B0009BF8F85F681CC1B24B1B0BF55F549A01E4
:10C7C0006264343420461521F6F7C6F83146204617
:10C7D000F6F7C2F820463F21F6F7BEF8204675214D
:10C7E000F6F7BAF829462046F6F7B6F82946204665
:10C7F0000BF5BB551835F6F7AFF8FFF79ABB03F109
:10C800000F0104EBC1066327CCF874707760CDE6A6
:10C81000A0250200540102004034FF1F4FECC44E1B
:10C820009E4FD6F8806007F1E00C394651F8040BB2
:10C83000864203DB7B689E4240F3A0800868864204
:10C8400003DB4B689E4240F399804868864203DBD5
:10C850008B689E4240F392808868864203DBCB68F7
:10C860009E4240F38B80C868864203DB0B699E4280
:10C8700040F384800869864202DB4B699E427DDD7D
:10C880004869864202DB8B699E4277DD8869864271
:10C8900001F11C0702DBCB699E426FDDBC45C4D1B0
:10C8A0000022FFF70BBA7E4E7E4D8BF8D07F0FCE65
:10C8B0000FC596E80F0085E80F00A5F11C02394668
:10C8C0000123A2F13400FCF7E9FF0BF1C0010BF5E5
:10C8D0007D6C61453DF417AE4FF0010E81F899E390
:10C8E00001F571718C45F9D1FDF70DBE0220E064B0
:10C8F000FDF7BDBE03F10F0104EBC1006FF0620252
:10C90000CCF87420426051E603F10B0104EBC1073F
:10C910000022826716467A60FFF7B1BB0321E1640B
:10C92000FDF7BDBE0125E564FDF78EBE9CF87210D3
:10C93000B1FA81F256098CF872609BF80E5095B1ED
:10C9400018440BEB800C9CF8731004297FF47EAD27
:10C95000554D042085F84400FDF7EEBE9BF80E10FF
:10C9600000297DF4E9AEA67A002260E507264F494A
:10C9700035465F202EE4E664FDF754BE1E1A02FB26
:10C9800006F2FFF79BB9484E45F610451E20705140
:10C99000FDF7EFBE4FF0FF33CBF8E83FFDF73FBEAA
:10C9A000DBF8DC6FFFF719B9012700E6632A1CD01A
:10C9B00063320ED000224A678DE6632A26D012F138
:10C9C000630116D01D440BEB850C0022CCF87C20B3
:10C9D00095E60BEBC30643F64C55705D0028E9D095
:10C9E00043F6485576594E6775E66FF06200486722
:10C9F00071E60BEBC30143F66C56885D0028E1D06D
:10CA000043F668568959CCF87C1078E66FF06200DE
:10CA1000CCF87C0073E60BEBC30543F62C56AE5DF9
:10CA2000002E3FF48BAE43F62856AD598567622D34
:10CA30003FF785AE25EAE57181E663217FE60121B6
:10CA4000FFF7DCBA40F6FF7640F6FF50311A02FBE2
:10CA500001F2FFF773BB40F6FF5640F6FF30F5E7F3
:10CA600040F6FF3640F6FF10F0E740F6FF1640F2C2
:10CA7000FF70EBE740F2FF764FF4C060E6E74FF45B
:10CA8000C0664FF48060E1E74FF480664FF40070B9
:10CA9000DCE74FF400760020D8E700BFF001020089
:10CAA0009874FF1F54C6FF1F4874FF1F44090200FB
:10CAB0002DE9F04F6D4FDFF830E26D4E6D496E4D50
:10CAC0006E4A6F4CDFF8D481DFF8D8C100232DED1A
:10CAD000068B8EF800303B70402733700F70502665
:10CAE00070212E70117025686649674F674E45F0BA
:10CAF000406222600A68664D04F57E34814642F445
:10CB000000300860634AC8F8003087B0103409F577
:10CB1000A3413B604C314FF08077336092462B60ED
:10CB200000912360CCF800301760DAF80030594EDD
:10CB3000DD01FAD4009C584A40F2771565603068F0
:10CB400020F008013160376827F47F2B2BF47F6ECB
:10CB50004EF4612848F0E003336016683407FCD5D2
:10CB60004C4A4A4C13684D4F474E49484C494D4D2D
:10CB700043F00803136040F243433B6033604FF4DB
:10CB8000886704F5C82627602C3603600B60394897
:10CB900045492B60454C346060254FF400330570E7
:10CBA0000B60176847F00066166010680001FCD43F
:10CBB0000098FCF7C5FB18B948463D49FDF768F8F1
:10CBC0003C4FDFF808B1344E09F5A442BA4603924F
:10CBD00039493A4DD1F8008004F026F9044604E0C2
:10CBE00004F022F9001BA842F2D83368D907F7D421
:10CBF000334A3448C2F80080506004F015F92F4CD5
:10CC0000054604E004F010F9421BA242E0D839685E
:10CC10002D4B0B40002BF5D0DAF80000CBF80000CC
:10CC2000CAF80000DBF80020274D284C1540012DE4
:10CC3000CED127490B68DA05CAD5DFF8B0A0254860
:10CC40008AF80050002525601D4A039C224E234F80
:10CC500004604FF48131224B224815603160136328
:10CC6000386004F0E1F8154D044647E019E400E0AF
:10CC70004AE400E051E400E01CE400E027E400E0C6
:10CC800000D800403080044004D0044008D0044064
:10CC90000CD004402C100B4024100B4000D004405A
:10CCA00010D0044014D0044008E100E00B007F11D4
:10CCB0008C01020030100B40A0E0012040420F0028
:10CCC00008100B4000001A0D01000F0098E0012031
:10CCD00010100B4000100B4004100B400C100B40C8
:10CCE00002007F1137003A1218E400E09CE00120B6
:10CCF00004F09AF8011BA94200F293849AF80020EC
:10CD0000002AF5D1DBF80060A74F3740022F40F032
:10CD100088840398A54B05689D4200F08D8409F531
:10CD2000A4460C363746039CA14901964FF00008F3
:10CD3000012542F29E60052208262360A0606660FD
:10CD40002B467960BA60FD603D61C7F81480C7F872
:10CD50001880C7F81C80414622460098FCF79EFDCB
:10CD600000283FF429AF09F5A84308331C4645F2D3
:10CD7000084145F20C4245F2204E049345F21C470F
:10CD8000632345F21D4C49F8018045F21E4049F8E5
:10CD9000023045F21F41C4F80880E360C4F81080F7
:10CDA00045F2344649F80E3045F2304E09F8078016
:10CDB00045F2314209F80C8045F2324C09F8008006
:10CDC00009F8018045F23340C4F81C802362C4F89E
:10CDD000248049F8063009F80E8045F2484645F2AD
:10CDE000444E09F80280029509F80C8009F5A84222
:10CDF00045F2454145F2464545F2474C09F8008069
:10CE00006C4FC4F830806363C4F8388049F806304A
:10CE100009F80E80684E09F801804FF0000E09F8FD
:10CE2000058009F80C80A364C4F84480C4F84C80E1
:10CE3000C2F858E0C2F85CE0C2F860E0CDF81490A7
:10CE4000DFF8A8915D4B5E4DD3F8008003F0ECFF56
:10CE5000044604E003F0E8FF031BAB42F2D831685C
:10CE6000CB07F7D4574A5848C2F80080C9F80000E9
:10CE700003F0DAFF524C054604E003F0D5FF411BF6
:10CE8000A142DFD83968514B0B40002BF5D04948FF
:10CE9000484A0568CBF800501560DBF800404B4B62
:10CEA0004B492340012BCDD14A480568E805C9D537
:10CEB00000240C604849494A08788AF80030049BED
:10CEC0001360002840F09783029D6C0244493D4B5B
:10CED000444A4548454D1C600860334C4449146041
:10CEE000296003F0A1FF364D044605E003F09CFFE6
:10CEF000011BA94200F281839AF80020002AF5D193
:10CF0000DBF80000284B0340022B40F07683029DA3
:10CF100004357D2D029593D1DDF81490019ED6ED58
:10CF2000017AB7EE007AF4EEC77AF1EE10FA06D481
:10CF3000B1EE040AF4EEC07AF1EE10FA02DD019CC3
:10CF40001B4F6760019A019C9068D3681169194F63
:10CF5000194E052884BF05209060012B84BF012352
:10CF6000D36007294FF0000584BF0121116165617D
:10CF7000A561E5611148124DD0F8008003F054FF1F
:10CF8000044604E003F050FF001BA842F2D83368C7
:10CF9000DB07F7D40B4A0C49C2F80080516003F05C
:10CFA00043FF074C05462AE002007F114B45454EE2
:10CFB0000000204030100B4024100B40A0E0012066
:10CFC00040420F0008100B4000001A0D01000F0036
:10CFD00098E0012010100B408CE0012000100B4065
:10CFE00004100B4038100B40000204000C100B40E2
:10CFF00027003A1903F018FF421BA242BAD838683A
:10D00000154B0340002BF5D01449144A0D68CBF89A
:10D0100000501560DBF800400F4B11492340012BF5
:10D02000A8D110480568E805A4D58AF800300E4C50
:10D030000E4A0F4E0F4F104D00230B6003992160D5
:10D040004FF481300D4C1360306015633C6003F089
:10D05000EBFE0B4E07461BE001000F0030100B40AB
:10D0600098E0012010100B4000100B4008100B40FE
:10D0700004100B400C100B4002007F1127003A19DE
:10D0800040420F0003F0D0FEC01BB04200F2C2824B
:10D090009AF80030002BF5D1DBF80020E049114070
:10D0A000022940F0B782039DDE4E0C350FCD09F109
:10D0B000500401940FC495E80F0084E80F00D9F8DC
:10D0C0006070D94A06EBC70C43F6080309F5A15670
:10D0D0009CF80410D154083643F60A0543F6090EAD
:10D0E00000239CF8050096F8C48202F80E00012780
:10D0F00009F5B65457550C341D46C6F890322268CF
:10D1000048FA05FA204697680AF001010135B84748
:10D11000042D04F10804F2D196F814B0C348B469A0
:10D1200006EB8B0C4D21DCF80C20256801FB0B066F
:10D13000530996F843E09F0007F1604808F56146FF
:10D1400002F01F0A4FF0010B0EF01F0145F04005E1
:10D150000BFA0AF21F29256032600AD05FEA0E62DC
:10D160004ABFE668102626F0100641F04003E6604C
:10D17000236009F564572C373E7DD7F8A022BC699F
:10D1800007EB860E07EB82084FF04D0CDEF80C70B3
:10D19000D8F88C520CFB06007909465D25688B0097
:10D1A00003F1604A07F01F0C0AF5614B012206F0FB
:10D1B0001F0145F0400702FA0CF01F292760CBF849
:10D1C000000009D033064ABFE368102323F01003A0
:10D1D00041F04006E36026600A2003F049FEB9F8FA
:10D1E0002C40B9F82E50B9F82A209FED911A914998
:10D1F000DFF864B2DFF864E29FED8F5ADFED8F5AFB
:10D2000009F5715706EE104A06EE905A00EE902A84
:10D2100009F570552E46B84609F56F5409F5725A4E
:10D220005346383418353836F8EE602AF8EE461A88
:10D23000B8EE662A1C3708F138080AF1140A09F515
:10D240007B5C0022C4ED031AC4ED041A2260626103
:10D25000616084ED021AC4F818B0C4F81CE085EDD2
:10D26000032A2A60696085ED021A85ED042AC5F853
:10D2700018B06A61C5F81CE0C6ED032A326071601F
:10D2800086ED021AC6ED042AC6F818B07261C6F817
:10D290001CE0C7ED031A3A607960C7ED021AC8F8BE
:10D2A0000020C8F8041088ED032A88ED022ACAED90
:10D2B000032ACAF80020CAF80410CAED022AC3EDF6
:10D2C0000F2A1A635963C3ED0E2A5D4BCCF8283040
:10D2D00009F5795363456046CCF80020CCF804107A
:10D2E0008CED021ACCF80C20CCF81020CCF818B039
:10D2F000CCF81420CCF81CE0CCF82020CCF824107A
:10D30000CCF82C20CCF830208CED0D5ACCED0E5AF8
:10D3100018BFDC460DD01A60596083ED021ADA603E
:10D320001A61C3F818C05A61C3F81CE02033984250
:10D33000F1D1B9F81C20B9F81E10B9F82000B9F8DD
:10D3400022B09FED408ADFED408A9FED409A9FED2D
:10D3500040AADFED409A03EE102A03EE901A04EE85
:10D36000100AB8EE630A04EE90BAF8EE43AA09F583
:10D37000765EB8EE447A09F57C5109F5775BCEED1F
:10D380000DAACEED0CAA8EED5F8A8EED628ACEEDEF
:10D39000608A734681ED018AF8EE647A8BED060AA5
:10D3A0008BED050A8C4609F5775B83ED638AC3ED47
:10D3B000648A09F581528CED068A8CED058A8BED25
:10D3C0000F7A8BED0E7A09F57C5C09F5785B83EDBD
:10D3D000678AC3ED688A8CED0A8A8CED098ACBEDE9
:10D3E000087ACBED077A09F57C5C02F1180B83ED26
:10D3F0006B8AC3ED6C8A5A468CED0E8A8CED0D8AD1
:10D400001E210098FCF798FB5946DDF804B05846F9
:10D4100002F046FC41F20603D4F810E020E000BF21
:10D4200002007F11440902004874FF1F903304007A
:10D43000BAE8144200F07F456666663F0B95813F6F
:10D440000000C8410000000000F07F4500A00C462D
:10D4500000007A4500409C460AD7233C87D4843F8D
:10D46000D5F810C0316909F57152002009F80300A0
:10D47000C4F80CE084ED058A09F5805385ED058A32
:10D48000C5F80CC0F16086ED058A156BB9F82C6003
:10D490009D6109F5725E09F57251DEF80CC0C3F8A2
:10D4A0001CC006EE106A886A1862B8EE460A20466A
:10D4B000DD68F3F703FFB9F82EC087ED030A06EE27
:10D4C00090CA09F5715609F5805387ED008AC7EDBA
:10D4D000018A04F120007562B8EE660A1F69F3F74D
:10D4E000EDFEB9F82A1088ED030A09F5725200EE34
:10D4F000901A09F5805588ED008AC8ED018A04F17B
:10D5000040001760B8EE600A6C69F3F7D7FE09F5C2
:10D51000725809F5B84509F5645709F563568AED5F
:10D52000030A8AED008ACAED018A1735C8F81C4043
:10D5300004373C364C46DA4694F8733015F8010F40
:10D5400098424CD094F87020002A3AD157ED025AF4
:10D55000307A032BB8EEE55A3ED025EE290A03F0C7
:10D5600021FB7268307A0121914001EBD17359108F
:10D5700003F00EF994F87300287094F872202A7260
:10D5800094F8701029711434A24507F10C0706F1C4
:10D590000C06D1D141F29805AB4F59F80520AB48A4
:10D5A0009668AB4946F001034FF080754FF0805408
:10D5B00093603D603960046007B0BDEC068BBDE848
:10D5C000F08F17ED021A94F87230307AB8EEC15A23
:10D5D00013B925EE0A0AC2E725EE090ABFE795F856
:10D5E00008B094F8721094F870208B45ACD128796B
:10D5F0009042A9D1C7E7029C68E44FF4027233213C
:10D60000009802F077FC00287FF481ACDDF81490DC
:10D61000FFF7D2BA4FF402723321009802F06AFC8D
:10D6200041E54FF4F4723121009802F063FC0028C8
:10D630003FF4C2AAFFF76DBB039CA26842F29E664C
:10D64000B24203D048468349FCF71CFC039F79682B
:10D6500009F5A446082906F10C0600F0F180039FA5
:10D660007D48BA6000240125082305217B603A46E5
:10D670007060B1602B46F56035617461B461F4612E
:10D68000214600980196FCF709F900283FF494AA76
:10D6900009F5A8420832049245F2084345F20C41CC
:10D6A00045F2204745F21C460295049D49F8034087
:10D6B00045F21D40632349F8013045F21E4CAC6031
:10D6C000EB602C6145F21F4E49F8073045F23448B3
:10D6D00009F80640049F09F8004045F2304645F23B
:10D6E000314245F2324145F2334009F80C4009F825
:10D6F0000E4045F2484CFC613B627C6249F80830C0
:10D7000009F8064045F2444609F8024045F2454E04
:10D7100009F8014009F5A84209F8004045F24645DC
:10D7200004983C6345F247487B63BC63002149F899
:10D730000C304A4F09F80640494E09F80E4009F8E6
:10D74000054009F8084083644464C464CDF814902B
:10D750009165D1651166DFF83C91424C424DD4F899
:10D76000008003F061FB044604E003F05DFB001B56
:10D77000A842F2D83368D907F7D43C4A3C49C2F8EA
:10D780000080C9F8001003F04FFB374C054604E059
:10D7900003F04AFB421BA242DFD83868354B0340F6
:10D7A000002BF5D02D492D4A0D68CBF8005015609F
:10D7B000DBF800402F48304920400128CDD12F4BC5
:10D7C0001D68EA05C9D500240C602D492D4A0B7847
:10D7D0008AF80000049810603BBB029D6C022A4945
:10D7E00022482A4A2A4B2B4D04600B602A4C2B49B5
:10D7F0001460296003F018FB1B4D044604E003F09D
:10D8000013FB011BA94212D89AF80020002AF6D176
:10D81000DBF80000204B0340022B08D1029D0435A9
:10D820007D2D029597D1FFF777BB029CD7E74FF488
:10D8300002723321009802F05DFB0028EED1E5E68C
:10D840000196FFF76CBB00BF00F0024000E100E072
:10D85000000100907C0102000000204030100B40CD
:10D8600024100B40A0E0012040420F0008100B40A4
:10D8700000001A0D01000F0098E0012010100B406D
:10D880008CE0012000100B4004100B4038100B40BE
:10D89000000204000C100B4002007F1127003A190F
:10D8A0002DE9F04F2DED048B044699B0454D65658B
:10D8B0000023632204F1C0074F26012104F60C4522
:10D8C0000520DFF804A101972660A065E1652166C7
:10D8D0006366A366E36684F8703084F8713084F878
:10D8E000723084F87330A367C4F8803084F88430D1
:10D8F00084F8853084F8863084F88730C4F88C301A
:10D90000C4F8943084F8983084F8993084F89A30C8
:10D9100084F89B30C4F8A030C4F8A8306267E2678E
:10D92000C4F888203E46C4F890204FF00008C4F8A0
:10D930009C20C4F8A42084F8AC3084F8AD3084F87E
:10D94000AE3084F8AF30C4F8B020C4F8B430C4F8B6
:10D95000B820C4F8BC3004F170070A95AB46002526
:10D9600029468022C6F88483C6F888A3C6F88C832B
:10D97000C6F89083C6F89483C6F89C83C6F8BC8327
:10D98000C6F8805386F8995386F8985386F8B853AA
:10D9900086F8B95386F8C053304606F031FD294663
:10D9A000302206F5007006F02BFD2946302206F5E0
:10D9B000307006F025FD5E454FF0000906D006F5F3
:10D9C0007176CCE70000204000005C4104F58050F7
:10D9D0000430029004F5805E0298019AC4F8DC5F7E
:10D9E00041F2040C04F581584FF0FF31C4F8E05FB8
:10D9F00084F8E45F84F8D05F84F8EC5F04F80C509E
:10DA0000C4F8D41FC4F8D81FC4F8E81F4570857047
:10DA10002946CEF80C90CEF81090CEF81490CEF89F
:10DA20001890CEF81C90CEF82090C8F814903D7055
:10DA30007D70BD70FD70BD603D61019DD61B07F11D
:10DA400014036322A6F1140A9D42CAF381067A6088
:10DA5000FA6058D0002E01F0AE87012E14D0022EAD
:10DA600009D0197059709970D9705A609960DA604C
:10DA7000196107F12803197059709970D9705A60AB
:10DA80009960DA60196114330198197059709970AE
:10DA9000D9705A609960DA6019611433984218BFDE
:10DAA000074630D0197059709970D9705A609960D2
:10DAB000DA601961197559759975D9759A61D961C5
:10DAC0001A62596283F8281083F8291083F82A1003
:10DAD00083F82B10DA6219635A63996383F83C1058
:10DAE00003F13C0B50339F428BF801108BF802106E
:10DAF0008BF80310CBF80420CBF80810CBF80C20DF
:10DB0000CBF81010CED1019904F57D67B94200F031
:10DB1000CB804FF000094FF000088E467E1ADFF8E8
:10DB200078A4C1F884830D46A6F5717C7046C1F8CF
:10DB30008C83C1F89083C1F89483C1F89C83C1F8A9
:10DB4000BC83C1F888A3C1F8809381F8999381F8C8
:10DB5000989381F8B89381F8B99381F8C0938022A3
:10DB60004946CCF3800606F04BFC4946302205F5C9
:10DB70000070019505F5717B06F042FC49463022A4
:10DB800005F5307006F03CFC5F4500F08D807EB3FB
:10DB9000CBF88093CBF88483CBF888A3CBF88C8325
:10DBA000CBF89083CBF894838BF899938BF8989368
:10DBB000CBF89C838BF8B8938BF8B993CBF8BC83E4
:10DBC0008BF8C09358468022494606F019FC019E06
:10DBD0003022494606F2C45006F012FC06F5F16BFD
:10DBE0004946302206F2846006F00AFC5F455BD0AD
:10DBF0000025CBF88483CBF888A3CBF88C83CBF8B3
:10DC00009083CBF89483CBF89C83CBF8BC83CBF880
:10DC100080538BF899538BF898538BF8B8538BF843
:10DC2000B9538BF8C05329468022584606F0E8FBCA
:10DC3000294630220BF5007006F0E2FB294630221F
:10DC40000BF5307006F0DCFB0BF571702946802275
:10DC5000C0F88483C0F88053C0F888A3C0F88C83D0
:10DC6000C0F89083C0F8948380F8995380F8985353
:10DC7000C0F89C8380F8B85380F8B953C0F8BC83CF
:10DC800080F8C05306F0BCFB294630220BF2C4508A
:10DC900006F0B6FB0BF28460294630220BF5F16BDF
:10DCA00006F0AEFB5F45A3D10298A74941F20407F5
:10DCB00041F2240200234FF0FF36E35504F5835967
:10DCC000C4F8DC3FC4F8E03F84F8E43F84F8D03F78
:10DCD00084F8EC3FC4F8D46FC4F8D86FC4F8E86F88
:10DCE00004F581584370837004F5825AA35441F2BD
:10DCF000380E41F24C0741F274026325C8F808104F
:10DD000004F80E3088F8193088F81A3088F81B307B
:10DD1000C8F82030C8F82830C8F81C50C8F824507B
:10DD2000E35504F584588AF80D308AF80E308AF8E5
:10DD30000F30CAF81050CAF81430CAF81850CAF890
:10DD40001C3089F8003089F8013089F8023089F8F0
:10DD50000330C9F80450C9F80830C9F80C50C9F8A4
:10DD60001030A35489F8153089F8163089F8173027
:10DD7000C9F81C30C9F82430744BC9F81850C9F8D8
:10DD800020500026724DC8F80860C8F80C60C8F82A
:10DD9000106003F5A07AA1461F6898685E689C69C8
:10DDA000196A9A6A05EBC70C05EBC00EDCF8047023
:10DDB000DEF804003E601F69DE68066005EBC70BF5
:10DDC00005EBC408DBF804705C693C60D8F804001B
:10DDD000DE69066005EBC1011E6B4C685F6A276057
:10DDE00005EBC20205EBC60C5068D96A9A6BDCF8E9
:10DDF000044001605E6B266005EBC20ED86BDEF856
:10DE0000047040339A453860C6D1524B524E19685F
:10DE1000524D534A41F400071F60306820F0020160
:10DE2000316041F298064FF4003749F806202F6020
:10DE300095684C4845F002014EF6602691601660E8
:10DE40001A684FF0804742F400451D604C468246F8
:10DE50000760DAF80030002BFBDB434A4349DFF868
:10DE60003C91DFF83CB1DFF83CE1414EDFF838810E
:10DE7000404F4148414B424D4FF24F0CC2F800C059
:10DE80004FF0010A00220A60C9F800A004F585518C
:10DE90004FF440390B91CBF80080CEF8009041F25E
:10DEA000AC0B376041F2A808364EDFF800C10560C0
:10DEB000D6F834E0344F354D81E8180044F80B2093
:10DEC00044F808C0D6F830B0DEF80000B36B304933
:10DED00004F58556103604F5865C41F2B00903431B
:10DEE000022044F809103273727332613071CCF839
:10DEF0004420CCF84820CEF80030C6F808B08BF8A3
:10DF00000020B3685A70B1688A70B368FF20D87077
:10DF1000B1684A71B36850209871B168CA71B0682D
:10DF200090F8028008F07F038370B1689646122251
:10DF3000CA70D346F446F0464FF0FF31154A0BFA4B
:10DF40000EF90020CEE000BF000080BF24E00100F9
:10DF5000103504003C8004400070034004E100E000
:10DF60001071034000F1024004F1024060F00240F1
:10DF700010F00240130F010014F00240F480010081
:10DF8000000F0F0F2C340400008793039F860100BD
:10DF90008C8001008A34040000005C4104F00240DF
:10DFA00008F002400CF0024003000007990E000048
:10DFB000CAF5C333A0338B4202D21946F0468446D9
:10DFC000B2F802A009FB0AF3B7FBF3FAAA4500F185
:10DFD000010000F29E80CAF5C333A0338B4202D207
:10DFE0001946F0468446938809FB03F3B7FBF3F325
:10DFF000AB4200F1010A40F29880A3F5C333A03B85
:10E000008B4205D2D446F046002B00F0CE80194654
:10E01000D38809FB03F3B7FBF3F3AB4200F1020A29
:10E0200040F28D80A3F5C333A03B8B4205D2D4468A
:10E03000F046002B00F0B9801946138909FB03F361
:10E04000B7FBF3F3AB4200F1030A40F28280A3F581
:10E05000C333A03B8B4205D2D446F046002B00F0E0
:10E06000A4801946538909FB03F3B7FBF3F3AB42D2
:10E0700000F1040A76D9A3F5C333A03B8B4205D245
:10E08000D446F046002B00F090801946938909FB96
:10E0900003F3B7FBF3F3AB4200F1050A6BD9A3F529
:10E0A000C333A03B8B4204D2D446F046002B7CD035
:10E0B0001946B2F80EA009FB0AF3B7FBF3F3AB4223
:10E0C00002F10E0200F1060A5ED9A3F5C333A03BAC
:10E0D0008B4204D2D446F046002B66D01946073056
:10E0E00040285CD0B2F802A009FB0AF3B7FBF3FAB0
:10E0F000AA4502F102027FF65BAFAAF5C333A03B4B
:10E100008B42BFF45DAFF0468446002B4DD01946DC
:10E1100056E7AAF5C333A03B8B42BFF464AFF04689
:10E120008446002B41D019465DE7C3F5C333A033C5
:10E130008B42BFF46DAFD4461946F04668E7C3F58D
:10E14000C333A0338B42BFF478AFD4461946F046B0
:10E1500073E7C3F5C333A0338B4283D2D446194649
:10E16000F0467FE7C3F5C333A0338B428ED2D4464B
:10E170001946F0468AE7C3F5C333A0338B4298D2E1
:10E18000D4461946F04694E7C3F5C333A0338B4217
:10E19000A5D207304028D4461946F046A2D1BEF198
:10E1A000020F02D00EF1010EC8E641F2B8050CF0E4
:10E1B0003F026159D94F42EA8810C3B24B70B2682E
:10E1C000DFF86C83507940F020015171B26892F809
:10E1D000059049F080035371B068D14B817841F0CC
:10E1E0008002827096F804A00AEB4A0C03EBCC0B79
:10E1F0004FF0010ADBF80C0041098A0002F1604986
:10E2000000F01F0004F5885E09F5614C0AFA00F27F
:10E2100041F21013C348CCF800200EF1100941F26E
:10E2200018118660F346E65004F5895E002341F23A
:10E230002412C9F8043044F8018006F16001CBF8DB
:10E240001C100691CEF800701946A35009F1180071
:10E25000402206F0D5F8382289F85A206559A87866
:10E2600000F0BF03AB70D9F8040086F80DA058B1D8
:10E270000268AD4955688D4209F1080241F08C836E
:10E2800040680221F3F740F904F58B50834641F2D0
:10E290006C1C0C3041F2741599F858A004900022BF
:10E2A00089F859A004F58C5344F80C6041F27C1EA7
:10E2B000426044F80580049D06F1BC00CBF81800CC
:10E2C000114644F80E7081461A6005F1180040228C
:10E2D00006F096F841F2B80A4FF0390C85F85AC0AA
:10E2E00054F80A20937803F0BF0090706868012109
:10E2F0002A46717358B103688B4D5B68AB4202F1DB
:10E30000080241F04E8340680221F3F7FDF804F55E
:10E310008E5B04985A46083290F858A080F859A0AD
:10E32000154641F2C81341F2D01E002141F2DC1023
:10E3300041F2D812E650696044F80E8006F58C78F8
:10E34000CBF814802150A75004F58F50402205953A
:10E35000CDF80C8006F054F805983A2741F2B80B36
:10E3600080F85A7054F80B20937803F0BF0595702D
:10E37000024640680127777358B106686A49736896
:10E380008B4202F1080241F0118340680221F3F749
:10E39000BBF8059D049995F858B041F2242004F586
:10E3A000915244F8009041F22C270398906000238A
:10E3B000142692464FF4FA755C48166155619361D4
:10E3C000D36182F8203082F82130E0514FF002070B
:10E3D000CAF8249082F82870484604F5965791F9B7
:10E3E0005990DFF850A10C3704F597514D46079727
:10E3F00001F10C0704F59259394665F003070897B7
:10E400004FF4FA77C9F814704BF00F0B41F24C2718
:10E41000464DCDF824B002F10C0B04F59358C9F821
:10E4200018B0C9F81060C9F81C3089F8203089F894
:10E430002130E551C9F8240007464FF0030089F860
:10E44000280002F12C09C8F8189041F26C294FF409
:10E45000FA70C8F81060C8F81400C8F81C3088F8C2
:10E46000203088F8213044F809504FF0040988F82A
:10E47000289004F5945C41F28C29C8F824704FF47C
:10E48000FA7002F14C08CCF81060CCF81400CCF80B
:10E490001C308CF820308CF82130CCF8188044F8EF
:10E4A00009504FF005098CF8289004F5955E41F26B
:10E4B000AC29CCF824704FF4FA7002F16C0CCEF851
:10E4C00018C0CEF81060CEF81400CEF81C308EF8CC
:10E4D00020308EF821304FF0060C44F80950079D8B
:10E4E000CEF824708EF828C002F18C0EC5F80CE02E
:10E4F0004FF4FA7041F2CC2EA8604FF0070C0B4895
:10E500006E602B612B756B7544F80E00AF6185F85A
:10E510001CC09DF82090049F08460DE0FD080000F7
:10E520002C3404007CE00120F5190000C8800100B3
:10E53000BC800100ACE0012087F8599002F1AC05E5
:10E5400041F2EC27CD604E60C84D03614FF4FA7183
:10E5500081600375437504F5985BE551039D856102
:10E56000037702F1CC0141F20C374FF4FA70CBF88B
:10E570001810CBF81400BD49CBF810604FF0010023
:10E58000CBF81C308BF820308BF8213004F59958EB
:10E59000E151CBF824508BF8280041F22C3B02F1DA
:10E5A000EC014FF4FA77B148C8F8181004F59A59FD
:10E5B000C8F81060C8F81470C8F81C3088F820300B
:10E5C00088F821304FF0020144F80B0041F24C3B37
:10E5D00088F8281002F586704FF4FA77A349C8F836
:10E5E0002450C9F81060C9F81470C9F81C3089F8B3
:10E5F000203089F82130C9F8180044F80B1005992B
:10E600009DF82480C9F8245002F5967004F59B5EAD
:10E6100041F270364FF0030789F8287081F859806D
:10E62000C2F84C010698A051CEF81450DAF8005008
:10E630000D95DDF83490DAF800600E96DDF838803C
:10E64000DAF800700F97DDF83CB0DAF8001010919E
:10E6500004F59C55109F069741F2783E2A4604F532
:10E660009E57DAF80010049504F59B5618320837C7
:10E6700044F80E001191049205974FF00207377786
:10E68000C6F8249041F2983741F2883604F59D513E
:10E69000A051C5F8148085F80CC0E051049FDDF846
:10E6A0004490C7F80CB041F2A83641F2B8384FF0A8
:10E6B000060B87F804B00A46A05141F2C835069E01
:10E6C0004E614FF005070F7344F80800C1F824901D
:10E6D0004FF0040111776051DAF800501295DDF81F
:10E6E00048E0DAF800601396DDF84CB0DAF8007014
:10E6F0001497014605984FF00102027104F5A057E6
:10E70000149ADAF80000049215903A460837159DDD
:10E71000DAF80060079741F2D838059F169604F59D
:10E720009E56C7F80CE044F808104FF0030131770B
:10E73000169F0695DAF80010C6F824B004F59F5528
:10E7400041F2E83917914FF00406039944F8091093
:10E7500028462E7341F2F838049E6E61069E44F8F6
:10E7600008100597466241F2084E079E41F218478D
:10E770004FF005050577059844F80E104FF0060593
:10E780003571F06041F2B80AE15182F81CC054F8CA
:10E790000AC03749179F576204F5A1559CF806E057
:10E7A000344E354F354A03C9083541F228484EF0FA
:10E7B000040A05F1040B8CF806A044F808608BE805
:10E7C00003002F4803C805F10C0989E803003968E4
:10E7D000C5F8843241F000604FF001062E75C5F88F
:10E7E0008832AA6138609368264F23F00C017D605F
:10E7F0009160966846F004009060536A43F0040705
:10E800005762516A21F003065662506A40F00103D4
:10E810005362D76847F00801D160966846F003005C
:10E820009060936843F020079760D16841F0040638
:10E83000D660106A10F0400004F1140104D0136A8D
:10E8400023F04007012017620C4A566A46F0C003C5
:10E850005362576A094E3F06FBD4736A336918B195
:10E86000306A40F040023262044B0DE0C880010083
:10E87000BC8101007C8001003080044000B00B406E
:10E88000C481010074DF0120AE48D3F84CC09E6CF7
:10E890005A6CD3F840E0DF6BDFF8D0826644164450
:10E8A00076449A6B3E443244560846F40042DA629B
:10E8B000D3F86CA09E6E5F6E564437441E6ED3F83C
:10E8C0005CB03E449F6DB344BB4493444FEA5B0746
:10E8D00047F4004C41F22847C3F830C004F5B5595D
:10E8E000E05141F2BC630020C5F890024FF0100BDC
:10E8F00004F5B6564FF0110E13204FF0120AC5F86A
:10E900008C120C3644F803B0C9F820E0C9F8240092
:10E91000C9F828A041F2CC698B4944F8091004F5E4
:10E92000B652C6F804B0134641F2D46C41F2DC6B27
:10E9300004F5B75744F80C100437C2F818E044F84F
:10E940000B1041F2E462186243464345A150C7F8F8
:10E9500004A04FF001010BD1307902F029FAB7423F
:10E960000BD056F8080F036843454FF00101F3D070
:10E97000012130469847B742F3D1D5F88C62DFF8D1
:10E98000F081DFF8F0C1D8F80000C5F8C862B31C08
:10E99000371DC5F8D032C5F8D872B11D06F108028E
:10E9A00006F10C0306F10E07C5F8E012C5F8E822DF
:10E9B000C5F8F832C5F8007306F10A0E06F1100129
:10E9C00006F1120206F1140906F1160306F11A0700
:10E9D0001836C5F81023C5F82033C5F82873C5F8D4
:10E9E00030630322042705260723C5F8DC22C5F877
:10E9F000E472C5F8EC62C5F8FC324FF0020B092254
:10EA00000A260B230C27C5F8F0E2C5F80813C5F851
:10EA1000D4B20021C5F80423C5F80C63C5F81C3333
:10EA2000C5F8247304F5BB534FF0010A4FF0080BEF
:10EA300040F480604FF0060E0D2232260027C5F804
:10EA40001893C5F8C412C5F8F4E2C5F814B3C5F8B4
:10EA50002C23C5F8CCA2C3E90067C8F80000DCF895
:10EA60000000DFF81491394F394E08F5012540F0C8
:10EA70000072CCF8002005F6DC78364A364DC9F82D
:10EA8000001047F6FF70C8F800004FF0280CD0695E
:10EA9000C7F800C0D2F818E0C6F800C0C5F800B04A
:10EAA000156A0768D96004F55D52383243F278760A
:10EAB00004F55E5B19615961234BA3513D435160DD
:10EAC0000392264ACBF800208BF80C108BF80D101F
:10EAD000CBF81010CBF85410CBF858108BF804A0DA
:10EAE0000560CBF808E08EF80010DBF808001C4E3B
:10EAF0004170DBF808301B4D9970DBF80820FF20CF
:10EB0000D070DBF808305971DBF808205020907184
:10EB1000DBF80830D971DBF80820907800F07F032B
:10EB20009370DBF808208E4612215F46D170D346E1
:10EB3000F046F4464FF0FF310B4A0BFA0EF9002075
:10EB4000C0E000BFD4800100A48001000CA00C40F4
:10EB500014A00C402C34040000A00C408C80010058
:10EB6000008793033F771B008A340400810E000066
:10EB70002C8004400480044004A00C40CAF5DB1A39
:10EB80000AF5BA53994202D919468446F046B2F8BA
:10EB900002A009FB0AF3B6FBF3FAAA4500F1010053
:10EBA00000F2A880CAF5DB1A0AF5BA53994202D9D5
:10EBB00019468446F046938809FB03F3B6FBF3F34A
:10EBC000AB4200F1010A40F2A280A3F5DB13A3F5EA
:10EBD000BA53994205D9D446F046002B00F0DE80A6
:10EBE0001946D38809FB03F3B6FBF3F3AB4200F1FC
:10EBF000020A40F29780A3F5DB13A3F5BA539942BA
:10EC000005D9D446F046002B00F0C8801946138978
:10EC100009FB03F3B6FBF3F3AB4200F1030A40F246
:10EC20008C80A3F5DB13A3F5BA53994205D9D446DA
:10EC3000F046002B00F0B2801946538909FB03F31C
:10EC4000B6FBF3F3AB4200F1040A40F28180A3F576
:10EC5000DB13A3F5BA53994205D9D446F046002BED
:10EC600000F09C801946938909FB03F3B6FBF3F38C
:10EC7000AB4200F1050A75D9A3F5DB13A3F5BA532E
:10EC8000994205D9D446F046002B00F087801946FA
:10EC9000B2F80EA009FB0AF3B6FBF3F3AB4202F1A4
:10ECA0000E0200F1060A67D9A3F5DB13A3F5BA53E8
:10ECB000994204D9D446F046002B6FD0194607304C
:10ECC000402865D0B2F802A009FB0AF3B6FBF3FABC
:10ECD000AA4502F102027FF651AFAAF5DB13A3F5B4
:10ECE000BA5399427FF653AFF0468446002B55D075
:10ECF00019464CE7AAF5DB13A3F5BA5399427FF600
:10ED00005AAFF0468446002B48D0194653E7C3F566
:10ED1000DB1303F5BA5399427FF663AFD446194625
:10ED2000F0465EE7C3F5DB1303F5BA5399427FF66D
:10ED30006EAFD4461946F04669E7C3F5DB1303F519
:10ED4000BA5399427FF679AFD4461946F04674E734
:10ED5000C3F5DB1303F5BA53994284D9D446194657
:10ED6000F04680E7C3F5DB1303F5BA5399428FD918
:10ED7000D4461946F0468BE7C3F5DB1303F5BA53C7
:10ED800099429CD907304028D4461946F04699D17B
:10ED9000BEF1020F02D00EF1010ECDE643F28879EA
:10EDA0000CF03F0254F80950E249DFF8A0B342EA00
:10EDB0008810C3B26B70BE68727942F02000707127
:10EDC000BD6895F805A04AF080036B71BE68DA4B08
:10EDD000B27842F08000B07097F804C00CEB4C059C
:10EDE00003EBC5080126D8F80C205009850005F171
:10EDF000604E02F01F0306FA03F20EF5614ACF4B94
:10EE0000CAF8002000255F60082039603D6687F859
:10EE10006450BD6601F0B2FA2946804601F090F8D0
:10EE2000B968C7F860808878C54ADFF824E300F045
:10EE3000FE038B70396E0879107097F804C0BE4AD3
:10EE40003B6E0CEB4C0A02EBCA081979D8F810009B
:10EE500001F1804C0CF5043300F03F0A4AF08002C7
:10EE60001D701A70386E97F80480B34B027908EB66
:10EE7000480103EBC10A02F1100C51118B00DAF8C2
:10EE800014104EF82C1003F1604E0EF5614802F09C
:10EE90001F02016806FA02F3C8F80030888B82B2BC
:10EEA00042F0080AA1F81CA0B1F81CC01FFA8CFEA1
:10EEB0004EF002038B8343F2F472A04904F55F58CD
:10EEC00004F5BB504FF03C0C4F6000F1180AA750FE
:10EED000039A88F840C00AF500534FF400571079A0
:10EEE000C8F83CA0C8F83830C8F84470314601F082
:10EEF0005FFFD8F83800036831469F68B847322072
:10EF000001F0B6FFD8F8380001688A6829469047B2
:10EF1000322001F0ADFFD8F83800036831469F6811
:10EF2000B84708F13408322001F0A2FF4046F3F759
:10EF3000A7FE42F2930042F2920154F809200AF827
:10EF400000600AF8015092F8069004F5605749F005
:10EF500007030C3704F5605A93710AF13C0804F575
:10EF60006159314638460222F5F760FA09F12C0959
:10EF70003D627D62BD62C7F82CB0404604F5625721
:10EF800006220521F5F752FA1C3704F5635AC8F832
:10EF90002050C8F82450C8F82850C8F82CB048466B
:10EFA00008220721F5F742FAD046C9F820500AF1A5
:10EFB0000C0AC9F82450C9F82850C9F82CB03846B2
:10EFC0000B221F21F5F732FA3D627D62BD62C7F860
:10EFD0002CB050461C221B21F5F728FA43F6FC0101
:10EFE00004274FF032090A22CAF82050CAF82450E8
:10EFF000CAF82850CAF82CB0384644F80190C8F82E
:10F000004420C8F8407001F0BDFD43F6FC0044F612
:10F01000206B235898F844000BFB03F100EE101A04
:10F02000B8EEC00A01F0BEFDD8F8402006FA02FC96
:10F030000CEBDC7131410A2001F0AAFB04F56458A5
:10F0400043F608104FF0030A44F80090C8F80C701B
:10F05000C8F810A0384601F095FD43F6081398F85B
:10F060001000E1580BFB01F200EE902AB8EEE00A26
:10F0700001F098FDD8F80C0006FA00FC0CEBDC71EE
:10F080003141504601F084FB04F5645843F61413F3
:10F090004FF01D0A44F803903846C8F81870C8F8B5
:10F0A0001CA001F06FFD43F6141198F81C00625883
:10F0B0000BFB02FC01EE10CAB8EEC10A01F072FDB2
:10F0C000D8F8180006FA00F303EBD371314150462B
:10F0D00001F05EFB04F5645843F620114FF0230A5B
:10F0E00044F801903846C8F8247043F62017C8F851
:10F0F00028A001F047FDE25998F828000BFB02F91F
:10F1000001EE909AB8EEE10A01F04CFDD8F8240027
:10F1100006FA00FB0BEBDB713141504601F038FB86
:10F12000084B094A04F5645793E803002C3743F66B
:10F130002C1C0FE0988001002C3404007CE001209E
:10F140001A800040BC8101007C8001000100008029
:10F150000002FF1F07F1040E44F80C208EE80300A4
:10F16000E149E24B03C907F10C0888E803001A687B
:10F170003D75C7F88452C7F88852DD4DDD48B86147
:10F1800042F000612F601960836823F00C058560F0
:10F19000826842F004018160436A43F004054562DD
:10F1A000426A22F003014162436A4362C56845F046
:10F1B0000802C260816841F003038360856845F0FE
:10F1C00020028260C16841F00403C360056A15F043
:10F1D00040021EBF026A22F040020262C548416A34
:10F1E00041F0C00308BF16464362456AC14A2B0678
:10F1F000FBD4536A13691EB1166A46F040001062D0
:10F20000DFF8F0A2DFF80093DAF84CB0DAF8482023
:10F21000DAF84430DAF84050DAF83C00DAF838101E
:10F22000B54E9FEDB68ADFF8E482DFEDB59A5A4419
:10F230001A442A4402440A44520842F40045CAF8D7
:10F240002C50DAF86CC0DAF86820DAF86430DAF8B2
:10F250006000DAF85C1062441A441044DAF858206E
:10F26000084400EB020E99E80F0075446D0843F660
:10F270002C1B45F40045CAF8305007F5237A04F5F5
:10F280006F5544F80B6043F6E43C00268AE80F0013
:10F2900043F6E8320B99C7F89C12C7F8A0620C231A
:10F2A00040F2DC5B974FC5F818801846EE612E627D
:10F2B00085ED048A85ED058A012144F80CB0A7503C
:10F2C000EB6201F075FDF7EE008A04F57051B6EEC1
:10F2D000009A2B4643F6584785F8346085ED0E8A30
:10F2E00085ED118A85ED128A85ED138AC5ED0F8AA9
:10F2F000C5ED158AC5ED109A85ED149A0A4681ED83
:10F30000068AC1ED078AC1ED089A81ED098A81ED6F
:10F310000C9A81ED0A8A81ED0B8AC1ED0D8A04F504
:10F32000715A383343F6744182ED0E8AC2ED0F8A6A
:10F33000C2ED109A82ED118A82ED149A82ED128A42
:10F3400082ED138AC2ED158AE35103F120020127F1
:10F3500004F5725ED4468AF82C708AED078ACAEDED
:10F36000088A8AED098A8AED0A8A625043F6904A31
:10F3700043F6AC4104F5735840338CED0E8A8CF89B
:10F380004870CCED0F8A8CED108A8CED118A44F810
:10F390000A3004F5745C8EED058ACEED068A8EED9A
:10F3A000078A8EED088A8EF8246063504FF0FF3391
:10F3B0008EED0C8ACEED0D8A8EED0E8A8EED0F8AC3
:10F3C0008EF8406008F168008CED038A8CED048AA9
:10F3D0008CED058A3146C8F85830C8F860302022D4
:10F3E00088F85C6088F85D6088F8646005F008F86B
:10F3F00008F188003146202205F002F809F1100BCF
:10F4000008F1A8003146202204F0FAFF9BE80F0023
:10F4100004F5765E0EF1200588F8CC7088F8C86097
:10F4200088F8C96088F8CA6088F8CB6085E80F0062
:10F430000EF1300009F12001902200F07FFE04F56A
:10F440007B5B04F5795304F57A5204F57C5904F595
:10F450007D5083ED008AC3ED018AC3ED029A83EDEE
:10F46000038A83ED069A83ED048A83ED058AC3ED52
:10F47000078A83ED088AC3ED098AC3ED0A9A83EDF2
:10F480000B8A83ED0E9A83ED0C8A83ED0D8AC3ED12
:10F490000F8A019982ED008AC2ED018AC2ED029ABB
:10F4A00082ED038A82ED069A82ED048A82ED058A56
:10F4B000C2ED078A82ED088AC2ED098AC2ED0A9A76
:10F4C00082ED0B8A82ED0E9A82ED0C8A82ED0D8A16
:10F4D0003830C2ED0F8A8BED008ACBED018ACBED7F
:10F4E000029A8BED038A13E0C48101003C80044042
:10F4F00074DF012000B00340E48001000000000040
:10F500000AD7233CA4800100CC810100000096436F
:10F510008BED069A8BED048A8BED058ACBED078A7D
:10F52000CBED0A9A8BED088ACBED098A8BED0B8A1D
:10F530008BED0D9A8BED0C8ACBED0E8A8BED0F8A3D
:10F54000CBED108A8BED118A8BED128A89ED038A3F
:10F55000C9ED048A89ED058A89ED068A89ED078A55
:10F56000C9ED088A89ED098A89ED0A8AC9ED0C8AF4
:10F5700089ED0B8A89ED0D8A89ED0E8AF7F700FD7A
:10F5800004F5874004F284417030F7F7F9FC04F584
:10F59000904004F648016830F7F7F2FC04F5994012
:10F5A0000A99B34D6030F7F7EBFC45F2581104F5BA
:10F5B000A242AF48665402F15C0EA968D0F804B0CC
:10F5C00045F25C130D46E654AA498EF80160A84B3B
:10F5D000DBF80020CEF8041004F5A2418A46186832
:10F5E000643145F264132A43A34DE5500E710E7346
:10F5F0004E730E61CAF8B860CAF8BC60CBF8002040
:10F600008860067088689D4A46708D689C4BAE7015
:10F6100088684FF0FF35C570886846718D68502046
:10F62000A8718D68EE71D1F8089099F8028004F500
:10F63000A24B08F07F0C5D4689F802C058358868F7
:10F6400003954FF0120A80F803A003980197043045
:10F650000EF108074FF0FF350597B146B04604900C
:10F660000198884F00FA06FA4FF0000C9CE0CBF5A9
:10F67000C330A030854202D90546B146E046B7F80E
:10F6800002B00AFB0BF0B2FBF0FB9B450CF1010C46
:10F6900000F2A180CBF5C330A030854202D90546E7
:10F6A000B146E046B8880AFB00F0B2FBF0F09842A1
:10F6B0000CF1010B40F29B80A0F5C330A0388542CD
:10F6C00005D9D846B146002800F0DE800546F88806
:10F6D0000AFB00F0B2FBF0F098420CF1020B40F292
:10F6E0009080A0F5C330A038854205D9D846B146F0
:10F6F000002800F0C980054638890AFB00F0B2FBFB
:10F70000F0F098420CF1030B40F28580A0F5C33075
:10F71000A038854205D9D846B146002800F0B4800B
:10F72000054678890AFB00F0B2FBF0F098420CF134
:10F73000040B79D9A0F5C330A038854205D9D84645
:10F74000B146002800F0A0800546B8890AFB00F009
:10F75000B2FBF0F098420CF1050B6ED9A0F5C33066
:10F76000A038854205D9D846B146002800F08C80E3
:10F770000546B7F80EB00AFB0BF0B2FBF0F098426A
:10F7800007F10E070CF1060B60D9A0F5C330A038C5
:10F79000854204D9D846B146002875D005460CF1FB
:10F7A000070CBCF1400F5ED0B7F802B00AFB0BF0BB
:10F7B000B2FBF0FB9B4507F102077FF658AFABF5B4
:10F7C000C330A03885427FF65AAFB146E0460028E4
:10F7D0005AD0054653E7ABF5C330A03885427FF6D3
:10F7E00061AFB146E04600284ED005465AE7C0F565
:10F7F000C330A03085427FF66AAFD8460546B14691
:10F8000065E7C0F5C330A03085427FF675AFD846B6
:10F810000546B14670E7C0F5C330A030854280D9B7
:10F82000D8460546B1467CE7C0F5C330A0308542D6
:10F830008BD9D8460546B14687E7C0F5C330A0301E
:10F84000854296D9D8460546B14692E7C0F5C33001
:10F85000A0308542A3D90CF1070CBCF1400FD8466B
:10F860000546B146A0D1022E0ED00136F8E600BF03
:10F870002C3404001D0D00008C80010000879303D0
:10F880009F8601008A34040045F26C1B08F03F0794
:10F8900054F80B5047EA8910C2B26A708E6896F825
:10F8A00005A04AF0200373718F68787940F08005D5
:10F8B0007D718A684148967846F08003937091F88C
:10F8C000048008EB480700EBC7090122D9F80C5067
:10F8D0006E09B30003F1604C05F01F070CF5614A97
:10F8E000374B059E02FA07F00025CAF800001E609B
:10F8F0008EF868508F68BD7000BF8868DFF8CC80D4
:10F90000304F039E3E60802383708868049B05709F
:10F9100054F80BE02C4F9EF80290DFF8B4A049F0A9
:10F92000400C8EF802C054F80BB0C8F8003002202A
:10F9300048739BF806E045F2741804F5A34304F5F8
:10F94000A8414EF007098BF806904C3344F8087034
:10F950000831B04645F2CC1C04F5A44B45F6104ED8
:10F9600045F614404FF0FF37029EC8F8706044F827
:10F970000C501D72DD601D745D748BF8042281F8DB
:10F98000042844F80E7027502046CAF8003019B0F9
:10F99000BDEC048BBDE8F08F11460222A847FEF7AC
:10F9A00073BC114602229847FEF7B1BC11460222F1
:10F9B0009847FEF7EEBC2F46FEF774B82C340400CF
:10F9C0007CE001204074FF1F5D8F000070DE01208D
:10F9D00094E00120104B30B50FCB85B08DE80F00BF
:10F9E00004206D4601F0CEF855F8044B9FED0B0A4C
:10F9F000E4B2204601F0D6F82046082100F0C8FE07
:10FA000004A88542F0D101210D2001F0D1F904486C
:10FA1000FDF74EF805B030BD7C82010000BADB482E
:10FA20004874FF1F554A564956482DE9F843136854
:10FA3000DFF8788123F0104444F2E43624F4807532
:10FA40000127156008F8067000F030FB44F2D8304A
:10FA50004D4B58F800E0D3F800909FED4C5ADFED85
:10FA60004C5ADFED4C4A44F2C81144F2D435A3F5A8
:10FA70008A620EF1940658F80110474B58F805C0F9
:10FA800002F58C6402F2544002EB8606002745E042
:10FA9000D0ED000ADFED416A9FED411AE6EE260A3D
:10FAA000F4EEC10AF1EE10FAA8BF70EEC10AC0ED83
:10FAB000000A013B2278D1ED031A3A4DA2B190ED34
:10FAC000002A75EE422AF4EEE52AF1EE10FA0BD880
:10FAD00032EE243A4FF0000C85F800C005ED033AF1
:10FAE000C6F800901746F44691F84020002A39D015
:10FAF0000025DFED2D3A81F840509FED284A9FED1B
:10FB0000286AE1EE843AF4EEC63AF1EE10FAA8BFA4
:10FB100073EEC63AC0ED003A013B26D0227891ED53
:10FB2000036A204DA2B1D0ED007A35EE677AB4EECB
:10FB3000E57AF1EE10FA0BD837EEA40A4FF0000C7C
:10FB400085F800C005ED030AC6F800901746F44694
:10FB500091F84020002A9BD00025DFED130A81F8A0
:10FB6000405097E7D0ED003AC7E70FB9BDE8F883FA
:10FB700044F2D43148F801C0F8E700BF00F0024079
:10FB80009C0102002029FF1F14B8FF1F33333346A6
:10FB9000B704CD4300003442A08601001F91EE3D22
:10FBA0000000804624B8FF1F000000004874FF1FBB
:10FBB00008B50648FAF75EFA02F0FCF800B908BD8D
:10FBC00002F0BCF8BDE80840FFF72CBF4874FF1FE7
:10FBD00070B50E4B0E4C0022802120460126FF25D9
:10FBE0001A605A60DA601A61DE621D729A621A75D2
:10FBF0005A759A61DA6119625962FDF751FE204621
:10FC0000044A0549BDE8704003F08CBA70D0FF1F6C
:10FC10004874FF1F8022FF1F110E000010B54FF423
:10FC2000007422460749084800F088FA224607492E
:10FC3000074800F083FA22460649074800F07EFA9A
:10FC400010BD00BFC0270200A0D4FF1FC0290200C2
:10FC5000A0D2FF1FC0250200A0D0FF1F10B54FF497
:10FC6000803422460449054800F068FA22460449D7
:10FC7000044800F063FA10BDC02B020070DE0020C3
:10FC8000C02B030070DEFF1F08B54FF4FA62024973
:10FC9000024800F053FA08BDC02B0400A0D6FF1F95
:10FCA000F0B50D4686460C460FCD0EF120060FC668
:10FCB00004F114070FCF2D6835600EF1340C04F1F8
:10FCC0002806ACE80F000FCE3F68CCF800700EF1AC
:10FCD00048050FC504F13C0C33682B60BCE80F00ED
:10FCE0000EF15C060FC6503494E807000EF6BC77A0
:10FCF000DCF80040346087E807007046F0BD00BFC4
:10FD000003680A6A9A4210B473D04FF0010C4B6B2F
:10FD1000426993425AD04FF0010C8C6C836A9C422A
:10FD200041D04FF0010CCA6DC46BA24228D04FF0F5
:10FD3000010C01F6BC7191ED007AD0ED147AB4EEAD
:10FD4000677AF1EE10FA17D190ED150AD1ED010A9C
:10FD5000B4EE600AF1EE10FA0ED190ED161AD1ED64
:10FD6000021A5DF8044BB4EE611AF1EE10FA0CBF02
:10FD700060464CF00100704701205DF8044B70476D
:10FD80000A6E036C9A42D2D14C6E426C9442CED130
:10FD90008C6E836C9C42CAD1CA6EC46CA24218BFDE
:10FDA0004CF0010CC5E7CA6CC46AA242B9D10A6D15
:10FDB000036B9A42B5D14C6D426B9442B1D18C6DBC
:10FDC000836B9C4218BF4CF0010CACE78C6B8369D1
:10FDD0009C42A0D1CC6BC26994429CD10B6C046A4A
:10FDE000A34298D14B6C426A934218BF4CF0010C6D
:10FDF00093E74C6A43689C4287D18A6A8468A2422E
:10FE000083D1CA6AC3689A427FF47FAF0A6B0469E0
:10FE1000B2EB040C18BF4FF0010C78E7F0B501F11C
:10FE2000200586460C460FCD76460FC604F13407F2
:10FE30000FCF2D6835600EF1140C04F14806ACE8C4
:10FE40000F000FCE3F68CCF800700EF128050FC5EB
:10FE500004F15C0C33682B60BCE80F000EF13C062B
:10FE60000FC604F6BC7494E80700DCF80070376035
:10FE70000EF1500585E807007046F0BD034B186889
:10FE800010B101680A681047704700BF74DF012095
:10FE9000034B586810B101680A681047704700BFEB
:10FEA00074DF0120034B186810B101680A6810471D
:10FEB000704700BF7CE00120034B586810B1016817
:10FEC0000A681047704700BF7CE00120034B986828
:10FED00010B101680A681047704700BF7CE001203C
:10FEE000034BD86810B101680A681047704700BF1B
:10FEF0007CE00120034600201972DA60704700BFE1
:10FF00000A4A0B4B0B480C4910B5002414601A68C0
:10FF100002601A600B6823B1186810B101680C68A0
:10FF2000A04706480022027010BD00BF38100B40E9
:10FF300030100B4098E0012094E001209CE001206B
:10FF4000F0B572B699B904688CB102790F2A0ED84F
:10FF500043490B8843FA02F5EF070AD502F1007610
:10FF600006F59067B4EB471F03D162B6F0BD3C497C
:10FF70000B8813F0010226D09E0757D55D0757D591
:10FF80001C0757D5DA0657D59F0657D55E0657D5B5
:10FF90001D0657D5DC0557D59A0557D55F0557D5AA
:10FFA0001E0557D5DD0457D59C0457D55A0409D5ED
:10FFB000DA0B08BF0F2206D062B6002410220460BC
:10FFC0000271F0BD0E22012595402B430B8062B6D5
:10FFD000244E254D254FDFF89CE0D1B201713368E6
:10FFE00043F00204346002F1007C2A68A6F5802602
:10FFF00042F002042C600CF59063283EDFF878C0D4
:020000021000EC
:100000001B4C5B0140F28245CEF8005039708CF8F1
:10001000001000273170217003601F605F609F60D7
:10002000DF601F615F619F61DF61F0BD0122CAE790
:100030000222C8E70322C6E70422C4E70522C2E77A
:100040000622C0E70722BEE70822BCE70922BAE77A
:100050000A22B8E70B22B6E70C22B4E70D22B2E77A
:10006000A4E00120408004403C8004401A8000400D
:100070001F800040008000401E80004000B5064AFE
:10008000036811885B6883B00222ADF8041001A9EF
:10009000984703B05DF804FB0C35040010B5036805
:1000A00014465B689847204610BD00BF0EB400B5EB
:1000B00082B003AA52F8041B019204F0B5FC02B00E
:1000C0005DF804EB03B0704730B314490B6833B9E3
:1000D000134B0B60B3FBF0FC00FB1C30704770B49B
:1000E000104C114A114E84FB035C9C44DD17C5EB98
:1000F0002C4402FB143206FB04F444F2A71303FB66
:100100000245002D02DA05F10046751E0D60B5FBB3
:10011000F0F100FB115070BC704700BFA8E0012057
:1001200042CE0C1F5F0B4E831DF30100ECF4FFFF6A
:1001300008B5FFF74FFCFFF73BFDFCE7844641EABB
:10014000000313F003036DD1403A41D351F8043B4F
:1001500040F8043B51F8043B40F8043B51F8043BA1
:1001600040F8043B51F8043B40F8043B51F8043B91
:1001700040F8043B51F8043B40F8043B51F8043B81
:1001800040F8043B51F8043B40F8043B51F8043B71
:1001900040F8043B51F8043B40F8043B51F8043B61
:1001A00040F8043B51F8043B40F8043B51F8043B51
:1001B00040F8043B51F8043B40F8043B51F8043B41
:1001C00040F8043B51F8043B40F8043B403ABDD2B0
:1001D000303211D351F8043B40F8043B51F8043B52
:1001E00040F8043B51F8043B40F8043B51F8043B11
:1001F00040F8043B103AEDD20C3205D351F8043BE1
:1002000040F8043B043AF9D2043208D0D2071CBFAC
:1002100011F8013B00F8013B01D30B8803806046D5
:10022000704700BF082A13D38B078DD010F003034B
:100230008AD0C3F10403D21ADB071CBF11F8013BBB
:1002400000F8013B80D331F8023B20F8023B7BE70A
:10025000043AD9D3013A11F8013B00F8013BF9D235
:100260000B7803704B7843708B78837060467047CF
:1002700008B5104C08E0206841050DD421680A0536
:100280000FD42268D30411D423685803F3D500F0A7
:1002900025FF20684105F1D502F0BEFA21680A0564
:1002A000EFD502F0C7FB2268D304EDD502F0D0FCF5
:1002B000EAE700BF3480044008B5FFF7D9FF00BF6C
:1002C000014B10221A80704700200540704700BF84
:1002D000094908B50B6830B16A461844A2F5005CBC
:1002E000604502D20860184608BD03F0E7FC0C2107
:1002F00001604FF0FF3008BD6427FF1F0078B0FA9F
:1003000080F14809704700BF01230370704700BFA8
:10031000084A1378802B01D0002070470649074B0C
:1003200007480860002119701378802BFCD0012049
:10033000704700BF03E007404480044001E00740ED
:10034000000028220A4A1378012B01D000207047B0
:1003500003F1804000F5FC2C60218CF8001013782C
:10036000802BFCD10348044A02600120704700BF83
:1003700003E00740448004400000060203F0CCBCC8
:1003800003F0D2BCF0B44D1E2E46002400E0013430
:10039000B0FBF2F302FB1300092800F130078ABF1B
:1003A0003730F8B2C0B206F8010F1846002BEED174
:1003B0000A1953704CB10133E01A15F801CF1678C1
:1003C0002E70834202F801C9F5DB0846F0BC704785
:1003D000704700BF3F28F0B445D8042A43D8DFE86F
:1003E00002F0474A4D0344004FF410252D4C04EB16
:1003F000C0035B681A6812F4E06648D02A4A2B4EA4
:100400002B4CC2F8306103F1404CACF592262948E0
:10041000294FC2F82C417C2E284CC2F83401C2F876
:100420003871C2F83C412CD9ACF594227C2A2AD9E7
:10043000ACF596207C2828D9ACF598277C2F2ED9AE
:10044000ACF59A247C2C0ED81D4E72B61A6822F494
:10045000702747F08070C3F3840C28431F6046F870
:100460002C10186062B6F0BC70474FF43025BDE721
:100470004FF40025BAE74FF44025B7E74FF42025A5
:10048000B4E7104EE1E7104EDFE7104EDDE754F819
:1004900030704FF4807087F880621860AEE70C4EC1
:1004A000D3E700BF103504000002FF1FCD21FF1F5E
:1004B000FD21FF1F9D21FF1F6D21FF1F3D21FF1FFC
:1004C000B028FF1F6827FF1FE027FF1F4028FF1FDE
:1004D0007028FF1F30B4054B054D064C002210213B
:1004E0001A602A602060196030BC704714D0034045
:1004F00004D0034000D003402DE9F843944B9548C5
:10050000954D964E964C9749DFF87CC2DFF87CE219
:10051000954F4FF000621A604FF080521A604FF012
:1005200000521A604FF080421A604FF000421A6089
:100530000022026028234EF6FF70CCF8000006F57A
:100540000028CEF8003005F5002C23600EF5012EB2
:100550000B6033602B603B60A36207F500278B6262
:1005600004F5012401F501210EF1100608F6E879E1
:100570000CF6E87507F57F6810312034C9F80030B3
:100580002B603360C8F800300B602360774CC8F8EC
:100590001830A8F5002C04F58057ACF1200E083770
:1005A0008B610921216007F5FD28CEF80020386015
:1005B000CEF80830FB600EF5FE2708F2FC74043715
:1005C0004EF8041C22603860A360FB6044F8041CF1
:1005D000083404F6FC7CC7F8FC2FCCF80000ACF51E
:1005E000E120A0F2DC78C9F800302B60C7F8F81FD2
:1005F000D8F800105E4841F40074C8F80040016863
:1006000006F57F4606F1E80E41F0007407F58837DD
:1006100009F5803905F58035564E0460CEF8002086
:1006200047F6FF7008223860C9F800302B6032604E
:1006300002F036F872B6504B504C514F1E68256888
:10064000396862B6490102D5322E88BF0135C6F538
:100650002F3C0CF21F304B4FDFF81C91DFF820814C
:1006600083084FF47A72A7FB031602FB05F505EB2E
:100670009605322672B6D9F800102268D8F800E044
:1006800062B6C1F52F3C0CF21F308308A7FB030CA8
:100690001EF0806FC5EB9C034FF47A7002D03229B4
:1006A00088BF013200FB0231B1F57A7F04D3013EED
:1006B00005D005F57A75DDE701F00AFEDAE701F00D
:1006C0005FFA72B62C4B2E4A18682668116862B61B
:1006D0004A0102D5322888BF0136C0F52F3E0EF2FE
:1006E0001F35284FDFF89090DFF89480AB084FF467
:1006F0007A7202FB06F6A7FB031006EB90054FF497
:10070000AF7672B6D9F800102268D8F800E062B669
:10071000C1F52F3C0CF21F339808A7FB000C1EF00C
:10072000806FC5EB9C034FF47A7002D0322988BFEA
:10073000013200FB0231B1F57A7F04D3013E05D0CE
:1007400005F57A75DDE701F0C3FDDAE7BDE8F8836A
:1007500004E100E0048003402C8003402480034037
:10076000148003401C800340348003400080034019
:100770000480044000900C4018E000E0ACE0012050
:1007800004ED00E0176CC116088003400C800340A4
:10079000A0F14203012B51D911B93F2864D9704708
:1007A00010B4A04A92F800C0012202FA0CF4A1424F
:1007B00050D2C31E012B40F2BD81A0F11D02012ABF
:1007C00040F2BF810E2800F28A8044F28414C440B3
:1007D000E20740F18480944A146804FB011323FA71
:1007E0000CF3A0F1020CBCF1240F00F28381DFE8CE
:1007F0001CF07A01730111010A010301FC00F500EC
:10080000EE00E700810181018101E0008101D90052
:10081000D20081018101CB00C400BD00B60081017E
:100820008101810181018101AF00A8008101810165
:1008300081018101A1009A0093008C00794B1A7804
:100840000B2A0CD8C2F10C0399404228084624D048
:1008500001F0B4BF3F2822D95DF8044B70470C2A41
:100860001CBF0C3AD140F0E7704B53F8302092F89F
:10087000801203EBC00C59B30120DCF8043082F87D
:1008800000014FF0010C4FF4A27182F880C2196090
:100890001A6822F020001860704701F071BF634BA6
:1008A00053F8301091F8804203EBC00C44BBDCF8E5
:1008B00004301A6842F00300186001244FF4A27259
:1008C00081F880421A60196821F020001860C3E79F
:1008D000DCF80430186820F002011960D1E7A0F1BB
:1008E0002303032B7FF677AFA0F11002012A94BFF8
:1008F0004F4A504A146804FB011323FA0CF370E7C3
:1009000081F88020DCF80430D7E74B494B480B6076
:100910004FF4517202609FE7494C4A4923604FF4FB
:1009200051730B6098E74848484A03604FF451748C
:10093000146091E7464947480B604FF451730360D8
:100940008AE7454C454A23604FF45171116083E7B3
:100950004348444C03604FF4517323607CE74249A1
:10096000424A0B6040F24440106075E7404C4149F8
:10097000236040F244430B606EE73F483F4A036008
:1009800040F24444146067E73D493E480B6040F242
:100990004443036060E73C4C3C4A236040F24461BE
:1009A000116059E73A483B4C036040F244632360CE
:1009B00052E73949394A0B6040F2444010604BE736
:1009C000374C3849236040F244430B6044E73648D3
:1009D000364A036040F2444414603DE734493548E8
:1009E0000B6040F24443036036E7334C334A2360E4
:1009F00040F2444111602FE73148324C036040F22D
:100A00004443236028E73049304A0B6040F24440B9
:100A1000106021E72E4C2F4923604FF451730B6077
:100A20001AE700BF1C29FF1F08900B401035040077
:100A300008900C400880034048900B402CB00440C4
:100A400040900B4028B0044038900B4024B0044044
:100A500030900B4020B0044018800B404CA0044064
:100A600010800B4048A004401880034008B00440A8
:100A70001080034004B004404080034018C004408C
:100A80003880034014C0044018900C4004A0044077
:100A900010900C4000A0044018900B4004C004408B
:100AA0002880034010B00440208003400CB0044074
:100AB00028900B400CC0044020900B4008C004401C
:100AC0003080034010C00440488003401CC00440F4
:100AD00018900340349004402348244A03604FF4A4
:100AE00051741460B8E6224922480B6040F2444336
:100AF0000360B1E63F283FF6AFAE1F4C54F83020FC
:100B000092F8803223B37F294FF0010C4FEAC003E3
:100B10008CBF82F880C082F800C1234401245B6846
:100B200082F880424FF4A2721A60186820F0200107
:100B3000196091E6114A146804FB011323FA0CF3BF
:100B40004FE60F4A146804FB011323FA0CF348E63E
:100B5000C300E0187F29406801688CBF41F00301A1
:100B600021F002010160D8E710900340309004406A
:100B700010900B4000C00440103504000890034062
:100B800008800B4038B1102828BF1020044AC3B297
:100B9000107813707047024A012310781370704761
:100BA0001C29FF1FA0F11002D2B2012A70B440F23A
:100BB000A280DFED647A6449B4EEE70AF1EE10FA40
:100BC00047F612234EBF10210B46082100EE903A43
:100BD0009FED5E7AB8EEE01A61EE076AB4EEE60ABF
:100BE000F1EE10FA80F29E805C0801EE104AB8EE39
:100BF000C11A61EE071AB4EEE10AF1EE10FA80F2C2
:100C000093809E0802EE106AB8EEC21A61EE072ABF
:100C1000B4EEE20AF1EE10FA80F28880DC0803EE0E
:100C2000104AB8EEC31A61EE073AF4EEC03AF1EE9C
:100C300010FA7DD91E0904EE106AB8EEC41A61EEEE
:100C4000074AB4EEE40AF1EE10FA73DA5C0905EE35
:100C5000104AB8EEC51A61EE075AB4EEE50AF1EE95
:100C600010FA69DA9E0906EE106AB8EEC61A61EE4D
:100C7000070AB4EEE00AF1EE10FAA8BF062505DA7D
:100C8000DD0907EE905AB8EEE71A072581EE007AE3
:100C90004FF6FF7CC31EB6EE000A77EE406AFCEE0C
:100CA000E61A11EE904A644528BF6446012B35D9F7
:100CB00017280ED9A0F11D03012B3FD90E281DD9ED
:100CC000233803281FD9012A13D8214B214E22484B
:100CD0001CE0224EC64006F0010383F00106002B03
:100CE000E8D01F4B1F48204A1E602943066014604D
:100CF000196070BC70471D4B082167E744F28416E9
:100D0000C640F307DCD51A4B1A4E1B482943002571
:100D10001D6035600460196070BC7047174B184E39
:100D20001848F3E70025B1E70125AFE70225ADE755
:100D30000325ABE70425A9E70525A7E7124B134ECA
:100D40001348E3E7C0E1E4400087930300008037E5
:100D500000900C4004900C4008900C406006F0009D
:100D60000080034004800340088003400024F40016
:100D700000900B4004900B4008900B400090034003
:100D8000049003400890034000800B4004800B4017
:100D900008800B403F2806D8044B53F8300090F8E9
:100DA0000012C8B270470020704700BF1035040021
:100DB0003F2820D81B4A02EBC00301295B680FD0F3
:100DC00004291DD052F83000002280F8802299B109
:100DD000022923D003290DD14FF481711960704786
:100DE00052F830004FF4A27280F880121A6019682D
:100DF00021F020021A6070474FF48070186070472D
:100E000052F830104FF0010C4FF4A27281F880C2FA
:100E10001A60186840F020011960704740F2031210
:100E20001A6070471035040072B60D490D4A0E4B1A
:100E30001B680868116862B64A0102D5322B88BF68
:100E40000130C3F52F3C0CF21F32084993084FF4D0
:100E50007A72A1FB031C02FB00F000EB9C007047C0
:100E6000ACE0012004ED00E018E000E0176CC116D2
:100E70002DE9F843054672B6224B234F234A1868E2
:100E80003C68116862B64A0102D5322888BF013435
:100E9000B5B3C0F52F3606F21F331D4EDFF8649050
:100EA000DFF8688098084FF47A72A6FB001C02FBFA
:100EB00004F404EB9C0472B6D9F800103A68D8F830
:100EC00000E062B6C1F52F3303F21F308308A6FBA2
:100ED000030C1EF0806FC4EB9C034FF47A7002D0B9
:100EE000322988BF013200FB0231B1F57A7F04D389
:100EF000013D05D004F57A74DDE701F0E9F9DAE7A0
:100F0000BDE8F88318E000E0ACE0012004ED00E06B
:100F1000176CC116431E032B14D872B60A4951F838
:100F2000230068B170B4094C058834F81320466872
:100F300041F82360511B24F8131062B670BC70474F
:100F400062B670470020704708E1012000E50120EB
:100F5000013803280BD872B6074B53F8201041B163
:100F60000020496801300029FBD162B6704700209B
:100F700070470846F9E700BF5CE1012030B472B663
:100F80002F4A13781D0706D52E4B196A00293BD02E
:100F90009C6A002C48D055782C0706D5294B196C33
:100FA000002947D09C6C002C41D092F802C05FEA27
:100FB0000C7105D5234B1D6E002D3DD0996E99B156
:100FC000D278130709D51F4BD3F88040002C35D0B9
:100FD000D3F888504FF0110C45B162B61A4B00217E
:100FE000197030BC00F084BE4FF00D0C164C174D3C
:100FF000217843F83C5003EBCC0308304A1E58607C
:10100000227062B630BC704704220F4C104D94F829
:1010100000C043F8325003EBC20108300CF1FF333B
:101020004860237062B6EDE74FF0050CDEE74FF045
:10103000090CDBE70822E8E70C22E6E71022E4E7E8
:10104000383704000000FF1F85E10120C800400080
:1010500088004000431E032B1FD81C4A400140F06B
:10106000100030B4104472B6194C14F803C0BCF12F
:10107000030F1BD8DFE80CF00212151703220D88AE
:10108000E25410F0080F14BFC823882343EA054335
:1010900008310360416062B630BC704708300222FC
:1010A000EDE70522EBE708300422E8E7094C54F8A5
:1010B000230038B1084A52F82350696042F82310DF
:1010C00062B6E9E744F82310034AF7E70000FF1F80
:1010D00094E101205CE101206CE101202DE9F04F59
:1010E000DFF82093DFF820A3DFF820B385B044E0D9
:1010F000B24D9E0805EBC60708F1FF3C7A6803F085
:1011000008015FFA8CF4A2F1080001F0FF0E00293B
:1011100040F0068155F836301B0C1FFA83F822F890
:10112000088C002B00F0F380A54922F806EC51F85A
:10113000243042F804EC002B00F0C282A14951F89F
:1011400024205060A04A41F8240032F814E0F04412
:1011500022F8148000F0ACFD002800F0AA829B4B1E
:101160009B4C17F0080F00F1080018BF1C46786070
:1011700045F83640082189F8001099F80040E6B299
:1011800075071CD5934B1878B0B193490A7802F0D3
:10119000FF0522B16F1EFCB20C7004B900BE8F486F
:1011A000017801F0FF0839B108F1FF3C5FFA8CF3D8
:1011B0000370002B00F05282042289F8002006F010
:1011C000080505F0FF02002D00F0D2809AF800001B
:1011D000C3B25FEA13188BD19808DFF8E08158F8A2
:1011E000305008EBC006C5F383077A1E71680C2ADD
:1011F00000F28980DFE802F07D7D87878787878717
:101200004587878707000F68754E704B4C6848F814
:101210003030BDB240F2816C724873497460002274
:101220000124654537600260C8F81020C8F818200E
:101230000C70624F00F2F080B5F5D06F80F03B8308
:10124000B5F5817F00F0F48200F28C82802D00F0F1
:101250006983822D40F0F282B38803F07F01042974
:1012600000F2EC82614D62488F003D440270427092
:1012700095F800E05FEA8E7540F14B84047002241B
:1012800034E3584E326842B3DFF884C1564BBCF8A1
:101290000010584F1C78387840290D4628BF40254B
:1012A000491B002C40F0020E84F0010489B21C702E
:1012B000ACF800100CBF8824C82408EBCE0C80F0DA
:1012C000010044EA0543CCF8042048F83E302A44A3
:1012D0003870002900F046813260414EB6F8008037
:1012E000B8F5A06F0FD1444DB278002777702A70FF
:1012F00009E03B4C238842F22106B34200F03681DC
:10130000324C48F8304001208BF8000032E72F4A79
:101310002F4817F0080F18BF104645F8360029E788
:1013200000F0E6FC354A52F82430002B00F0CC8166
:10133000DFF8E0E058681EF804C042F8240003F12A
:1013400008027A60BCF1030F07D8DFE80CF0320224
:101350002E2A4FF002080EF804801C8817F0080FA0
:101360000CBF8823C82343EA044345F8363001E71D
:10137000F00700F17681310600F1B681B20708D599
:101380001F4D204A95F8009002275FFA89F32B70D1
:101390001770F30602D51B4E1024347005B0BDE85B
:1013A000F08F04210EF80410D7E705200EF8040092
:1013B000D3E74FF0030C0EF804C0CEE70000FF1F88
:1013C00008E10120B4E0012000E50120C800400050
:1013D0008800400090E1012019E1012098E10120FE
:1013E0007CE10120B0E0012018E10120C02007408D
:1013F00088E1012084E10120982007405CE1012080
:101400008820074080200740902007409420074014
:10141000C4E0012094E1012042F22100854200F065
:10142000198100F2CE80B5F5086F00F05B82B5F54A
:10143000106F40F003823D6AB049B6780E702C06FA
:1014400000F1F782D8F82840AD4A200600F1EB827F
:10145000D8F83000AA49020600F1DF82D8F83860D7
:10146000A74F330600F1D382D8F84020A44B1706CB
:1014700000F13083D8F84850A1492E0600F12483AA
:10148000D8F850709E4C3D0600F11883D8F85830BB
:101490009B481C0600F10C83D8F860609849300620
:1014A00000F10083D8F86840954B220600F1F482E1
:1014B000D8F87000924D030600F1C782D8F8787012
:1014C0008F493F0600F1BB82D8F880308C4A1E0657
:1014D00000F11983D8F88850894E2D0600F10C834D
:1014E000D8F890408649240600F1FF82D8F8982069
:1014F000834D100600F1F382824C834E8349844F62
:1015000003940025019602912C46386828B146685C
:1015100000F0EEFB3046002EF9D1019B7D4A1868A1
:101520003C6042F8254028B1466800F0E1FB3046B7
:10153000002EF9D10298039B90F800E0019943F83E
:10154000044B754A0C60AEF1020C039322F815406F
:10155000BCF1030F00F22581DFE81CF067011F01D9
:1015600067011F01402D18BF0022B5E66B4F0A78B6
:101570004C788D78CB783A707C70BD70FB703E688B
:101580000A794C7989793A71862E7C71B97100F0AB
:101590008E81634B634C93F800C021784CF00202BB
:1015A00000298CF001061E700CBF8823C82348F860
:1015B000323008EBC20381F00107002527705D601F
:1015C0009EE642F221239D4240F0B781564F574B91
:1015D0005749B0783E681E600870002101918C4622
:1015E0008E4608464E4E357845F0020708EBC70395
:1015F000002C58600CBF8820C82040EA0C0348F833
:101600003730484BDFF818C11A7085F00100307090
:10161000002940F01A81BEF1400F1BD140F0020CAE
:1016200008EBCC030198DFF8D8E05860002A40F0BE
:1016300021810F0447F088023A4B4EF83C200844C1
:101640001C7035700746402904D10021394C3A4EB0
:101650002180376001258BF8005054E600F012FE1F
:10166000AAE5274B35482E491A614FF0020E80F843
:1016700000E0334F0A70334919609960324E334DA0
:10168000334C9A610D213970FF213170DFF8D0E0C1
:10169000297022702F4D304A8EF800104FF09F0AAB
:1016A000012706F804AC5D600770DA6005B0BDE89C
:1016B000F08F2A4F45F836003D7801353D7059E5E9
:1016C00041F8240013493DE5104E305D032800F237
:1016D000E78001A151F820F075110100751101009A
:1016E000951701008F170100154F184C0D20802110
:1016F000B207387021707FF54CAE41E690E10120D1
:101700000000FF1F6CE101205CE1012094E1012059
:1017100008E10120B4E0012000E5012008E50120F6
:1017200084E1012018E10120ACE0012010E5012056
:10173000A8E10120C4E00120B0E00120942007408E
:10174000C0200740880040008820074080200740D4
:1017500098200740C8E001201CE1012085E101201C
:101760008C20074040F20232954240F0E080B08881
:1017700000F07F03042B61D87288002A5ED1B64E38
:1017800099000E44357845F00207377025E70121AE
:101790003155EFE400273755ECE4029E4FF001008D
:1017A0003070019B029A013504330132042D07F198
:1017B0000407019302927FF4A8AEA84CA84D2778A5
:1017C000A84800263A072E70077000F1F58060786F
:1017D000A549A64F08700023C8F83030C8F8383043
:1017E000030700F1D480A378A14AA04E1370002112
:1017F0001F07C8F85010C8F8581000F1F380E778B8
:101800009C499A4C0F7000233E07C8F87030C8F806
:10181000783000F1A48098490C78002384F001020C
:10182000C8F89030C8F89830D7E602990C70B8E73D
:10183000B28802F07F03042B40F28480864A0F2591
:10184000157001258BF800505DE540297FF6E6AE66
:10185000864E019F40F0020806EBC8004760A2B127
:101860008CF80050814D854E1C704039403745F84A
:101870003860EBE60804804B019F1C7040F0C80202
:1018800035700F444EF83C20DDE61C70019F774C0C
:101890007B4A8CF800504039403744F83820D5E670
:1018A00017F0080F0CBF02200320305562E4754F7B
:1018B0000F253D706DE6744F78680028BED074889F
:1018C000B58803E00C3778680028B7D03A88A24280
:1018D000F8D17B88AB42F5D1240A032C0CBF0478E5
:1018E0003C8903E0694A6A4817780770B6F806C071
:1018F000A44580F03581674E357845F0020708EB46
:10190000C701BCF1400FE64628BF4FF0400E4860CB
:1019100070440190CEEB0C0100224FEA0E4C0124E2
:10192000C8206AE65A48022402704270DEE7B5F524
:10193000A06F83D1002201244FE642F22136B54246
:10194000F8D07BE77288002A7FF478AF42489E0087
:10195000304490F800C02CF0020101703DE600F028
:10196000A7F9002800F0EF800830C4F8840044484C
:10197000C8F8800000F09CF93C4E002800F0DD80A3
:1019800008303E4DC6F88C00C6F8885043E700F09A
:101990008FF9002800F0C480083078643848C8F80F
:1019A000400000F085F9314E002800F0B480083086
:1019B000324FF064B76416E700F07AF9002800F0BF
:1019C000CB800830C8F824002D48C8F8200000F06B
:1019D0006FF9264B002800F0BA800830274ED862F5
:1019E0009E62F4E600F064F9002800F0A28008305E
:1019F00070662348C8F8600000F05AF91B4B0028B5
:101A000000F0928008301D4ED8669E66F7E6FC6BAB
:101A1000A4F1080000F06CF926E54D6BA5F1080073
:101A200000F066F91AE5D36AA3F1080000F060F946
:101A30000EE57F6AA7F1080000F05AF902E5CC6FC5
:101A4000A4F1080000F054F93EE56E6FA6F108001D
:101A500000F04EF932E500BFC020074038370400DF
:101A600085E10120C4200740C82007400000FF1F77
:101A7000CC200740D020074018E10120C8004000DA
:101A80008800400019E101203C37040090E101206A
:101A900088E1012084E10120DA6EA2F1080000F063
:101AA00027F905E54F6EA7F1080000F021F9F9E4E8
:101AB000C56DA5F1080000F01BF9EDE4626DA2F11F
:101AC000080000F015F9E1E4CE6CA6F1080000F082
:101AD0000FF9D5E4586C083800F00AF9CAE4D5F8D3
:101AE0009C00083800F004F906E5D1F89430A3F121
:101AF000080000F0FDF8F9E4D6F88C70A7F10800B2
:101B000000F0F6F8ECE4D2F88400083800F0F0F8C1
:101B1000E0E40224EAE62978B064481C287062E612
:101B20002A7801322A703AE72A789866501C287081
:101B300065E62F7801372F705CE72F78C6F88800AC
:101B4000781C287067E62A7801322A7010E72A7814
:101B50009862571C2F703AE629780131297034E7D2
:101B6000402CA64628BF4FF0400ECEEB040100EB00
:101B70000E0401944FEA0E4C0022012432E500BF0E
:101B80002DE9F04101F05CFA324C334B3348DFF879
:101B9000E880DFF8E8C0324E324FDFF8E4E00022A0
:101BA0001A605A609A60DA601A615A619A61DA6161
:101BB0001A625A629A62DA621A635A639A63DA6341
:101BC0001A645A649A64DA641A655A659A65DA6521
:101BD0001A665A669A66DA661A675A679A67DA6701
:101BE000C3F880202168C3F8842041F48025256053
:101BF00001681D4D41F040710160032088F800002C
:101C0000C3F30721C3F3074004F528341B0E4FF03C
